:100000000C947B080C94CA080C94CA080C94CA0877
:100010000C94CA080C94CA080C94CA080C94CA0818
:100020000C94CA080C94711B0C94CA080C94CA084E
:100030000C9474350C94CA080C94CA080C94CA0821
:100040000C94CA080C94CA080C94DB170C94CA08C8
:100050000C94090E0C94CA080C94D30D0C94CA0885
:100060000C94541E0C94CA080C94FA300C94CA08D0
:100070000C9411890C94CA080C9403820C94CA083D
:100080000C94CA080C94CA080C94CA087B1E801EE3
:10009000851E8E1EA51EBC1ECC1EDC1E171F002139
:1000A000BC1EC21FD31F022020203D209720F2201B
:1000B0000D23DA236924E9242125C425CB273528FB
:1000C000AF28F828422970299D29002A4A2A942A13
:1000D0008D2B19314D319031003218325932103395
:1000E000D733D733D733D733D733D733D733D733C0
:1000F000D733D733D7338C338E339333AB33AD33DE
:100100001074A9742E759075E4754D76A27DCE7627
:10011000F276F676F676F676F676F676F676F67683
:10012000F67624779F77347859789C78F8788379B5
:100130006C7AC57AC97AC97AC97AC97AC97AC97A08
:10014000C97AC97A017B1F7B447BA07BDC7B4B7C1B
:10015000787C187D787D7D7D7D7D7D7D7D7D7D7D3F
:100160007D7D7D7D7D7D64876787678767877087F5
:1001700073877687888785870A0D3D3D3D3D3D3DE8
:100180003D3D3D3D3D3D3D3D3D3D3D3D3D3D3D3D9F
:100190003D3D3D3D3D3D3D3D3D3D3D3D3D000A0D2F
:1001A000426174743A002025642043656C6C7320AE
:1001B00000204C6F77207761726E696E673A202558
:1001C000642E2564000A0D466F756E6420424C2D26
:1001D0004374726C3A20002564000A0D0A0D212137
:1001E000204D495353494E4720424C2D4354524CC5
:1001F0003A202564202121000A0D43616C69627256
:100200006174696E672070726573737572652073AF
:10021000656E736F722E2E004F4B0A0D000A0D464D
:100220006C696768742D74696D65202575206D692A
:100230006E20546F74616C3A2575206D696E0041B3
:100240006E676C654E69636B202020202020204162
:100250006E676C65526F6C6C20202020202020413E
:1002600063634E69636B20202020202020202041E2
:100270006363526F6C6C20202020202020202059A6
:1002800061774779726F202020202020202020488D
:1002900065696768742056616C756520202020416F
:1002A00063635A2020202020202020202020204767
:1002B0006173202020202020202020202020204387
:1002C0006F6D706173732056616C756520202056C8
:1002D0006F6C74616765205B302E31565D20205253
:1002E00065636569766572204C6576656C2020478C
:1002F00079726F20436F6D70617373202020204DE1
:100300006F746F7220312020202020202020204D6B
:100310006F746F7220322020202020202020204D5A
:100320006F746F7220332020202020202020204D49
:100330006F746F7220342020202020202020203154
:100340003620202020202020202020202020203186
:100350003720202020202020202020202020203175
:100360003820202020202020202020202020203164
:100370003920202020202020202020202020205331
:100380006572766F20202020202020202020204809
:100390006F76657267617320202020202020204323
:1003A000757272656E74205B302E31415D20204382
:1003B00061706163697479205B6D41685D202048DC
:1003C000656967687420536574706F696E74203254
:1003D00035202020202020202020202020202032F6
:1003E00036202020202020202020202020202043D4
:1003F0006F6D7061737320536574706F696E7449AB
:1004000032432D4572726F7220202020202020421E
:100410004C204C696D69742020202020202020472A
:1004200050535F4E69636B202020202020202047FE
:1004300050535F526F6C6C20202020202020202100
:10044000212120494E434F4D50415449424C4520B3
:10045000212121002A002E000A0D20444143206F53
:100460007220493243204552524F52212043686541
:10047000636B204932432C2033567265662C20442E
:10048000414320616E6420424C2D4374726C005BCA
:1004900025695D005B25695D002B204D696B726FDE
:1004A0004B6F70746572202B0048573A5625642EA6
:1004B00025642053573A25642E256425630053652F
:1004C0007474696E673A2564202573004D697865F8
:1004D00072204572726F7221004552522532643A81
:1004E000004861726477617265204572726F722094
:1004F000313A2564202121004D697373696E6720AC
:10050000424C2D4374726C3A2564212100493243D8
:10051000204552524F522121210048656967687475
:100520003A202025356900536574706F696E743AFE
:100530002535690050726573737572653A253569A2
:10054000004F66667365743A20202535690048655A
:100550006967687420636F6E74726F6C00444953EE
:1005600041424C4544006163742E206265617269AA
:100570006E67004E69636B3A2020202020202535CD
:100580006900526F6C6C3A202020202020253569AC
:1005900000436F6D706173733A2020202535690028
:1005A0004B25693A25346920204B25693A25346961
:1005B00020004E693A2534692020526F3A2534696B
:1005C000200047733A253469202047693A25346969
:1005D000200050313A253469202050323A253469C0
:1005E000200050333A253469202050343A253469AC
:1005F00020004779726F202D2053656E736F720053
:100600004E69636B25346920282533692E256929B5
:1006100000526F6C6C25346920282533692E2569BA
:100620002900476965722534692028253369290026
:100630004E69636B2025346920282533692E25787F
:100640002900526F6C6C2025346920282533692ECF
:100650002578290059617720202534692028253301
:100660006929004E69636B20253469202825336988
:1006700029282533692900526F6C6C2025346920A4
:1006800028253369292825336929005961772020D5
:100690002534692028253369292825336929004113
:1006A0004343202D2053656E736F72004E69636B58
:1006B0002025346920282533692900526F6C6C206D
:1006C000253469202825336929005A202020202537
:1006D000346920282533692900566F6C7461676579
:1006E0003A2020202533692E253169560043757242
:1006F00072656E743A2020202533692E25316941B8
:1007000000506F7765723A202020202025346957E9
:10071000004469736368617267653A202535696DC5
:1007200041680052656365697665720052432D52D7
:100730005353493A202020202534690052432D513B
:1007400075616C6974793A202534690052432D43F0
:1007500068616E6E656C733A25346900436F6D7025
:10076000617373004D61676E65743A2020202535F2
:1007700069004779726F3A202020202025356900D2
:10078000536574706F696E743A2025356900506F37
:10079000746925693A202025336900506F746925F2
:1007A000693A202025336900536572766F20200056
:1007B000536574706F696E74202025336900506F23
:1007C000736974696F6E3A202533690052616E67F0
:1007D000653A2533692D25336900424C2D437472E7
:1007E0006C204572726F72732000253364202533AC
:1007F0006420253364202533642000424C20546556
:100800006D706572617475726500253364202533DF
:100810006420253364202533642000424C2D43742A
:10082000726C20666F756E64200020256320202086
:1008300025632020202563202020256320002025FB
:10084000632020202563202020256320202025638D
:1008500020002025632020202D2020202D20202056
:100860002D2000313000313100313200466C696793
:1008700068742D54696D65202000546F74616C3A62
:100880002535756D696E004163743A2020253575F4
:100890006D696E0028726573657429000A0D4765DD
:1008A0006E65726174696E672064656661756C74EB
:1008B00020506172616D65746572205365742025E6
:1008C00064000A0D5573696E6720506172616D6531
:1008D00074657220536574202564000A0D47656EA7
:1008E00065726174696E672064656661756C7420F9
:1008F0004D69786572205461626C65000A0D4D691E
:100900007865722D436F6E6669673A2027257327D5
:1009100020282575204D6F746F727329000A0D41D0
:100920004343206E6F742063616C69627261746509
:1009300064210D0A0000008F001E01AD013B02CAB8
:10094000025803E603740402058F051B06A706334D
:1009500007BE074808D2085B09E3096B0AF20A7868
:100960000BFD0B810C040D860D070E870E060F8400
:100970000F00107B10F5106E11E5115B12CF1242C3
:1009800013B31323149214FE146A15D3153B16A146
:100990001605176717C81727188318DE1837198E1A
:1009A00019E319361A871AD61A231B6E1BB61BFDBC
:1009B0001B411C831CC31C001D3C1D751DAB1DE091
:1009C0001D121E421E6F1E9A1EC31EE91E0D1F2EF3
:1009D0001F4D1F691F841F9B1FB01FC31FD31FE123
:1009E0001FEC1FF51FFB1FFF1F00204E6F204572DD
:1009F000726F722020202020202020004E6F742053
:100A0000636F6D70617469626C652020004D4B33BB
:100A10004D6167206E6F7420636F6D7061004E6F63
:100A200020464320636F6D6D756E69636174004D80
:100A30004B334D616720636F6D6D756E6963610047
:100A400047505320636F6D6D756E69636174696F94
:100A500000636F6D706173732076616C7565202023
:100A600020005243205369676E616C206C6F737471
:100A700020200046432073706920727820657272CE
:100A80006F7220004E6F204E4320636F6D6D756E48
:100A900069636174004643204E69636B2047797235
:100AA0006F2020202000464320526F6C6C20477935
:100AB000726F20202020004643205961772047791B
:100AC000726F2020202020004643204E69636B2057
:100AD000414343202020202000464320526F6C6C6D
:100AE000204143432020202020004643205A2D410E
:100AF0004343202020202020202000507265737363
:100B00007572652073656E736F72200049324320E1
:100B100046432D3E424C2D4374726C2000426C20A3
:100B20004D697373696E67202020202020004D6975
:100B3000786572204572726F722020202020004359
:100B400061726566726565204572726F7220200061
:100B500047505320466978206C6F73742020202002
:100B6000004D61676E6574204572726F722020209F
:100B700020004D6F746F72207265737461727420FF
:100B8000202000424C204C696D69746174696F6E5D
:100B9000202020004750532052616E67652020209E
:100BA00020202020004E6F2053442D43617264208A
:100BB00020202020200053442D4C6F6767696E670A
:100BC000206572726F7200466C79696E672072617F
:100BD0006E676521202020004D617820416C74698A
:100BE00074756465212020200020202020202020F2
:100BF0002020202020202020202020202020002015
:100C0000202532692E2531695620200020202532EA
:100C1000692E25316956202000414C543A2534690B
:100C20006D20256300414C543A2534696D20200025
:100C3000414C543A2D2D2D2D200020202532693A8B
:100C40002530326920200020202532693A253032B3
:100C5000692020004449523A20253364256300432B
:100C6000002000202025356920200020202535691E
:100C7000202000493A2532692E2531694120003A69
:100C8000003A003A002D2D2D2D2D2D2D2D2D2B2D03
:100C90002D2D2D2D2D2D2D2D2D2D002D2D2D2D2DB1
:100CA0002D2D2D2D2D2D2D2D2D2D2D2D2D2D2D2D74
:100CB000003A005341543A253264200044495354C9
:100CC0003A2533646D004420003344002121004D57
:100CD00041473A25337525252000484D3A25336490
:100CE000256320256300696E636C3A2532642563B1
:100CF000282532692900202020202532756D2F7388
:100D00003A2020484D3A2533642563202563004569
:100D100052523A202532642021004552523A200096
:100D2000207777772E4D696B726F4B6F7074657299
:100D30002E6465202000202532693A253032692052
:100D4000202532692E25316956202534696D416888
:100D500000202532693A2530326920202532692E5B
:100D600025316956202534696D4168004449523A5D
:100D7000253364256300414C543A2534696D0041A4
:100D80004C543A2534696D00414C543A2D2D2D2D8B
:100D90002000256300484D3A253364256320204414
:100DA0004953543A2533646D202563005057523A15
:100DB0002532692E253169412028256957292000CF
:100DC0004346002020004750533A2532756D2F735B
:100DD000205341543A256420002020334420004E03
:100DE0004F464958004447505320002020204E6F62
:100DF000204E6176694374726C20202020202020D0
:100E0000002532692E2569202532692E2569202585
:100E100032692E2569202532692E25694100253346
:100E200069202533692025336920253369256343EB
:100E3000002532692E2569202532692E2569410059
:100E40002532692E2569202532692E256920253213
:100E5000692E2569202532692E25694100253369CF
:100E600020253369256343202020202020202000D6
:100E700025336920253369202533692025336925E9
:100E80006343004552523A202532642021004552E6
:100E9000523A2000207777772E4D696B726F4B6F37
:100EA000707465722E646520200053657474696ED9
:100EB000673A257520257320004D696E3A25326901
:100EC0002E253169562025732000414C543A00509C
:100ED0004F54493A2533752000284F4E29202000D1
:100EE000284F46462920004C494D4954005641524E
:100EF000494F0044495341424C45440043463A005F
:100F000044495341424C45440020284F4E2920007B
:100F100020284F4646290020544541434800475069
:100F2000533A0044495341424C45440028465245F7
:100F300045290028484F4D4529002841494429208A
:100F40000028484F4C4429002046533A25757365C4
:100F50006B2000484F4D4520414C543A0025756D9B
:100F600000484F4C4420004E693A25346920526FA6
:100F70003A25346920433A2533690047733A2534CA
:100F8000692059613A253469200050313A25346985
:100F90002050323A25346920333A253369005034E1
:100FA0003A2534692050353A25346920363A2533BC
:100FB0006900434F55504C494E47204F464621202B
:100FC000004C4F4F50494E472120004848212000F7
:100FD000434F4D50415353204F46462120000A0DA8
:100FE0007777772E4D696B726F4B6F707465722EC9
:100FF00064652028632920486953797374656D738B
:1010000020476D6248000A0D74686520757365207D
:101010006F66207468697320736F66747761726598
:10102000206973206F6E6C79207065726D697474BD
:101030006564200A0D6F6E206F726967696E616C5E
:10104000204D696B726F4B6F707465722D486172C1
:101050006477617265005573657200486F5454205F
:101060005633004143542044534C004A6574690090
:101070005370656B7472756D0050504D000A0D52BF
:10108000656365697665723A2000532E4275730078
:10109000756E6B6E6F776E2E205573696E6720507C
:1010A000504D2E2E2E006E6F7420737570706F72FF
:1010B0007465642062792068617264776172652169
:1010C000000A0D466C69676874436F6E74726F6CCA
:1010D0000A0D48617264776172653A25642E256451
:1010E0000A0D536F6674776172653A5625642E2532
:1010F00064256320000011241FBECFEFD0E4DEBFC3
:10110000CDBF11E0A0E0B1E0E0EEF7E101E00BBF00
:1011100002C007900D92A63AB107D9F71AE0A6EAE5
:10112000B1E001C01D92A034B107E1F77AEAE2E034
:10113000F0E081E280935700D4907E010894E11C96
:10114000F11C20EF37EF41E050E087016FE0DA015A
:10115000C9012F5F3F4F4F4F5F4FABBFFC018791DE
:10116000F80181938F01615067FFF1CFF7016EE0C5
:10117000819178277095615067FFFACF8889781739
:1011800029F0F7E9DF1611F40000FECF0E949D0957
:101190000C94EF8B0C94000088E791E09F938F9361
:1011A0008FEB94E19F938F93E091FC03F091FD030B
:1011B00009950F900F900F900F900895809143061E
:1011C000E82FFF27EE0FFF1FEB58F84F808191812A
:1011D0008D5E9F4F14F010920201808191818A5B95
:1011E0009F4FCCF4809102018823A9F481E0809381
:1011F0000201809130048F5F80933004853038F095
:1012000088EE93E09093DB018093DA0104C066E9F5
:1012100070E00E940E398091300499279093C805A0
:101220008093C70508951F93CF93DF93182F8823CA
:1012300089F08EE991E09F938F938FEB94E19F93D8
:101240008F93E091FC03F091FD0309950F900F90AF
:101250000F900F9080916606823308F044C084EFAF
:1012600091E00E94CE18EC01112329F0CE010E94DA
:10127000D7188823D9F3C2E0D0E026E530E080918A
:101280001D0190911E018217930730F02196255D74
:101290003F4FC730D10598F3809166069927C89FC4
:1012A0009001C99F300DD89F300D1124209300016B
:1012B0001123D9F068EC70E08C2F0E940E39DF9377
:1012C000CF9386EA91E09F938F938FEB94E19F9366
:1012D0008F93E091FC03F091FD0309958DB79EB7C4
:1012E00006968DBF02C080930001112311F18091F9
:1012F00000016AE00E94428B892F99279F938F9368
:10130000809100010E94428B99279F938F9381EBDC
:1013100091E09F938F938FEB94E19F938F93E09154
:10132000FC03F091FD0309952DB73EB7285F3F4FB1
:101330002DBFDF91CF911F910895CFEFD0E4DEBF95
:10134000CDBF8824992414B815B8B7EEEB2EB3E0BE
:10135000FB2E2EEC3FEFE20EF31EF7FEFACF85E1F7
:101360008093010181E887B93E9A8FEF88B98BE1BC
:1013700084B911E015B98EE38AB987E48BB9469A2E
:1013800084B7877F84BF809160008861809360000C
:101390001092600084EC99E09093DB018093DA0175
:1013A0001092E6021092E50210927A0710927907E5
:1013B0001092E8021092E7021092EA021092E902FB
:1013C00084EC94E0A0E0B0E080934201909343016C
:1013D000A0934401B093450128980E9437190E94B8
:1013E00008190E94C7140E944B350E94E51C812FEA
:1013F0000E94AE300E94C7660E9403700E94DC8784
:10140000809101018C3010F4299A01C029987894B8
:101410000E94CD2F80912102826080932102109240
:1014200024020E94404484EF91E00E94CE187C0187
:101430008091210280FD05C0C7010E94D718882332
:10144000B9F385EC91E09F938F93AFEBAA2EA4E1C3
:10145000BA2EBF92AF92E091FC03F091FD03099583
:1014600080EA9FE00E94CE187C0100E010E00F901F
:101470000F900F900F90C7E1D7E0FBECCF2EF6E076
:10148000DF2E0E9440448091210280FD05C0C701EB
:101490000E94D7188823B9F3F60180811816A4F4A6
:1014A0000BC00E9440448091210280FD05C0C7010D
:1014B0000E94D7188823B9F3C7010E94D718882340
:1014C00019F4888188236CF7888187FF1BC00F5F20
:1014D0001F4F1F930F930150104087ED91E09F9392
:1014E0008F93BF92AF92E091FC03F091FD030995B9
:1014F0008091A7018F5F8093A7012DB73EB72A5F28
:101500003F4F2DBF0F5F1F4F84E090E0C80ED91EE4
:1015100028960C30110508F4B4CF00E010E0C4E1C7
:10152000D7E0EBECEE2EE6E0FE2E8B8187FD1FC0B0
:10153000F70180811816DCF40F5F1F4F1F930F9384
:10154000015010408AED91E09F938F938FEB94E1CF
:101550009F938F93E091FC03F091FD03099582E046
:101560008093D8012DB73EB72A5F3F4F2DBF8B81A7
:1015700080788B830F5F1F4F84E090E0E80EF91EA8
:1015800028960C30110588F20E94CC0890914106F3
:101590008091A701981728F48091160480618093A8
:1015A000160488EF91E09F938F93CFEBD4E1DF9304
:1015B000CF93E091FC03F091FD03099588EE93E051
:1015C0000E94CE187C010E94EB1C0F900F900F9090
:1015D0000F90C7010E94D7188823D9F388E192E0C1
:1015E0009F938F93DF93CF93E091FC03F091FD03E2
:1015F000099580E00E94DD39809101010F900F90E4
:101600000F900F908A3011F0843110F0289801C0AB
:10161000289A80ED97E09093DB018093DA0185E5CD
:10162000809332048EE090E00E94F12D9927182FCC
:1016300000278FE090E00E94F12D080F111D1093FC
:10164000AD010093AC018AE090E00E94F12D992752
:10165000182F00278BE090E00E94F12D080F111D3C
:101660001093AB010093AA010F5F1F4F39F08091D7
:10167000AC019091AD018F5F9F4F41F41092AD018D
:101680001092AC011092AB011092AA018091AA01B4
:101690009091AB019F938F938091AC019091AD019C
:1016A0009F938F938DE192E09F938F93DF93CF93DE
:1016B000E091FC03F091FD0309950E947F2288E8E8
:1016C00093E190933D0180933C01C1E0C0933104CC
:1016D0008C2F0E941309809169060E9428870E941E
:1016E000CC0880ED97E00E94CE187C018AEF90E054
:1016F0000E94CE1883E080939F051092A6018091EE
:10170000AF062DB73EB7285F3F4F2DBF84FF02C005
:10171000C093AE018091B001882311F04798FECFAD
:101720008091DE01882309F436C280910F0188235D
:1017300009F431C21092DE0180913004882319F03F
:101740000E94DE0802C00E9470470E94404420911F
:1017500001012A3011F0243110F0289801C0289A94
:101760008091D902882331F08091D90281508093F1
:10177000D9020EC080916F00806280936F0010923A
:10178000760710927507809116048860809316047E
:1017900080913C0190913D01019790933D01809390
:1017A0003C0180913C0190913D01892B21F0809179
:1017B00022028823C9F180913C0190913D01892B3F
:1017C000D9F40E94D83085E090E090933D01809359
:1017D0003C018091D9059091DA0501969093DA0544
:1017E0008093D905809116048160809316048091BE
:1017F000A00582608093A005809107019091080167
:101800008F5F9F4FC1F48091D8028823A1F088EAAE
:1018100091E69093DB018093DA0180E890E0909369
:1018200008018093070107C02A3011F0243110F01D
:10183000289801C0289A0E9494888091DE0188230C
:1018400009F0A9C18091E303882319F00E94267E44
:10185000A2C180910D01882311F00E944E190E94AF
:101860000B150E945910C7010E94D718882309F44C
:101870008EC184E190E0E80EF91E80916906863001
:1018800011F40E94D47380912202882349F0809140
:1018900016048260809316048091A00582600FC0B8
:1018A0008091DA019091DB01892B59F480913C0100
:1018B00090913D01079728F08091A0058D7F80933E
:1018C000A0058091AE01882361F08091D90287390B
:1018D00040F01092AE0188E893E19093DB01809391
:1018E000DA0180910401882321F081508093040162
:1018F0002EC080933C041092AD021092AC02109264
:10190000AB021092AA021092A9021092A802809132
:10191000D9028823E1F480910701909108018F5F3B
:101920009F4FA9F42091AE01223089F088E99AE313
:101930009093DB018093DA0180E09CE090930801B2
:1019400080930701222319F082E08093AE018091F9
:101950009B01893C48F0815080939B018091160443
:101960008B7F809316043FC0809156088823F9F03E
:101970008091160484608093160489E08093B303F9
:1019800080910701909108018F5F9F4F81F48091B2
:10199000D802882361F088E99AE39093DB01809371
:1019A000DA0180E098EA9093080180930701109291
:1019B000A5031092A4031092A3031092A203109205
:1019C000A10310924908109288081092870810927B
:1019D0008A08109289088FEF9FEF90938608809372
:1019E000850810929B0180910001282F3327809158
:1019F0001D0190911E0182179307CCF48091A102E2
:101A000080628093A10280910701909108018F5F0D
:101A10009F4FC1F480E797E19093DB018093DA0157
:101A200080E093E090930801809307010BC08091C0
:101A3000DA019091DB01892B29F48091A1028F7D3D
:101A40008093A1020E94896B84E08093D9018091E8
:101A5000AF018F5F8093AF01813309F04FC01092C7
:101A6000AF018091A10281FF0AC08091A8019091ED
:101A7000A90101969093A9018093A8013FC05AEA59
:101A8000852E55E0952E8091E6059091E7059C0105
:101A9000442737FD4095542F8091150190911601F0
:101AA000A0911701B0911801281739074A075B0761
:101AB00034F48091E6059091E70501961BC0809172
:101AC000E6059091E7059C01442737FD4095542F8A
:101AD0008091150190911601A0911701B091180104
:101AE00082179307A407B5074CF48091E6059091FF
:101AF000E70501979093E7058093E6050894811C1C
:101B0000911C32E783163BE0930609F040C088241D
:101B100099242091AC013091AD012F5F3F4F30935C
:101B2000AD012093AC018091AA019091AB01019687
:101B30009093AB018093AA01832F9927682F8EE0A1
:101B400090E00E94F92D8091AC019091AD019070D0
:101B5000682F8FE090E00E94F92D8091AA0190916A
:101B6000AB01892F9927682F8AE090E00E94F92D18
:101B70008091AA019091AB019070682F8BE090E06A
:101B80000E94F92D84E190E00E94CE187C010E9411
:101B9000D96B0E941A708091D901882309F0BACDBF
:101BA0000E94E866B7CD1F920F920FB60F921124D4
:101BB0008F939F93EF93FF93809106018823E1F425
:101BC0008091CA019091CB0101969093CB018093B3
:101BD000CA01FC01E051FB4FE081ED3019F08F3A72
:101BE000910539F41092CB011092CA0181E08093E3
:101BF0000601E093C60004C01092CB011092CA0106
:101C0000FF91EF919F918F910F900FBE0F901F90BA
:101C100018951F920F920FB60F9211242F933F9396
:101C20004F935F936F937F938F939F93AF93BF93E4
:101C3000CF93EF93FF9390E08091B001813029F42E
:101C40008091C6008093CE00CCC08091B0018230DC
:101C500029F48091C60080933F04C3C08091C600E0
:101C60008093C2015091D0015F3A10F09093D1015E
:101C70008091C2018D3009F065C08091D101823020
:101C800009F060C09093D101852F9927815C9B4F0B
:101C9000FC01329740812091CC013091CD01241B71
:101CA0003109DC0111978C91281B3109C9019F7002
:101CB0009093CD018093CC0146E0969587954A9507
:101CC000E1F7982F935C9093CE012F733070235CD3
:101CD0002093CF018081981729F48C91281711F453
:101CE00091E006C090E08091BF018F5F8093BF01BB
:101CF000C091C101CC2309F074C0992309F471C0CB
:101D000081E08093C101580F5093BE015150E52FDF
:101D1000FF27E15CFB4F8DE0808380914104823599
:101D200009F05FC00E947F2288E190E02CE00FB6AE
:101D3000F894A895809360000FBE20936000C09334
:101D4000D8014FC02091D101822F99278130910570
:101D5000F9F0823091051CF4892B21F040C00297E4
:101D600011F13DC08091C201833239F48091C101EB
:101D7000882319F481E08093D1018091C20180937E
:101D80003F0481E08093D0018091C201992722C055
:101D90002F5F2093D101E52FFF27E15CFB4F80915E
:101DA000C201808309C0E52FFF27E15CFB4F8091D2
:101DB000C20180835F3A20F45F5F5093D00102C07C
:101DC0001092D1012091C2018091CC019091CD015E
:101DD000820F911D9093CD018093CC0102C010928F
:101DE000D101FF91EF91CF91BF91AF919F918F91D1
:101DF0007F916F915F914F913F912F910F900FBE07
:101E00000F901F901895AC01A0E0B0E09D01A817BD
:101E1000B90748F4E0EFF4E08191280F311D1196E5
:101E2000A417B507C8F33F70FD01E051FB4FC9018E
:101E300056E0969587955A95E1F7835C80831196D5
:101E4000FD01E051FB4F2F733070822F835C808344
:101E5000AF50BB4F8DE08C93109206018091F0043F
:101E60008093C6000895A0E0B0E0E9E3FFE00C94A1
:101E7000BB8B2C859D850E85BB2483E28093F0046B
:101E80009F599093F1042093F20433E0E32EF12C58
:101E9000002309F49EC0CF84D888BE016D5E7F4FB9
:101EA000A989BA890150109709F493C01097B9F025
:101EB000F601EB0DF11DB3949081119791F400237D
:101EC00049F1FB016E5F7F4FDB01C080D1806E5F07
:101ED0007F4F0D90BC91A02DBB24015002C090E01B
:101EE00019C01097B9F0F601EB0DF11DB3944081C4
:101EF000119791F4002341F1FB016E5F7F4FDB01ED
:101F0000C080D1806E5F7F4F0D90BC91A02DBB240F
:101F1000015002C040E018C01097B1F0F601EB0D7F
:101F2000F11DB3941081119781F4002371F0FB012E
:101F30003296DB01CD90DC90BF016E5F7F4FA081B8
:101F4000B181BB24015001C010E0F701E051FB4F0B
:101F5000892F86958695835C80830894E11CF11C0B
:101F6000F701E051FB4F892F99278370907024E08F
:101F7000880F991F2A95E1F755279A0194E0369525
:101F800027959A95E1F7822B835C80830894E11C66
:101F9000F11CF701E051FB4F4F705070440F551F7B
:101FA000440F551F812F992726E0969587952A95EE
:101FB000E1F7842B835C80830894E11CF11CF7011A
:101FC000E051FB4F1F73135C10830894E11CF11C5C
:101FD0006ACFC7010E94030FE9E00C94D78BA3E0FE
:101FE0007A2F4091BE014650442309F458C0E72F90
:101FF000FF27E15CFB4F80818D537F5FE72FFF2739
:10200000E15CFB4F20812D537F5FE72FFF27E15CD1
:10201000FB4F30813D537F5FE72FFF27E15CFB4F94
:1020200060816D537F5F9927880F991F880F991FD3
:10203000522F52955F70582B822F99278F70907076
:10204000F4E0880F991FFA95E1F7232F269526953E
:10205000282B832F992783709070E6E0880F991FB3
:10206000EA95E1F7682B41504F3FC9F0EA2FFF276F
:10207000E15CFB4F5083AF5F41504F3F81F0EA2F4F
:10208000FF27E15CFB4F2083AF5F41504F3F39F0AA
:10209000EA2FFF27E15CFB4F6083AF5FA5CF82E4AF
:1020A00094E09093BD018093BC01A350A093BB0129
:1020B0000895A2E0B0E0EFE5F0E10C94C18B8091CF
:1020C000C101882309F457C40E94EF0F8091400496
:1020D000823609F023C38091410499278037910506
:1020E00009F4AFC081379105C4F48A36910509F42B
:1020F00080C28B36910544F48B34910571F186369C
:10210000910509F45FC10AC38D36910509F469C0D0
:102110008E36910509F44DC001C38437910541F114
:10212000853791054CF48137910509F491C08337C7
:10213000910509F4DFC0F2C28737910509F41BC28B
:10214000883791052CF48537910509F4D7C1E6C28B
:102150008937910509F46DC1E1C2E091BC01F091AC
:10216000BD018081918190938F0180938E01D6C2B1
:102170008091BE01A091BC01B091BD01853140F0BC
:1021800080E1EAE1F4E00D9001928A95E1F70DC05B
:102190008D919D910D90BC91A02D80931A049093E8
:1021A0001B04A0931C04B0931D0480EF8093B9011D
:1021B0004BC0809106018823E1F38DE490E09F936A
:1021C0008F938EEB96E09F938F9381E08F938F9305
:1021D0008EE48F930E94330F8DB79EB707968DBF05
:1021E0009DC2A091BC01B091BD011C91113081F440
:1021F0008DE4EEEBF6E00D9001928A95E1F70E94F6
:102200000A2F1983809116048F7E8093160401C0D3
:102210001982809106018823E1F381E090E09F9389
:102220008F93CE0101969F938F9381E08F938F932D
:102230008DE48F930E94330FADB7BEB71796ADBF35
:102240006DC281E08093C4018FEF8093040166C268
:10225000E091BC01F091BD01E0818E2F8A508A305F
:1022600058F48983882311F481E003C0863010F08C
:1022700085E0898361E00EC08E2F84518A3070F42E
:102280008983882311F481E003C0863010F085E053
:10229000898360E089810E948A2F12C0E983EF3F21
:1022A00019F40E946D2F89838981882311F481E0BC
:1022B00003C0863010F085E0898389810E940F2E4B
:1022C000809106018823E1F38BE790E09F938F9341
:1022D00082E496E09F938F9381E090E09F938F93A9
:1022E000CE0101969F938F9382E08F9381E08F932D
:1022F00081E577C12091BC013091BD01D9018C915C
:102300008150853008F045C0F90181818A3509F096
:1023100040C08091D8028823E1F52F5F3F4F8BE7C3
:10232000E2E4F6E0D9010D9001928A95E1F7F90116
:1023300082910E947A2E809183069927AA27BB2733
:10234000BC01CD0124EC39E040E050E00E94238B39
:10235000DC01CB018093860190938701A0938801D3
:10236000B0938901809184069927AA27BB27BC01D5
:10237000CD010E94238BDC01CB01809382019093DD
:102380008301A0938401B09385010E946D2F8983FE
:1023900001C01982809106018823E1F381E090E079
:1023A0009F938F93CE0101969F938F9381E08F939C
:1023B0008F9383E58F930E94330F8DB79EB7079657
:1023C0008DBF26C0E091BC01F091BD01E0818E2F50
:1023D0008150853018F48E2F0E940F2E0E946D2F91
:1023E0008983809106018823E1F381E090E09F9347
:1023F0008F93CE0101969F938F9381E08F938F935C
:1024000086E48F930E94330FADB7BEB71796ADBF6A
:102410008091D802882329F46EE670E089810E94B9
:102420000E3980E00E941309809169060E94288776
:1024300075C1E091BC01F091BD018081992787FDB4
:1024400090959093900780938F078181992787FDBE
:10245000909590939207809391078281992787FDA9
:10246000909590939407809393078381992787FD94
:10247000909590939607809395078481992787FD7F
:10248000909590939807809397078581992787FD6A
:10249000909590939A07809399078681992787FD55
:1024A000909590939C0780939B078781992787FD40
:1024B000909590939E0780939D078085992787FD2F
:1024C00090959093A00780939F078185992787FD1A
:1024D00090959093A2078093A1078285992787FD05
:1024E00090959093A4078093A3078385992787FDF0
:1024F00090959093A6078093A50710C1E091BC0129
:10250000F091BD0180810E94A4348A83882319F44C
:1025100081E0898301C01982809106018823E1F35B
:1025200088E090E09F938F938CE097E09F938F9348
:1025300021E030E03F932F938091BC019091BD0149
:102540009F938F933F932F93CE0102969F938F93E8
:102550003F932F93CE01820F931F9F938F9384E01D
:102560008F9381E08F9385E58F930E94330FEDB7B2
:10257000FEB773963CC08091BB01893008F4CEC091
:102580002091BC013091BD012F5F3F4F88E0ACE04E
:10259000B7E0F90101900D928A95E1F7D9018E918A
:1025A0000E94FA338A83882319F481E0898301C069
:1025B0001982809106018823E1F321E030E03F9306
:1025C0002F93CE0102969F938F933F932F93CE012B
:1025D000820F931F9F938F9382E08F9381E08F935D
:1025E00087E58F930E94330FEDB7FEB73B96EDBFA3
:1025F00095C08091D802882309F090C00E94DB86A4
:102600008983823019F0843009F088C020E430E0FA
:10261000F8948091C1008F738093C1008091C900AC
:102620008F738093C9008091C100877E8093C10021
:102630008091C900877E8093C9008091C80087FF80
:1026400003C08091CE00F9CF8091C00087FF03C006
:102650008091C600F9CFE091BC01F091BD01E0810D
:10266000E13021F482E08093B0012EC0E43611F411
:1026700021E830E081E08093B001832F9927809397
:10268000CD002093CC008091CD008093C500809137
:10269000CC008093C4008091CA008F7D8093CA00D3
:1026A0008091CA008F7E8093CA008091C9008B7F81
:1026B0008093C9008091CA0084608093CA00809191
:1026C000CA0082608093CA008091CA00877F80938D
:1026D000CA008091C200877F8093C2008091C900A8
:1026E0008E7F8093C9008091C10088618093C10072
:1026F0008091C90088618093C9008091C100806881
:102700008093C1008091C90080688093C9001092B5
:102710006E0010926F0010927000789480914104C6
:1027200099278436910509F4BBC085369105ACF430
:102730008136910509F46FC0823691052CF48B34F3
:10274000910509F45DC00FC18236910509F470C08E
:102750008336910509F47FC006C18C36910509F4D2
:10276000EDC08D3691054CF48736910509F4F8C01B
:102770008836910509F4B2C0F6C08437910529F076
:102780008637910509F4E8C0EEC08091BE01A091A2
:10279000BC01B091BD01803140F080E1EAE1F4E09C
:1027A0000D9001928A95E1F70DC08D919D910D904C
:1027B000BC91A02D80931A0490931B04A0931C0439
:1027C000B0931D04809106018823E1F31F9280914C
:1027D00003018F9384E58F930E94330F8AEF8093D8
:1027E000B9018FEF8093040180EA9FE00E94CE1828
:1027F0009093B2018093B1010F900F900F90B3C0EE
:10280000E091BC01F091BD018081918190938F0195
:1028100080938E01A8C0E091BC01F091BD01808140
:1028200080930501803298F08FE1809305010FC0FD
:10283000A091BC01B091BD018BE0E2E3F4E00D900A
:1028400001928A95E1F780913B048093E1058FEF37
:102850008093040188C08091B5019091B601892BC5
:1028600089F4E091BC01F091BD01E081EE2351F0CB
:102870008AE0E89FC00111240E94CE1890930D04B5
:1028800080930C04E091BC01F091BD0190818AE03D
:10289000989FC00111249093B6018093B50115C093
:1028A0008FEF80930401E091BC01F091BD01908114
:1028B0008AE0989FC00111249093B8018093B701DA
:1028C000892B19F081E08093C60180EA9FE00E9485
:1028D000CE189093B2018093B10145C08FEF8093E1
:1028E0000401E091BC01F091BD01908197FD08C009
:1028F00082E08093C3011092B4011092B3011AC018
:10290000909580911A02892B80931A0291818AE016
:10291000989FC00111249093B4018093B30184E087
:102920008093C30180EA9FE00E94CE189093B20189
:102930008093B10181E08093C70115C08FEF809330
:102940000401E091BC01F091BD01808180931B02E4
:1029500081E08093C80107C081E08093C50103C076
:1029600081E08093C9011092C1011092BD011092C3
:10297000BC011092BB01E3E0CE5F0C94DD8B982F7D
:102980008091C00085FFFCCF9093C60008950F93FF
:102990001F9388E18093C1008091C0008260809382
:1029A000C0008091C10080688093C1008091C10007
:1029B00080648093C10000E010E00093C5008AE2CB
:1029C00090E08093C4008091B7019091B8010E947B
:1029D000CE1890930F0480930E048CED90E00E942B
:1029E000CE1890933E0480933D041092100488E525
:1029F0008093110484E0809314048BE0809312048C
:102A0000109213041093BD010093BC011092BB01FE
:102A10001F910F910895A0E1B0E0E1E1F5E10C9480
:102A2000BE8B80910601882309F4C1C28091B10157
:102A30009091B2010E94D718882361F01092B401DE
:102A40001092B3011092B8011092B7011092B60122
:102A50001092B5018091B3019091B401892B41F09E
:102A60008091EE049091EF040E94D718882329F4F6
:102A70008091C701882309F460C0809106018823F2
:102A800009F45BC08091C30101EF15E08430A8F028
:102A90000E94952280E590E09F938F931F930F9360
:102AA00081E08F938F9388E48F930E94330F2DB72B
:102AB0003EB7295F3F4F2DBF34C010921C028FE3F9
:102AC00094E09F938F9388E892E29F938F93E09195
:102AD000FC03F091FD03099584E190E09F938F93AF
:102AE0001F930F9381E090E09F938F9383EC91E08D
:102AF0009F938F9382E08F9381E08F9388E48F93ED
:102B00000E94330F8091C301982F8F5F8093C30180
:102B10002DB73EB7215F3F4F2DBF943010F010927C
:102B2000C3018091B3019091B4010E94CE1890939B
:102B3000EF048093EE041092C7018091C8018823AE
:102B400051F180910601882331F10E94952280E5A0
:102B500090E09F938F9381EF95E09F938F9321E077
:102B600030E03F932F938FE191E09F938F933F93BA
:102B70002F938BE192E09F938F9383E08F9381E07B
:102B80008F938CE48F930E94330F1092C8018DB7FE
:102B90009EB70F968DBF8091C5018823D1F080919B
:102BA00006018823B1F08AE090E09F938F9380E143
:102BB00094E09F938F9381E08F938F9386E58F931B
:102BC0000E94330F1092C5012DB73EB7295F3F4FCA
:102BD0002DBF8091C9018823D9F0809106018823F7
:102BE000B9F08BE090E09F938F9382E394E09F9302
:102BF0008F9381E08F93809103018F9387E48F936C
:102C00000E94330F1092C9018DB79EB707968DBFF2
:102C100080913D0490913E040E94D718882309F4C6
:102C200061C080910601882309F45CC080915E0632
:102C30009927880F991F880F991F7C010027F7FC9F
:102C40000095102F8091330390913403A0913503A8
:102C5000B0913603BC01CD01A80197010E94978B6A
:102C600030932B0420932A0480912B0390912C0302
:102C7000A0912D03B0912E03BC01CD01A8019701B5
:102C80000E94978B30932D0420932C048091B602E0
:102C900080932E048091B50280932F0488E090E009
:102CA0009F938F938AE294E09F938F9381E08F9319
:102CB00083E08F938BE68F930E94330F80913004D3
:102CC0002DB73EB7295F3F4F2DBF853018F086E006
:102CD0008093300483E690E00E94CE1890933E04E7
:102CE00080933D048091B7019091B801892B41F008
:102CF00080910E0490910F040E94D718882321F42C
:102D00008091C601882339F180910601882319F149
:102D10000E94F83782E490E09F938F938FE995E0CB
:102D20009F938F9381E08F938F9384E48F930E947E
:102D3000330F1092C6018DB79EB707968DBF809155
:102D4000B7019091B801009731F00E94CE1890938E
:102D50000F0480930E048091B5019091B601892BE8
:102D600009F4B8C080910C0490910D040E94D7180A
:102D7000882309F4AFC080910601882309F4AAC012
:102D800080915E069927880F991F880F991F7C01F3
:102D90000027F7FC0095102F8091330390913403A6
:102DA000A0913503B0913603BC01CD01A801970174
:102DB0000E94978B3093FF032093FE0380912B0397
:102DC00090912C03A0912D03B0912E03BC01CD0155
:102DD000A80197010E94978B30930104209300046F
:102DE00020913E0830913F084091400850914108A1
:102DF000DA01C90163E0880F991FAA1FBB1F6A95FA
:102E0000D1F7820F931FA41FB51F820F931FA41F1A
:102E1000B51F2091420130914301409144015091EE
:102E20004501BC01CD010E94978B30930304209390
:102E300002048091FB029091FC02A091FD02B091EE
:102E4000FE0249E0B595A795979587954A95D1F7E4
:102E5000809304048091F7029091F802A091F90206
:102E6000B091FA0239E0B595A795979587953A956F
:102E7000D1F7809305048091030390910403A091FE
:102E80000503B091060329E0B595A7959795879519
:102E90002A95D1F7809306048EE090E09F938F935C
:102EA0008EEF93E09F938F9381E08F938F9383E4D2
:102EB0008F930E94330F8091B5019091B6010E94CB
:102EC000CE1890930D0480930C042DB73EB7295F64
:102ED0003F4F2DBF809105018F3F71F1992704E08D
:102EE000880F991F0A95E1F7815C9D4F40E150E002
:102EF000BC01CE0101960E94768980E190E09F930B
:102F00008F93CE0101969F938F9381E090E09F93E2
:102F10008F9385E091E09F938F9382E08F9381E080
:102F20008F9381E48F930E94330F8FEF809305017D
:102F30008DB79EB70B968DBF8091E1058823D1F0A8
:102F4000809106018823B1F081E090E09F938F93F8
:102F500081EE95E09F938F9381E08F938F9382E42E
:102F60008F930E94330F1092E1052DB73EB7295F72
:102F70003F4F2DBF8091C4018823C9F08091060185
:102F80008823A9F084E390E09F938F9385E797E0EF
:102F90009F938F9381E08F938F9380E58F930E940F
:102FA000330F1092C4018DB79EB707968DBFE6E030
:102FB000C05F0C94DA8B1F920F920FB60F92112400
:102FC0002F933F935F936F937F938F939F93AF93D1
:102FD000BF93EF93FF9320E08091D901882329F0DC
:102FE0008091D90181508093D9018091C6038823B3
:102FF00019F081508093C6038091E1018150809344
:10300000E1018F3F09F05BC089E08093E10180918D
:10301000DF019091E00101969093E0018093DF0140
:1030200080910E018F5F817080930E01882319F4C7
:1030300081E08093DE01349903C081E08093E20156
:103040008091DA019091DB01892B21F18091DA01E5
:103050009091DB010B9750F08091DA019091DB01A8
:103060000A979093DB018093DA0104C01092DB0190
:103070001092DA018091DA019091DB012091070131
:103080003091080182239323892B11F021E008C09D
:1030900020E006C08FEF9FEF909308018093070117
:1030A00080910101222331F08A3011F45A9A07C02D
:1030B000479A05C08A3011F45A9801C04798809108
:1030C000E201882309F45AC020919B01222309F0D0
:1030D00055C080912E0883FF51C086B19927FC010D
:1030E000E071F07084FF13C08091DC019091DD01EC
:1030F00001969093DD018093DC018091DC01909139
:10310000DD01895E9340D0F12093E20137C08091C8
:10311000DC019091DD01892B69F18091DC019091B6
:10312000DD018A56914030F58091DC019091DD01FE
:1031300069E270E00E944E8B8091DC019091DD018C
:10314000860F971F9093DD018093DC018091DC0155
:103150009091DD010B9750F08091DC019091DD01A1
:103160000A9790938F0180938E0104C0F0938F0192
:10317000E0938E011092DD011092DC01FF91EF913E
:10318000BF91AF919F918F917F916F915F913F918F
:103190002F910F900FBE0F901F9018952091DF0177
:1031A0003091E001280F391FC9010196089520913F
:1031B000DF013091E001821B930B892F99278695BF
:1031C000807490700895CF93DF930E94CE18EC0125
:1031D000CE010E94D7188823D9F3DF91CF910895AB
:1031E000CF93DF930E94CE18EC0109C080910F01AC
:1031F000882329F090930F018FEC80937A00CE0101
:103200000E94D718982F882389F3DF91CF910895D2
:103210009FB7F8945F983E9A469A8091B0008F705D
:103220008093B0008091B00083608093B000809163
:10323000B1008B738093B1008091B1008B6080935B
:10324000B1001092B2008FEF8093B3008091B00074
:1032500080688093B000809170008A7F80937000B6
:10326000809170008260809370009FBF08958AE013
:1032700090E00E94CE189093E8018093E70182E0ED
:1032800085BD83EA84BD17BC84EB88BD86E086BD1E
:1032900080916E00816080936E000895A0E0B0E0A0
:1032A000E4E5F9E10C94BD8B80917906E82FFF27C6
:1032B000E85BFE4F9681D08080910D01A92FBB273E
:1032C000A7FDB095CB2FDB2F813009F012C12091E3
:1032D0003303309134034091350350913603BD01DF
:1032E000CE010E94238B97FF04C061587F4F8F4F00
:1032F0009F4F7B018C0187E015950795F794E79424
:103300008A95D1F78D2D992787FD9095A92FB92FF3
:1033100020912B0330912C0340912D0350912E03CB
:10332000BC01CD010E94238B97FF04C061587F4FE1
:103330008F4F9F4FC7E09595879577956795CA956D
:10334000D1F7F801E701C61BD70BE80BF90B209169
:10335000AC033091AD03C901B3E0880F991FBA9552
:10336000E1F7821B930BAA2797FDA095BA2FC81BE4
:10337000D90BEA0BFB0B809170069927AA27BB2774
:10338000BC01CD019E01AF010E94238B97FF04C0B9
:1033900061507E4F8F4F9F4FFC01EB01A9E0F595E7
:1033A000E795D795C795AA95D1F780916D01992793
:1033B00076E0880F991F7A95E1F740910B015091C3
:1033C0000C01209178063327841B950BB9010E94CC
:1033D000628B80910B0190910C01860F971F909347
:1033E0000C0180930B018091AE0680FF14C0809188
:1033F0000B0190910C0197FD0F9664E095958795D0
:103400006A95E1F7AA2797FDA095BA2FC80FD91F93
:10341000EA1FFB1F15C080910B0190910C0197FDD5
:103420000F9654E0959587955A95E1F7AA2797FD51
:10343000A095BA2F8C1B9D0BAE0BBF0BFD01EC01B1
:103440002091AB06222321F133278091D401909162
:10345000D501829FA001839F500D929F500D112492
:10346000CA01AA2797FDA095BA2F8C0F9D1FAE1FEA
:10347000BF1F2F5F3F4F442737FD4095542FBC019E
:10348000CD010E94978B3093D5012093D40104C0C5
:10349000D093D501C093D40180917106282F332792
:1034A000220F331F220F331F8091D4019091D50139
:1034B000821793077CF080917206282F3327220F02
:1034C000331F220F331F8091D4019091D50128170B
:1034D000390724F43093D5012093D4018091010160
:1034E000843108F4F7C080910D018F5F80930D0146
:1034F000F3C020912B0330912C0340912D03509168
:103500002E03BD01CE010E94238B97FF04C061589A
:103510007F4F8F4F9F4F7B018C0187E0159507955B
:10352000F794E7948A95D1F78D2D992787FD90958B
:10353000A92FB92F209133033091340340913503E3
:1035400050913603BC01CD010E94238B9B01AC013D
:1035500097FF04C021583F4F4F4F5F4FC7E055952D
:10356000479537952795CA95D1F72E0D3F1D401FDA
:10357000511F809174069927AA27BB27BC01CD0152
:103580000E94238B97FF04C061507E4F8F4F9F4F47
:10359000FC01EB01B9E0F595E795D795C795BA958C
:1035A000D1F780916C019927A6E0880F991FAA9501
:1035B000E1F74091090150910A01209178063327E3
:1035C000841B950BB9010E94628B80910901909137
:1035D0000A01860F971F90930A0180930901809139
:1035E000AE0681FF14C08091090190910A0197FDF8
:1035F0000F9674E0959587957A95E1F7AA2797FD40
:10360000A095BA2FC80FD91FEA1FFB1F15C08091C4
:10361000090190910A0197FD0F9664E095958795B1
:103620006A95E1F7AA2797FDA095BA2F8C1B9D0BF1
:10363000AE0BBF0BFD01EC012091AC06222321F162
:1036400033278091D2019091D301829FA001839F63
:10365000500D929F500D1124CA01AA2797FDA095E5
:10366000BA2F8C0F9D1FAE1FBF1F2F5F3F4F4427E8
:1036700037FD4095542FBC01CD010E94978B3093AC
:10368000D3012093D20104C0D093D301C093D201BF
:1036900080917506282F3327220F331F220F331FE7
:1036A0008091D2019091D301821793077CF0809191
:1036B0007606282F3327220F331F220F331F8091C6
:1036C000D2019091D3012817390724F43093D30104
:1036D0002093D20110920D01E7E0CDB7DEB70C9434
:1036E000D98B1F920F920FB60F9211242F933F93F5
:1036F0004F935F938F939F93EF93FF93809101017B
:103700009091E301843108F04CC0992309F01CC169
:103710008091B00086FF24C08091B0008F7B8093A1
:10372000B0008091D4019091D50187559E4F909320
:10373000D7018093D60125E08D3D920718F08CEDDE
:1037400095E005C08757914030F487E791E090936A
:10375000D7018093D6018091D6019091D701BAC04C
:103760008091B00080648093B00080917706282F0C
:1037700033278DED96E0289FA001299F500D389F9B
:10378000500D1124CA012091E4013091E501821B02
:10379000930B9093D7018093D60181E080930D0124
:1037A000D0C0992309F0D0C08091B00086FF97C0A7
:1037B0008091B0008F7B8093B000E091E601EE2312
:1037C000F1F480917706282F33278DED96E0289F1E
:1037D000A001299F500D389F500D1124CA0120913E
:1037E000E4013091E501821B930B9093D701809304
:1037F000D6011092E5011092E401469AA2C089EA2E
:1038000093E09093D7018093D6018E2F9927833030
:103810009105D9F08430910534F48130910549F057
:10382000029761F020C08430910591F0059799F0DE
:103830001AC08091D4019091D50104C08091D20129
:103840009091D30187559E4F1DC080910A0805C0F5
:103850008091E30702C0809113089927880F991F70
:10386000880F991FEFCFFF27EE0FFF1FEB58F84F80
:1038700020813181220F331F8091D6019091D70191
:10388000820F931F9093D7018093D6018091D60128
:103890009091D70155E08D3D950718F08CED95E09E
:1038A00005C08757914030F487E791E09093D701A6
:1038B0008093D6012091D6013091D7012C5B304006
:1038C0003093D7012093D6018091E4019091E501D6
:1038D000820F931F9093E5018093E40132C08091A1
:1038E000B00080648093B0008CEB90E09093D7019F
:1038F0008093D6018091E4019091E50184549F4F1B
:103900009093E5018093E4018091D801882321F010
:103910008091D902882321F48091D801823011F45A
:10392000469801C0469A8091E6018F5F8093E60138
:1039300090917706981728F481E080930D011092FA
:10394000E60181E08093E3012091D6013091D70117
:1039500041E02F37340730F08FEF8093B3002F5FB3
:1039600030400FC02F3F3105C9F0C0F0A9014F5FB3
:1039700050404F37510550F480E88093B3002058F1
:1039800030403093D7012093D60112C08FEF80933F
:10399000B3005093D7014093D6010AC08091D6015D
:1039A0008093B3001092D7011092D6011092E301D8
:1039B000FF91EF919F918F915F914F913F912F9147
:1039C0000F900FBE0F901F90189510927C008FECF7
:1039D00080937A000895CF93DF931092ED0186E9EA
:1039E00087BD83E090E00E94F12DC82F863E08F449
:1039F000C65FC8BD84E690E00E94F0188091130174
:103A0000909114018152934010F0C0EF02C0C53074
:103A1000F8F0C8BD82E390E00E94F01884E594E0DD
:103A20009F938F938FEB94E19F938F93E091FC038F
:103A3000F091FD03099580911301909114010F906D
:103A40000F900F900F908152934010F4C550DFCF2C
:103A50006C2F83E090E00E94F92DCF3018F0CCE875
:103A6000D0E002C0C0E0D0E0CA3FD105F8F4C7BD45
:103A700082E390E00E94F01886E594E09F938F9394
:103A80008FEB94E19F938F93E091FC03F091FD0302
:103A9000099580911301909114010F900F900F9050
:103AA0000F908052934010F02196DECFC093EE0528
:103AB00080914F0680FF09C08C2F8A508B3E28F0E2
:103AC00080911504806480931504C7BD8CE291E059
:103AD0000E94F018DF91CF910895EF92FF921F930B
:103AE000CF9310E080ED97E00E94CE187C01CCE8E7
:103AF000133019F4CB3008F0C9E010E08091FC01DC
:103B00009091FD018C5F934024F4809112018150CB
:103B10000AC08091FC019091FD018750944034F0DF
:103B2000809112018F5F8093120101C011E080919A
:103B3000FA019091FB018C5F934024F48091110174
:103B400081500AC08091FA019091FB018750944006
:103B500034F0809111018F5F8093110101C01F5FCC
:103B60008091F8019091F9018C5F934024F4809149
:103B7000100181500AC08091F8019091F90187509D
:103B80009440C4F0809110018F5F8093100113C0A6
:103B900088E594E09F938F938FEB94E19F938F93AD
:103BA000E091FC03F091FD0309950F900F900F90A9
:103BB0000F905FC01F5F82E18093270280912102F6
:103BC0008E7F8093210285EA8093BC008091120150
:103BD0008A3040F4809115048160809315048AE056
:103BE0008093120180911201863F40F0809115046C
:103BF00081608093150485EF8093120180911101FB
:103C00008A3040F4809115048260809315048AE024
:103C10008093110180911101863F40F0809115043D
:103C200082608093150485EF8093110180911001CB
:103C30008A3040F4809115048460809315048AE0F2
:103C40008093100180911001863F40F0809115040F
:103C500084608093150485EF809310018091270282
:103C6000882339F0C7010E94D718882309F090CF24
:103C7000F5CF10920F018FEC80937A0080910F01A5
:103C80008823E1F3CA3020F48AE090E00E94F01823
:103C9000C15009F02DCF86E490E00E94F018CF913A
:103CA0001F91FF90EF9008951F920F920FB60F9201
:103CB0001124EF92FF920F931F932F933F934F93F3
:103CC0005F936F937F938F939F93AF93BF93EF9384
:103CD000FF9380910502282F3327442755278F5FB4
:103CE00080930502F9012231310508F0E3C3EA5B54
:103CF000FF4F0C94E98B809178009091790046C039
:103D0000809178009091790047C1809178009091DE
:103D10007900909308028093070272C180913C035E
:103D200090913D032091780030917900821B930B94
:103D30009093E3058093E2058091E2059091E3057D
:103D4000909312028093110279C180917800909132
:103D5000790020913E0330913F03821B930B909397
:103D6000ED058093EC058091EC059091ED05909325
:103D7000140280931302A0C380910B0290910C0255
:103D80002091780030917900820F931F90930C025C
:103D900080930B0281E091C38091090290910A0205
:103DA0002091780030917900820F931F90930A023E
:103DB0008093090284E081C38091AF0683FF1AC01B
:103DC00080911D0190911E019C01220F331F280F2D
:103DD000391F40917800509179008BE090E0489F26
:103DE000B001499F700D589F700D1124CB016EE1F9
:103DF00070E00FC080911D0190911E019C01220F67
:103E0000331F280F391F809178009091790063E06B
:103E100070E00E944E8B260F371F369527953695FA
:103E2000279530931E0120931D0185E046C38091A4
:103E30007800909179004091380350913903841BA8
:103E4000950B9093F3018093F2018091F201909190
:103E5000F301029704F172E04E3E570784F420917B
:103E600006022B5F2093060225508091A2029091BA
:103E7000A302845F914018F4215F20930602809191
:103E80000602853684F14F5F5F4F509339034093AC
:103E90003803845626C08091F2019091F3018F5F20
:103EA0009F4F0CF572E047325707ECF02091060265
:103EB0002550209306022B5F8091A2029091A302CD
:103EC000845F914018F42F502093060280910602DF
:103ED0008C394CF44150504050933903409338038F
:103EE0008C5980930602809178009091790090938C
:103EF000E5058093E4058091F2019091F3019C0126
:103F0000442737FD4095542F8091F3029091F4029D
:103F1000A091F502B091F602820F931FA41FB51F66
:103F20008093F3029093F402A093F502B093F6020B
:103F30002091F3023091F4024091F5025091F60283
:103F400057FF04C021503C4F4F4F5F4F6AE05595DB
:103F50004795379527956A95D1F78091F30290910F
:103F6000F402A091F502B091F602821B930BA40B10
:103F7000B50B8093F3029093F402A093F502B093F3
:103F8000F6022EC18091090290910A0220917800D8
:103F900030917900820F931F90930A028093090257
:103FA000109204028CC2809101018A3071F48091D8
:103FB0007800909179002091070230910802820FD9
:103FC000931F01969695879517C0409107025091CF
:103FD0000802843158F02091780030917900240F44
:103FE000351F8FEF97E0821B930B06C080917800FE
:103FF00090917900840F951F9093F9018093F801B7
:1040000086E05BC280913C0390913D032091780053
:1040100030917900821B930B9093E3058093E20526
:104020008091E2059091E3052091110230911202F6
:10403000820F931F9093F7018093F60187E03DC2B2
:10404000809178009091790020913E0330913F0358
:10405000821B930B9093ED058093EC058091EC050A
:104060009091ED052091130230911402820F931F5D
:104070009093F5018093F4011FC220910B023091BF
:104080000C028091780090917900280F391F3093AD
:104090000C0220930B02809101018A3019F4220F47
:1040A000331F04C0220F331F220F331F30930C0223
:1040B00020930B0220910B0230910C02C90137FDB5
:1040C000079603E0959587950A95E1F79093FD0192
:1040D0008093FC0180910D0290910E02820F931F3C
:1040E00097FD01969595879590930E0280930D020A
:1040F0002091480330914903821B930B90931C013C
:1041000080931B01209102023091030280911B01D8
:1041100090911C01280F391F37FF02C02F5F3F4FBE
:1041200035952795309303022093020233CE2091D8
:10413000090230910A028091780090917900280F4D
:10414000391F30930A0220930902809101018A30BD
:1041500019F4220F331F04C0220F331F220F331F05
:1041600030930A02209309022091090230910A0239
:10417000C90137FD0796F3E095958795FA95E1F724
:104180009093FB018093FA0180910F0290911002AD
:10419000820F931F97FD0196959587959093100236
:1041A00080930F022091460330914703821B930BAB
:1041B00090931A018093190120910002309101021D
:1041C0008091190190911A01280F391F37FF02C001
:1041D0002F5F3F4F359527953093010220930002C2
:1041E00083E06BC11092050281E080930F01809102
:1041F000E9019091EA0101969093EA018093E90127
:10420000809178009091790090931401809313012C
:104210008091130190911401AA27BB2720911502C8
:10422000309116024091170250911802280F391F41
:104230004A1F5B1F2093150230931602409317020A
:1042400050931802809119028F5F80931902803178
:1042500008F432C18091150190911601A0911701C7
:10426000B09118017C018D0163E0EE0CFF1C001F72
:10427000111F6A95D1F7E81AF90A0A0B1B0BE20E17
:10428000F31E041F151F8091ED01992787FD90955E
:10429000A92FB92FBC01CD0120EB30E240E050E066
:1042A0000E94238BDC01CB01E81AF90A0A0B1B0BD5
:1042B000D801C7010496A11DB11DB7FF05C0D801E3
:1042C000C7010B96A11DB11D23E0B595A795979544
:1042D00087952A95D1F78093150190931601A093A5
:1042E0001701B09318018091E6059091E7057C01D4
:1042F0000027F7FC0095102F809115019091160171
:10430000A0911701B0911801E81AF90A0A0B1B0BCA
:10431000E092D302F092D4020093D5021093D60219
:104320002091EE013091EF014091F0015091F101A7
:1043300057FF04C0215F3F4F4F4F5F4F84E05595BB
:104340004795379527958A95D1F78091EE01909101
:10435000EF01A091F001B091F101821B930BA40B2E
:10436000B50B8093EE019093EF01A093F001B09311
:10437000F1018091EE019091EF01A091F001B091D7
:10438000F1018E0D9F1DA01FB11F8093EE01909330
:10439000EF01A093F001B093F1018091EE019091B3
:1043A000EF01A091F001B091F101B7FF03C00F96AA
:1043B000A11DB11D14E0B595A795979587951A9500
:1043C000D1F72091D3023091D402281B390B64E03D
:1043D000213036071CF020E034E006C07CEF2030AE
:1043E000370714F420E03CEF8091EB019091EC0151
:1043F0008091EB019091EC0197FF03C0909581951E
:104400009F4FA901F3E0440F551FFA95E1F78D5B2B
:104410009240C4F08091EB019091EC019C01E4E0AA
:10442000220F331FEA95E1F7281B390B240F351FA4
:1044300037FF02C0215F3F4F74E0359527957A958D
:10444000E1F717C08091EB019091EC019C0165E0D0
:10445000220F331F6A95E1F7281B390B240F351FF4
:1044600037FF02C0215E3F4F45E0359527954A95BD
:10447000E1F73093EC012093EB01809115029091CC
:104480001602A0911702B0911802B7FF03C001965F
:10449000A11DB11DB595A795979587958093150298
:1044A00090931602A0931702B093180288E08093AD
:1044B000190202C01092050282E0809304028091EA
:1044C000040280937C0080910502882319F08FEC10
:1044D00080937A00FF91EF91BF91AF919F918F915F
:1044E0007F916F915F914F913F912F911F910F910C
:1044F000FF90EF900F900FBE0F901F90189590E2D5
:10450000E1EFF5E08FE49193815087FFFCCF0895B0
:1045100090911C02903540F4E92FFF27EF50FA4F9D
:1045200080839F5F90931C020895AF92BF92CF92B9
:10453000DF92FF920F931F93CF93DF9320911A0284
:1045400020FF0AC080911B02882311F0815002C015
:1045500080911F0180931B0221FF0CC090911B02D0
:1045600080911F01981719F410921B0203C09F5FDE
:1045700090931B02822F992780FF04C081FF02C005
:1045800010921B020E947F2280911B02282F33274A
:1045900098E8C92E92E2D92EC091FC03D091FD0378
:1045A0008A3098F481E180931C023F932F938FE827
:1045B00094E09F938F93DF92CF92FE0109952DB7E0
:1045C0003EB72A5F3F4F2DBF11C080E180931C0290
:1045D0003F932F9384E994E09F938F93DF92CF9240
:1045E000FE0109958DB79EB706968DBF20911B02DF
:1045F000822F9927AA27BB27FC01419710F00C9422
:10460000ED2BE85AFF4F08E8C02E02E2D02EC091F1
:10461000FC03D091FD030C94E98B10921C0289E9F4
:1046200094E09F938F9308E812E2DF92CF92FE010D
:10463000099584E180931C020F900F900F900F90CA
:1046400085E690E09F938F9388E590E09F938F930A
:104650001F921F92809101016AE00E94428B892F74
:1046600099279F938F93809101010E94428B9927F4
:104670009F938F9389EA94E09F938F93DF92CF92D9
:10468000E091FC03F091FD03099588E280931C0200
:10469000EDB7FEB73E96EDBF8FEB96E09F938F93FD
:1046A0000E946D2F99279F938F938EEB94E09F9399
:1046B0008F93DF92CF92E091FC03F091FD03099577
:1046C0008091160499272DB73EB7285F3F4F2DBF25
:1046D000EC01C071D07084FF06C08CE380931C0293
:1046E0008CEC94E0F1C09091B303992349F18CE3F1
:1046F00080931C02892F99279F938F9389ED94E0D3
:104700009F938F931F930F93E091FC03F091FD0310
:104710000995DF93CF939091B30381E1989FC001F6
:1047200011248551964F9F938F931F930F93E09180
:10473000FC03F091FD0309958DB79EB70C9647C118
:10474000909115049923B1F08CE380931C02892F7A
:1047500099279F938F9381EE94E09F938F931F935C
:104760000F93E091FC03F091FD030995EDB7FEB7BF
:10477000369679C490912202992371F08CE380934C
:104780001C02892F99279F938F9388EF94E09F9322
:104790008F931F930F93D9C480913C0190913D0159
:1047A000069710F00C94F62B8CE380931C028DE09E
:1047B00095E0A5C780912E0818E8C12E12E2D12EEF
:1047C000C091FC03D091FD0380FF6BC010921C02CE
:1047D0008091D3029091D402A091D502B091D602DB
:1047E000BC01CD0125E030E040E050E00E94978B15
:1047F0003F932F938AE195E09F938F93DF92CF921F
:10480000FE01099584E180931C028DB79EB7069640
:104810008DBF8091CF029091D002A091D102B09132
:10482000D202BC01CD0125E030E040E050E00E9422
:10483000978B3F932F9387E295E09F938F93DF921F
:10484000CF92E091FC03F091FD03099588E28093FB
:104850001C02EDB7FEB73696EDBF80911301909123
:1048600014019F938F9384E395E09F938F93DF923E
:10487000CF92E091FC03F091FD0309958CE38093C6
:104880001C022DB73EB72A5F3F4F2DBF87B5992732
:104890009F938F9381E495E09F938F93DF92CF92C4
:1048A0008EC010921C028EE495E09F938F93DF924E
:1048B000CF92FE01099584E180931C020F900F9026
:1048C0000F900F908DE595E09F938F93DF92CF929D
:1048D0001AC710921C0286E695E09F938F9308E812
:1048E00012E2DF92CF92FE01099584E180931C02CF
:1048F0000F900F900F900F9080913303909134039D
:10490000A0913503B0913603B7FF04C081509C4F8E
:10491000AF4FBF4FCAE0B595A79597958795CA95B4
:10492000D1F7BF93AF939F938F9383E795E09F93C6
:104930008F931F930F93E091FC03F091FD03099572
:1049400088E280931C02EDB7FEB73896EDBF8091E8
:104950002B0390912C03A0912D03B0912E03B7FF50
:1049600004C081509C4FAF4FBF4FFAE0B595A7955B
:1049700097958795FA95D1F7BF93AF939F938F93B0
:1049800082E895E09F938F931F930F93E091FC0330
:10499000F091FD0309958CE380931C022DB73EB77F
:1049A000285F3F4F2DBF8091EB079091EC079F93BD
:1049B0008F9381E995E09F938F931F930F93E091DD
:1049C000FC03F091FD0309958DB79EB706968DBF48
:1049D0000DC7E1E0FE2EC1E0D0E007E717E09F2D14
:1049E000969584E1989FC001112480931C02F801E0
:1049F000828193819F938F932196DF93CF93219709
:104A0000808191819F938F93DF93CF9380EA95E08C
:104A10009F938F9388E892E29F938F93E091FC039A
:104A2000F091FD0309952DB73EB7245F3F4F2DBF91
:104A300032E0F30E22960C5F1F4F88E08F1578F658
:104A4000D5C610921C0280914406E82FFF27EE0F76
:104A5000FF1FEB58F84F808191819F938F93809136
:104A60004306E82FFF27EE0FFF1FEB58F84F80811A
:104A700091819F938F9382EB95E09F938F93DF9229
:104A8000CF92FE01099584E180931C02EDB7FEB739
:104A90003896EDBF80914606E82FFF27EE0FFF1FE7
:104AA000EB58F84F808191819F938F9380914506B9
:104AB000E82FFF27EE0FFF1FEB58F84F8081918101
:104AC00081589F4F9F938F9382EC95E09F938F9394
:104AD000DF92CF92E091FC03F091FD03099588E20B
:104AE00080931C022DB73EB7285F3F4F2DBF8091AA
:104AF0004806E82FFF27EE0FFF1FEB58F84F808185
:104B0000918181589F4F9F938F9380914706E82F03
:104B1000FF27EE0FFF1FEB58F84F808191818158DE
:104B20009F4F9F938F9382ED95E09F938F93DF929A
:104B3000CF92E091FC03F091FD0309958CE3809303
:104B40001C028DB79EB708968DBF80914A06E82F4C
:104B5000FF27EE0FFF1FEB58F84F8081918181589E
:104B60009F4F9F938F9380914906E82FFF27EE0F69
:104B7000FF1FEB58F84F8081918181589F4F9F9381
:104B80008F9382EE95E063C210921C0282EF95E053
:104B90009F938F9308E812E2DF92CF92FE0109956E
:104BA000809101010F900F900F900F908A3009F0C3
:104BB0009DC084E180931C02809148039091490339
:104BC0009C0197FF02C0295F3F4F287F821B930BF8
:104BD0009F938F93809148039091490397FD079687
:104BE00073E0959587957A95E1F79F938F93209140
:104BF00048033091490337FF02C0295F3F4F63E00C
:104C0000359527956A95E1F78091FC019091FD011A
:104C1000821B930B9F938F9380E096E09F938F93DB
:104C20001F930F93E091FC03F091FD03099588E237
:104C300080931C022DB73EB7265F3F4F2DBF80915A
:104C40004603909147039C0197FF02C0295F3F4FA5
:104C5000287F821B930B9F938F93809146039091A3
:104C6000470397FD079653E0959587955A95E1F789
:104C70009F938F93209146033091470337FF02C0E3
:104C8000295F3F4F43E0359527954A95E1F780919D
:104C9000FA019091FB01821B930B9F938F9381E10B
:104CA00096E09F938F931F930F93E091FC03F091F5
:104CB000FD0309958CE380931C028DB79EB70A967D
:104CC0008DBF80914403909145039F938F93809172
:104CD0004403909145032091F8013091F901821B22
:104CE000930B9F938F9382E296E0ADC08B3019F0C7
:104CF000843108F4ADC084E180931C0280914803A4
:104D0000909149039C0197FF02C0215F3F4F207F94
:104D1000821B930B97FD0196959587959F938F9393
:104D2000809148039091490397FD0F9624E0959553
:104D300087952A95E1F79F938F93209148033091AF
:104D4000490337FF02C0295F3F4FC3E035952795E0
:104D5000CA95E1F78091FC019091FD01821B930BB4
:104D60009F938F9380E396E09F938F931F930F936E
:104D7000E091FC03F091FD03099588E280931C0209
:104D80002DB73EB7265F3F4F2DBF809146039091D0
:104D900047039C0197FF02C0215F3F4F207F821B8A
:104DA000930B97FD0196959587959F938F9380918F
:104DB00046039091470397FD0F96A4E0959587953C
:104DC000AA95E1F79F938F93209146033091470373
:104DD00037FF02C0295F3F4FF3E035952795FA95DD
:104DE000E1F78091FA019091FB01821B930B9F9355
:104DF0008F9382E496E09F938F931F930F93E0919C
:104E0000FC03F091FD0309958CE380931C028DB7A0
:104E10009EB70A968DBF809144039091450397FDFC
:104E20000196959587959F938F93809144039091D8
:104E300045032091F8013091F901821B930B9F9358
:104E40008F9384E596E09F938F931F930F9303C1F5
:104E50008D3009F0CBC484E180931C028091120153
:104E600099279F938F93809148039091490397FDD1
:104E70000F9674E0959587957A95E1F79F938F93B8
:104E8000209148033091490337FF02C0295F3F4F0B
:104E900063E0359527956A95E1F78091FC01909143
:104EA000FD01821B930B9F938F9383E696E09F9364
:104EB0008F931F930F93E091FC03F091FD030995ED
:104EC00088E280931C022DB73EB7265F3F4F2DBF6F
:104ED0008091110199279F938F9380914603909120
:104EE000470397FD0F9654E0959587955A95E1F7FE
:104EF0009F938F93209146033091470337FF02C061
:104F0000295F3F4F43E0359527954A95E1F780911A
:104F1000FA019091FB01821B930B9F938F9387E77C
:104F200096E09F938F931F930F93E091FC03F09172
:104F3000FD0309958CE380931C028DB79EB70A96FA
:104F40008DBF8091100199279F938F938091440387
:104F50009091450397FD0196959587959F938F9323
:104F600080914403909145032091F8013091F9011B
:104F7000821B930B9F938F938BE896E09F938F9365
:104F80001F930F93E091FC03F091FD030995EDB79A
:104F9000FEB73A9668C010921C028FE996E09F9384
:104FA0008F93DF92CF92FE01099584E180931C02DA
:104FB0000F900F900F900F9080913E0390913F03C0
:104FC0009F938F938091F4019091F5019F938F931C
:104FD0008CEA96E09F938F93DF92CF92E091FC034F
:104FE000F091FD03099588E280931C022DB73EB72E
:104FF000285F3F4F2DBF80913C0390913D039F93CD
:105000008F938091F6019091F7019F938F938BEB93
:1050100096E09F938F93DF92CF92E091FC03F09103
:10502000FD0309958CE380931C028DB79EB708960B
:105030008DBF80913803909139039F938F93809116
:10504000F2019091F3019F938F938AEC96E09F93E6
:105050008F93DF92CF92E091FC03F091FD030995CD
:10506000EDB7FEB73896EDBFC1C310921C02809118
:105070001D0190911E016AE070E00E94628B9F9377
:105080008F9380911D0190911E016AE070E00E9453
:10509000628B7F936F9389ED96E09F938F93DF925E
:1050A000CF92FE01099584E180931C022DB73EB793
:1050B000285F3F4F2DBF8091CE089091CF086AE0C6
:1050C00070E00E944E8B9F938F938091CE089091B9
:1050D000CF086AE070E00E944E8B7F936F938DEE55
:1050E00096E09F938F93DF92CF92E091FC03F09133
:1050F000FD03099588E280931C028DB79EB7089640
:105100008DBF8091D0089091D1089F938F9381E0BB
:1051100097E09F938F93DF92CF92E091FC03F09101
:10512000FD0309958CE380931C02EDB7FEB736961C
:10513000EDBF8091D2089091D3089F938F9381E126
:1051400097E09F938F93DF92CF92E091FC03F091D1
:10515000FD0309952DB73EB72A5F3F4F4FC110920F
:105160001C0283E297E09F938F93DF92CF92FE0120
:10517000099584E180931C020F900F900F900F907F
:1051800080917507909176079F938F938CE297E0BB
:105190009F938F93DF92CF92E091FC03F091FD03F8
:1051A000099588E280931C028DB79EB706968DBF45
:1051B0008091D90299279F938F938CE397E09F93D7
:1051C0008F93DF92CF92E091FC03F091FD0309955C
:1051D0008CE380931C02EDB7FEB73696EDBF80914D
:1051E0007407992701979F938F938CE497E0A9CF39
:1051F00010921C028CE597E09F938F93DF92CF92E1
:10520000FE01099584E180931C020F900F900F908E
:105210000F9080918E0190918F019F938F9384E6E0
:1052200097E09F938F93DF92CF92E091FC03F091F0
:10523000FD03099588E280931C028DB79EB7069600
:105240008DBF8091EB079091EC079F938F9382E73E
:1052500097E09F938F93DF92CF92E091FC03F091C0
:10526000FD0309958CE380931C02EDB7FEB73696DB
:10527000EDBF8091F1029091F2029F938F9380E8AD
:1052800097E05FCFCAEDCC2EC2E0DC2E20E030E00C
:10529000E901B3E0FB2EC0931C02F60181916F017E
:1052A00099279F938F9389010F5F1F4F1F930F9330
:1052B0008EE897E09F938F9388E892E29F938F9375
:1052C000E091FC03F091FD0309952DB73EB7285FEF
:1052D0003F4F2DBFFA9464969801F7FEDCCF86C24B
:1052E000AEEDCA2EA2E0DA2EC0E0D0E08E01F3E0EF
:1052F000FF2E00931C02F60181916F0199279F9365
:105300008F932596DF93CF938BE997E09F938F93AD
:1053100088E892E29F938F93E091FC03F091FD0364
:1053200009952DB73EB7285F3F4F2DBFFA940C5E0D
:105330001F4F2497F7FEDDCF59C210921C0288EA56
:1053400097E09F938F9308E812E2DF92CF92FE01DD
:10535000099584E180931C020F900F900F900F909D
:1053600080916D0199279F938F9380EB97E09F9396
:105370008F93DF92CF92E091FC03F091FD030995AA
:1053800088E280931C028DB79EB706968DBF8091F0
:10539000D4019091D50197FD0396959587959595A4
:1053A00087959F938F938EEB97E09F938F931F9397
:1053B0000F93E091FC03F091FD0309958CE380933A
:1053C0001C02EDB7FEB73696EDBF809172069927A5
:1053D0009F938F938091710699279F938F938CEC65
:1053E00097E09F938F931F930F93E091FC03F091AD
:1053F000FD0309952DB73EB7285F3F4F2DBFF6C17E
:1054000010921C028AED97E09F938F9378E8A72E65
:1054100072E2B72EDF92CF92FE0109950F900F90A6
:105420000F900F90C4E1D7E000E010E062E0F62EAC
:10543000802F8C5E80931C028B8D99278F779070C4
:105440009F938F938B8999278F7790709F938F93DA
:105450008B8599278F7790709F938F938B81992756
:105460008F7790709F938F938AEE97E09F938F939F
:10547000BF92AF92E091FC03F091FD0309958DB7C7
:105480009EB70C968DBFFA940C5E1F4FA096F7FE48
:10549000CFCFACC110921C028BEF97E09F938F93FC
:1054A00058E8A52E52E2B52EDF92CF92FE01099563
:1054B0000F900F900F900F90C4E1D7E000E010E044
:1054C00042E0F42E802F8C5E80931C028F8D9927F2
:1054D00087FD90959F938F938F89992787FD90954E
:1054E0009F938F938F85992787FD90959F938F9397
:1054F0008F81992787FD90959F938F938AE098E0FD
:105500009F938F93BF92AF92E091FC03F091FD03C4
:105510000995EDB7FEB73C96EDBFFA940C5E1F4FB0
:10552000A096F7FECFCF62C110921C028BE198E0EB
:105530009F938F9308E812E2DF92CF92FE010995C4
:1055400084E180931C020F900F900F900F90809138
:105550002F07881F8827881F97E0899FC001112483
:105560008D969F938F9380912707881F8827881F88
:1055700096E0899FC00111248D969F938F9380910F
:105580001F07881F8827881F95E0899FC001112465
:105590008D969F938F9380911707881F8827881F68
:1055A0009927880F991F880F991F8D969F938F9326
:1055B0008AE298E09F938F93DF92CF92E091FC0371
:1055C000F091FD03099588E280931C022DB73EB748
:1055D000245F3F4F2DBF80914F07881F8827881F6A
:1055E0009BE0899FC00111248D969F938F9380919A
:1055F0004707881F8827881F9AE0899FC0011124C8
:105600008D969F938F9380913F07881F8827881FCF
:1056100099E0899FC00111248D969F938F9380916B
:105620003707881F8827881F992723E0880F991F2D
:105630002A95E1F78D969F938F938EE398E09F9341
:105640008F93DF92CF92E091FC03F091FD030995D7
:105650008CE380931C028DB79EB70C968DBF809112
:105660005707881F8827881F9CE0899FC001112445
:105670008D969F938F9382E598E09F938F93DF920F
:10568000CF92E091FC03F091FD03099580915F07B3
:10569000EDB7FEB73696EDBF87FF12C080E480936A
:1056A0001C0283E698E09F938F93DF92CF92E09164
:1056B000FC03F091FD0309950F900F900F900F9050
:1056C0008091670787FF12C084E480931C0286E6FE
:1056D00098E09F938F931F930F93E091FC03F091B9
:1056E000FD0309950F900F900F900F9080916F0719
:1056F00087FF7CC088E480931C0289E698E09F9332
:105700008F931F930F93E091FC03F091FD03099594
:105710000F900F900F900F9069C010921C028CE6B2
:1057200098E09F938F93DF92CF92FE01099584E1D9
:1057300080931C020F900F900F900F908091AA0100
:105740009091AB019F938F938AE798E09F938F93FB
:10575000DF92CF92E091FC03F091FD03099588E27E
:1057600080931C022DB73EB72A5F3F4F2DBF80911B
:10577000AC019091AD019F938F9387E898E09F9340
:105780008F93DF92CF92E091FC03F091FD03099596
:1057900089E480931C028DB79EB706968DBF84E97D
:1057A00098E09F938F93DF92CF92E091FC03F0916A
:1057B000FD03099580911A020F900F900F900F90A2
:1057C00083FF14C01092AD011092AC0160E070E054
:1057D0008EE090E00E940A2E09C080911F012817D8
:1057E00019F4215020931F0110921B0210921A02EB
:1057F000DF91CF911F910F91FF90DF90CF90BF90DD
:10580000AF900895F999FECF92BD81BDF89A80B509
:1058100099270895F999FECF1FBA92BD81BD60BD49
:105820000FB6F894FA9AF99A0FBE08954AEA20E062
:1058300030E02617370740F4FC018191480F2F5FB5
:105840003F4F26173707C8F3842F99270895EAEAB0
:1058500040E050E04617570778F49C01F999FECFD5
:1058600032BD21BDF89A80B5E80F4F5F5F4F2F5FC3
:105870003F4F4617570790F38E2F9927089581E0E1
:105880008093450682E08093440683E0809343063C
:1058900084E08093460685E08093470686E0809307
:1058A000480687E08093490688E080934A0689E0AD
:1058B00080934B068AE080934C068BE080934D06E4
:1058C0008CE080934E0608958AE58093420680918D
:1058D0000101843150F08AE08093620610928606BE
:1058E0008BE180935E068EE40AC083E080936206BB
:1058F00080E2809386068EE180935E0685E5809344
:1059000083068093840680E2809385061092AD061C
:105910008AE680934F0682E28093AF061092B0062B
:1059200064E0609369061092A5061092A20648E012
:1059300040935C0656EE50935D0680E480935F06CC
:105940009EE1909350068FEF809352062FE02093B4
:10595000530690935106109255064093560684E1E3
:1059600080935706109258062093540610926B06A7
:1059700010926C0610926D0610926E0610928806B8
:105980001092890610928A0610928B0690E89093E6
:105990006F0632E33093700682E08093AE06209368
:1059A000710650937206609377068DE780937A06AE
:1059B00080937B0680937C069093730625E5209365
:1059C000740686E4809375068CED809376068CE3EE
:1059D00080937806109279068FE580938C0683EF8A
:1059E00080938E068AEA809390068093910688E2DF
:1059F00080938D0680938F0630937D069AE5909371
:105A00007E0630937F068EEF8093920684E6809325
:105A100093069093940690939506909396068BE444
:105A200080939706209398068093990610929A0681
:105A300086E080939B0640939C0690939D068AE2A5
:105A400080939E0685EF80939F068CE88093A00646
:105A500085E08093A1061092A3061092A40681E22D
:105A60008093660681E4809367069093680610929F
:105A7000A6061092A7061092A80686E98093A906AA
:105A80009093800687E3809381061092AA06109275
:105A9000AB061092AC060895CF93DF930E94642C5E
:105AA0008AE08093590680E180935A0626E020938D
:105AB0005B069AE59093600688E780936106909371
:105AC0006306809364062093650680E280936A06ED
:105AD0008CE3809382068BE480938706A1EBB6E08B
:105AE0008CE0E0E2F1E0ED01019009928A95E1F7A6
:105AF0006BE770E0CD018F5690400E94162C80938A
:105B0000BD06DF91CF910895CF93DF930E94642C5F
:105B100088E08093590630E130935A0626E02093BE
:105B20005B0694E69093600688E780936106909305
:105B30006306809364062093650630936A0686E4C4
:105B40008093820680938706A1EBB6E08CE0E6E2C4
:105B5000F1E0ED01019009928A95E1F76BE770E0C1
:105B6000CD018F5690400E94162C8093BD06DF9188
:105B7000CF910895CF93DF930E94642C26E0209369
:105B800059068AE080935A0684E080935B0694E687
:105B90009093600688E780936106909363068093F4
:105BA00064062093650680E180936A0686E480930C
:105BB000820680938706A1EBB6E08CE0EEE2F1E08E
:105BC000ED01019009928A95E1F76BE770E0CD0154
:105BD0008F5690400E94162C8093BD06DF91CF9186
:105BE0000895F999FECF92BD81BDF89A80B59927A5
:105BF0000895F999FECF1FBA92BD81BD60BD0FB661
:105C0000F894FA9AF99A0FBE089562E07CE20E9435
:105C1000B18908954AE05CE20E94EB890895EF9211
:105C2000FF920F931F93CF93C82F8150853008F0B8
:105C3000C3E08CE7C89F8001112488EEE82E8FEF27
:105C4000F82EE00EF11E6BE770E0C7010E94272CD2
:105C5000682F98012D593F4F8FB39927AC0142709F
:105C6000507081FDF9CF32BD21BDF89A80B58617FD
:105C700011F0CA0123C08FB399279C0122703070A4
:105C800081FDF9CFF2BCE1BCF89A80B58A3511F0FC
:105C9000C90114C08CE7C89FC0011124489722E0B5
:105CA0003CE24CE750E0BC0182E496E00E948C8923
:105CB0000E94CA6B0E94868581E090E0CF911F917F
:105CC0000F91FF90EF900895282F863010F025E077
:105CD00003C0882309F421E0F999FECF1FBA82E0BE
:105CE00090E092BD81BD20BD0FB6F894FA9AF99A62
:105CF0000FBE0895CF93C82F809142068A3509F0D0
:105D000051C0C63010F0C5E003C0CC2309F44AC02E
:105D10000E947E888091B00682FF07C0809167064E
:105D2000843618F080E5809367066BE770E082E4C4
:105D300096E00E94162C8093BD068CE7C89FC00198
:105D400011242AE03CE24CE750E062E476E0489718
:105D50000E94C9892AE03CE24CE050E063E476E02E
:105D600080E590E00E94C9896CE070E083E496E0F1
:105D70000E94162C282FF999FECF1FBA8CE590E0CF
:105D800092BD81BD20BD0FB6F894FA9AF99A0FBE64
:105D90008C2F0E94642E0E94CA6B0E94868581E02F
:105DA00090E002C080E090E0CF9108956DE470E053
:105DB00088EE93E00E94272C482F8FB399279C01EF
:105DC0002270307081FDF9CF85E394E092BD81BDF2
:105DD000F89A80B5841779F48FB399279C012270C3
:105DE000307081FDF9CF88EE93E092BD81BDF89AC5
:105DF00080B5813011F0C901089522E03CE24EE403
:105E000050E068EE73E08EEB96E00E948C8981E0B2
:105E100090E008958091BE068130A9F46DE470E0B1
:105E20008EEB96E00E94162C80930B072AE03CE252
:105E30004EE450E06EEB76E088EE93E00E94C98974
:105E400081E090E0089580E090E00895CF93DF93A3
:105E500081E08093BE06EEEBF6E08FE015861686B5
:105E60001786108A8150349687FFF8CF80E480939C
:105E7000CB068093CC061092CD068093CE068093FD
:105E8000CF0690EC9093D0061092D1068093D20664
:105E90008093D3061092D4069093D5069093D6069D
:105EA0008093D7061092D8068093D9069093DA068D
:105EB000AFEBB6E087E0E4E3F1E0ED010190099299
:105EC0008A95E1F76DE470E0CD0101970E94162CF0
:105ED00080930B07DF91CF910895F999FECF82E06F
:105EE00090E092BD81BDF89A80B5282F863078F079
:105EF00023E0322FF999FECF1FBA82E090E092BDE5
:105F000081BD30BD0FB6F894FA9AF99A0FBE822F70
:105F1000992708951F93CF93C82F162F863010F01E
:105F2000C5E003C0882309F4C1E08C2F9927823093
:105F3000910541F08330910544F4019731F40E94BA
:105F40004C2D05C00E94842D02C00E94BA2D112341
:105F5000E1F06CE070E080E590E00E94272C282FB3
:105F6000F999FECF8CE590E092BD81BDF89A80B59D
:105F7000821759F422E03CE24CE050E060E570E02A
:105F800083E496E00E948C8902C00E943F2C8C2FF3
:105F90000E947A2ECF911F910895DF92EF92FF9287
:105FA0000F931F93CF93FF24DF2CEF2C81E090E021
:105FB0000E94F12D8A3511F031E0E32E6CE070E0A3
:105FC00080E590E00E94272CC82FF999FECF8CE540
:105FD00090E092BD81BDF89A80B58C1711F421E054
:105FE000D22EC1E001E010E0EE2029F48C2F0E94B7
:105FF0000F2E8823C9F591E0F92E1F930F938CE99A
:1060000098E09F938F938FEB94E19F938F93E09110
:10601000FC03F091FD0309952DB73EB72A5F3F4F72
:106020002DBF0230110549F0033011054CF4013049
:10603000110531F40E944C2D05C00E94842D02C030
:106040000E94BA2DDD2059F022E03CE24CE050E005
:1060500060E570E083E496E00E948C8902C00E94B3
:106060003F2C8C2F0E947A2ECF5F0F5F1F4FC630C0
:1060700008F4BACFFF2019F083E00E94642E0E943A
:106080006D2FC82F0E940F2E8C2F99279F938F93CF
:1060900082EC98E09F938F930FEB14E11F930F9383
:1060A000E091FC03F091FD03099581E090E00E94EE
:1060B000F12D2DB73EB72A5F3F4F2DBF8F3F21F007
:1060C0000E94D62E882399F48BED98E09F938F93AE
:1060D0001F930F93E091FC03F091FD0309950E943B
:1060E000262F0E940A2F0F900F900F900F90EE20F6
:1060F00029F06AE581E090E00E94F92D10924106B6
:1061000090E0EBECF6E0CFE08081349618160CF4CA
:106110009F5FC150C7FFF8CF90934106892F992701
:106120009F938F938FEB96E09F938F938CEF98E0E4
:106130009F938F931F930F93E091FC03F091FD03C6
:1061400009950E94CC088DB79EB708968DBFCF9158
:106150001F910F91FF90EF90DF900895982F2FB728
:10616000F8943998389A88B1836088B98091B900D9
:106170008C7F8093B9008AE28093B8001092270246
:106180001092250210922402992379F0E4E1F7E0BD
:106190008BE0108211821282138214821582168281
:1061A00017828150389687FFF4CF78942FBF0895D7
:1061B0001092270284E98093BC0080E88093BC00A1
:1061C0001092BD001092BA001092BB001092B9005C
:1061D0001092B8001092230280E00E94AE3010921C
:1061E000BB0085E88093BC0080912102826080938F
:1061F000210208951F920F920FB60F9211242F9330
:106200003F934F935F938F939F93EF93FF9380916F
:106210002702282F3327442755278F5F8093270293
:10622000F9012731310508F0C2C2E759FF4F0C943C
:10623000E98B81E08093230209C0809125028C3094
:1062400090F4809125028F5F809325028091250232
:10625000E82FFF27EE0FFF1FEE0FFF1FE254F94F4D
:106260008585181654F7809125028C3070F01092B5
:10627000200210921F021092250285E080932702CF
:1062800080912402880F8D5A04C080912502880FC6
:106290008E5A8093BB0085E87FC280912502E82F4B
:1062A000FF2783E0EE0FFF1F8A95E1F7EC5EF84FC2
:1062B00081818093BB0085E88093BC00809125029A
:1062C000E82FFF27EE0FFF1FEE0FFF1FEE0FFF1F40
:1062D000EC5EF84F808180FF91C080912502E82F0D
:1062E000FF27EE0FFF1FEE0FFF1FEE0FFF1FEC5EED
:1062F000F84F8281882329F080914106873008F485
:106300006CC280911F0290912002892B09F065C216
:1063100080911D0290911E02892B09F05EC26EC011
:106320008091250221E030E002C0220F331F8A95C0
:10633000E2F780911D0290911E0228233923232B1E
:1063400079F080912502E82FFF27EE0FFF1FEE0F57
:10635000FF1FEE0FFF1FEC5EF84F80E184830DC03E
:1063600080912502E82FFF27EE0FFF1FEE0FFF1F82
:10637000EE0FFF1FEC5EF84F148280912502E82F8C
:10638000FF2753E0EE0FFF1F5A95E1F7EC5EF84F41
:106390008481282F332743E0220F331F4A95E1F7EA
:1063A00080912502E82FFF2793E0EE0FFF1F9A95BB
:1063B000E1F7EC5EF84F82818770822B8093BB00FF
:1063C00085E88093BC002091250281E090E002C026
:1063D000880F991F2A95E2F720911F023091200221
:1063E00082239323892B51F08CE097E090932B022A
:1063F00080932A0288E080932C02EFC184E089C157
:10640000E0912A02F0912B0281918093BB0085E8F4
:106410008093BC00F0932B02E0932A0280912C021F
:10642000815080932C02882309F4D7C183E071C185
:106430008091B900803351F580912802882329F496
:10644000809125028F5F8093280280912502E82F9A
:10645000FF2783E0EE0FFF1F8A95E1F7EC5EF84F10
:10646000838199278F7790708F3791057CF4809185
:106470002502E82FFF27EE0FFF1FEE0FFF1FEE0F85
:10648000FF1FEC5EF84F83818F5F8383109227029A
:1064900084E98093BC008AE090E090933D01809372
:1064A0003C01809125028F5F809325021092270284
:1064B0006DC18091B9008034C9F180912402E82F28
:1064C000FF27EE0FFF1FEE0FFF1FEE0FFF1FEC5E0B
:1064D000F84F83818F778383809124028F5F80932D
:1064E0002402809124028C30A0F010922402109299
:1064F0001E0210921D02809129028F5F8093290253
:106500008C3038F010922902809121028D7F809387
:106510002102809121028160809321021092270242
:1065200084E98093BC001092230273C080912402FE
:10653000E82FFF27EE0FFF1FEE0FFF1FEE0FFF1FCD
:10654000EC5EF84F83818068838380912402E82F7A
:10655000FF27EE0FFF1FEE0FFF1FEE0FFF1FEC5E7A
:10656000F84F808180FF2FC080912402E82FFF2701
:1065700053E0EE0FFF1F5A95E1F7EC5EF84F848170
:106580009927009751F04097D9F58CE097E09093C8
:106590002B0280932A0288E031C08091240299273F
:1065A00043E0880F991F4A95E1F7875E984F9093D3
:1065B0002B0280932A02909124028091290298173D
:1065C000E1F483E01BC080912402992733E0880F17
:1065D000991F3A95E1F7875E984F90932B0280932D
:1065E0002A028091210281FD06C0909124028091AF
:1065F0002902981711F482E001C081E080932C02F7
:1066000080912C02813011F485E801C085EC8093E3
:10661000BC00809128028093220210922802DDC0E3
:10662000E0912A02F0912B028091BB00808380913F
:106630002A0290912B02019690932B0280932A02BA
:1066400080912C02815080932C02823010F085ECD6
:106650005DC0813011F485E859C08091210281FF2D
:106660002DC08091A10280FD1DC080912402E82FE1
:10667000FF2723E0EE0FFF1F2A95E1F7EC5EF84FAE
:1066800086818A3F79F480912402E82FFF2793E0E6
:10669000EE0FFF1F9A95E1F7EC5EF84F8081816065
:1066A00080830CC080912402E82FFF2783E0EE0F47
:1066B000FF1F8A95E1F7EC5EF84F1082809124026B
:1066C0008F5F80932402809124028C30A0F010927E
:1066D000240210921E0210921D02809129028F5FE7
:1066E000809329028C3038F0109229028091210287
:1066F0008D7F809321021092270284E98093BC0051
:106700008091210281608093210265C08093BC004A
:1067100086E08093270261C088E9BBCD8091260284
:10672000880F805FB6CD8091260299278130910530
:1067300061F0823091051CF4892B21F04EC0029744
:1067400039F04BC080911201A4CD80911101A1CDEF
:10675000809110019ECD80E89CCD1092270284E9A3
:106760008093BC00109223028AE090E090933D0158
:1067700080933C0180912602823088F48091260229
:106780008F5F8093260282E180932702809121020D
:106790008E7F8093210285EA8093BC001EC01092F8
:1067A00026028091210281608093210216C01092FE
:1067B000270284E98093BC0080912102816080934C
:1067C00021028AE090E090933D0180933C01109279
:1067D00025021092240210922302FF91EF919F91C3
:1067E0008F915F914F913F912F910F900FBE0F901E
:1067F0001F9018951F93CF93DF93182F8091D80285
:10680000882321F48091B901882319F081E090E078
:1068100097C01D3008F092C01123B1F0E12FFF277F
:1068200023E0EE0FFF1F2A95E1F7EC5EF84F359756
:106830008081359688230CF081C03897808180FD57
:1068400003C083E090E07CC080910C07823019F097
:1068500084E090E075C067E070E08CE097E00E9413
:10686000162C90911307891719F085E090E068C005
:1068700080ED97E00E94CE18EC018091210280FD0E
:1068800005C0CE010E94D7188823B9F3112319F44B
:106890008FEF90E00BC0212F33272150304081E053
:1068A00090E002C0880F991F2A95E2F7909320028A
:1068B00080931F02A1E0B0E0E4E1F7E040E050E0A7
:1068C0006BE0CD01042E02C0880F991F0A94E2F7F5
:1068D00020911F023091200282239323892B11F0F3
:1068E0001182128261504F5F5F4F389667FFE9CF88
:1068F0001092250210922702809121028E7F8093B0
:10690000210285EA8093BC008091210280FD05C0B0
:10691000CE010E94D7188823B9F380911F0290916D
:106920002002892B29F0CE010E94D718882311F369
:1069300080911F0290912002009711F082E090E078
:10694000DF91CF911F9108950F931F93CF93DF9302
:10695000982F8091D802882321F48091B90188234F
:1069600019F081E090E092C09D30A0F4992319F4D1
:1069700086E090E08BC0C92FDD27FE0133E0EE0FEB
:10698000FF1F3A95E1F7EC5EF84F35978081359619
:1069900087FD03C082E090E079C03897808180FD58
:1069A00003C083E090E072C080ED97E00E94CE18B3
:1069B0008C018091210280FD05C0C8010E94D7187A
:1069C0008823B9F3219721E030E0C90102C0880F84
:1069D000991FCA95E2F790931E0280931D02D90178
:1069E000E4E1F7E040E050E06BE0CD01042E02C0AE
:1069F000880F991F0A94E2F720911D0230911E0220
:106A000082239323892B11F01182128261504F5FF0
:106A10005F4F389667FFE9CF1092240210920C075F
:106A20001092130710922702809121028E7F80938B
:106A3000210285EA8093BC008091210280FD05C07F
:106A4000C8010E94D7188823B9F380911D02909144
:106A50001E02892B29F0C8010E94D718882311F340
:106A600080910C07823019F084E090E00FC067E05D
:106A700070E08CE097E00E94162C90911307891724
:106A800019F085E090E002C080E090E0DF91CF91C6
:106A90001F910F910895CF93DF9380E022E83FEF9D
:106AA000C9EAD7E0E5E7F7E0DF01853020F4119689
:106AB0001C921E9202C03183208319821882229672
:106AC0008F5F129632968A3180F3109245031092AE
:106AD0004403109247031092460310924903109208
:106AE0004803DF91CF9108951F920F920FB60F9236
:106AF00011240F931F932F933F934F935F936F93A3
:106B00007F938F939F93AF93BF93CF93DF93EF9335
:106B1000FF938091AF0682FDE1C0409186005091C5
:106B2000870080912E0290912F02481B590B809173
:106B300086009091870090932F0280932E02CA01C5
:106B40008D549440A0913002B0913102835F9A41FC
:106B500078F48091300280937407149714F01092A7
:106B6000400181E090E090933102809330022BC28B
:106B7000AD30B1050CF027C2CA018B5F9040845B39
:106B8000914008F086C080913E0190913F01481BE2
:106B9000590BE091AA06EE2351F0FF27EE0FFF1FDD
:106BA000EB58F84F8081918184369105ECF4FD011A
:106BB000EA0FFB1FEB58F84F80819181FA01E81B27
:106BC000F90BCF01F7FF03C0909581959F4F069772
:106BD0005CF48091D902883C20F48091D902865FD0
:106BE00001C088EC8093D902FD01EA0FFB1FEB582E
:106BF000F84F808191819C01220F331F280F391F8C
:106C0000240F351F37FF02C02D5F3F4FE901D59597
:106C1000C795D595C795CA0101968C179D0714F4A1
:106C2000219706C041505040C417D5070CF4219657
:106C30008091D902833CE0F08D010A0F1B1FF801FF
:106C4000EB58F84F808191819E01281B390BC901B7
:106C500063E070E00E94628BCB01880F991F860F62
:106C6000971F0755184FD80111969C938E9307C014
:106C7000AA0FBB1FA755B84F11961C921E92E09108
:106C80003002F0913102EE0FFF1FEB58F84FD18325
:106C9000C08320913002309131022F5F3F4F3093FB
:106CA00031022093300280910101843108F08BC1C0
:106CB0002530310511F45D9A01C05D988091300254
:106CC000909131028630910511F45C9A01C05C9874
:106CD000079711F45B9A77C15B9875C14091860064
:106CE000509187008091320290913302481B590BDA
:106CF00080918600909187009093330280933202B6
:106D0000CA018D54944060919C02835F9A4108F0BF
:106D10007AC060932D0280912D02843008F453C014
:106D20009091740780912D02981709F04CC05091F2
:106D30009D025B3008F43FC01092400110929C020B
:106D400040E05F31C0F0E42FFF27EE0FFF1F9F01EF
:106D500028593D4FDF01AB58B84F8D919C91D90117
:106D60008D939C93DF01A755B84F8D919C91EE5761
:106D7000FD4F91838083E42FFF27EE0FFF1F9F01BC
:106D80002B58384FDF01AC5CBD4F8D919C91D901E0
:106D900011969C938E93DF01A25BBD4F8D919C91C8
:106DA000E755F84F91838083842F8F5F482F8D3074
:106DB00040F280939C0280919D028F3FB9F08F5FDB
:106DC00080939D0213C080919D02853620F08AE059
:106DD00080939D0202C010929D02809101018A3031
:106DE00011F0843110F0289A01C0289881E0809336
:106DF0009C028091D802882309F0E5C080912D0281
:106E000080937407E0C06D3008F0B5C0CA018B5F95
:106E10009040845B914008F090C080913E01909139
:106E20003F01481B590BE62FFF27EE0FFF1FEC5CBD
:106E3000FD4F80819181FA01E81BF90BCF01059686
:106E40000B9720F5E091AA06EE2351F0FF27EE0FF5
:106E5000FF1FEB58F84F8081918184369105B4F47F
:106E600080919D028A3120F08091D902865F05C011
:106E70008B3028F08091D9028E5F8093D902809167
:106E8000D902893C18F088EC8093D902E62FFF27BD
:106E9000EE0FFF1FEC5CFD4F808191819C01220F62
:106EA000331F280F391F240F351F37FF02C02D5FF6
:106EB0003F4FE901D595C795D595C795CA0101966C
:106EC0008C179D0714F4219706C041505040C417F9
:106ED000D5070CF421968091D9028E3BD8F0E62F8D
:106EE000FF27EE0FFF1FDF01AC5CBD4F8D919C9122
:106EF0009E01281B390BC90163E070E00E94628B80
:106F0000CB01880F991F860F971FE25BFD4F91837E
:106F1000808308C0E62FFF27EE0FFF1FE25BFD4FC7
:106F20001182108280919C02E82FFF27EE0FFF1F35
:106F3000EC5CFD4FD183C08309C0809101018A3090
:106F400011F0843110F0289A01C028988091010135
:106F5000843188F480919C02853011F45D9A05C0DB
:106F60005D98863011F45C9A05C05C98873011F406
:106F70005B9A01C05B9880919C02843120F48F5F02
:106F800080939C0220C08431F1F4809101018A3009
:106F900011F0843110F0289A01C028988EE1809376
:106FA0009C022CE0C9EAD7E0A8E6B2E0E5E7F7E00A
:106FB0008D919D91918380833296198218822296B9
:106FC000215027FFF5CFFF91EF91DF91CF91BF9136
:106FD000AF919F918F917F916F915F914F913F9171
:106FE0002F911F910F910F900FBE0F901F9018952A
:106FF000EF92FF920F931F9380915E069927880F5F
:10700000991F880F991F7C010027F7FC0095102F0E
:107010008091330390913403A0913503B0913603EE
:10702000BC01CD01A80197010E94978B3093A20566
:107030002093A10580912B0390912C03A0912D0307
:10704000B0912E03BC01CD01A80197010E94978B3E
:107050003093A4052093A3058091320890913308C2
:1070600097FD039695958795959587959093A60599
:107070008093A505809142089091430897FD03965F
:1070800095958795959587959093A8058093A705E5
:1070900080914403909145032091F8013091F901CA
:1070A000821B930B9093AA058093A9058091D3022C
:1070B0009091D402A091D502B091D602BC01CD012D
:1070C00025E030E040E050E00E94978B3093AC0523
:1070D0002093AB058091F2019091F3019093AE055E
:1070E0008093AD0580918E0190918F019093B205B0
:1070F0008093B10580911D0190911E019093B4057C
:107100008093B3058091D90299279093B605809317
:10711000B5058091EB079091EC079093B8058093AB
:10712000B7058091150799279093BA058093B90503
:1071300080911D0799279093BC058093BB05809192
:10714000250799279093BE058093BD0580912D0753
:1071500099279093C0058093BF058091D4019091A9
:10716000D5019093CA058093C9058091CE0890916E
:10717000CF089093CE058093CD058091D208909151
:10718000D3089093D0058093CF058091CF02909142
:10719000D002A091D102B091D202BC01CD0125E074
:1071A00030E040E050E00E94978B3093D20520936E
:1071B000D1058091F1029091F2029093D8058093CD
:1071C000D7058091D40899279093DC058093DB053F
:1071D0008091A4039091A5039093DE058093DD0533
:1071E0008091A2039091A3039093E0058093DF0523
:1071F00080911504882321F480911604882321F0BE
:107200008091A005816003C08091A0058E7F80934E
:10721000A0051F910F91FF90EF9008951F93CF93BA
:10722000DF93182FEB018091D802882309F5809114
:1072300001018C3010F4299801C0299A11501F3F88
:1072400081F0D093DB01C093DA018091DA01909153
:10725000DB01892BD1F7CE018C0F9D1F0E94E31813
:10726000EDCF809101018C3010F4299A01C029984A
:10727000DF91CF911F910895CF93DF93809101010A
:107280008D3011F40E946D1D10927A008091FC01E6
:107290009091FD019093F7078093F6078091FA0192
:1072A0009091FB019093E7078093E6078091F801A6
:1072B0009091F90190933808809337082091F40158
:1072C0003091F501C901880F991F880F991F820F0E
:1072D000931F820F931F909333088093320820915D
:1072E000F6013091F701C901880F991F880F991F86
:1072F000820F931F820F931F90934308809342083D
:107300008FEC80937A00AAEDB2E0C7E4D6E097E074
:107310008991E82FFF27EE0FFF1FEB58F84F0190E0
:10732000F081E02DE158FF4F1E161F061CF0E0E033
:10733000F0E005C0EF3FF10514F0EFEFF0E08C91C5
:10734000282F3327E217F30714F4815004C02E17B7
:107350003F0714F48F5F8C939150119697FFD8CF0D
:10736000809183069927AA27BB27BC01CD0124EC75
:1073700039E040E050E00E94238BDC01CB01809398
:10738000860190938701A0938801B0938901809131
:1073900084069927AA27BB27BC01CD010E94238B15
:1073A000DC01CB018093820190938301A09384013F
:1073B000B0938501DF91CF910895A0E0B0E0E3EEB6
:1073C000F9E30C94B88B882EC0E0D0E07E016E010A
:1073D00010921504469AD0933F03C0933E03D09376
:1073E0003D03C0933C03D0933903C0933803D0933B
:1073F0004903C0934803D0934703C0934603D093F7
:107400004503C093440310926A01109269011092DF
:10741000ED010E943C3984E690E00E94F0180E9441
:107420003C3980914F0680FF10C0809113019091EC
:107430001401875B934038F48091130190911401FB
:107440008E5E924010F40E94EB1C0FE18AE090E007
:107450000E94F0188091F8019091F901C80FD91F8E
:107460008091FC019091FD01E80EF91E8091FA01D6
:107470009091FB01C80ED91E015007FFE7CF97017D
:10748000205F3F4F369527953695279530934903D2
:1074900020934803C60140969695879596958795C3
:1074A00090934703809346036096F5E0D695C79581
:1074B000FA95E1F7D0934503C093440390934303B7
:1074C000809342033093410320934003882009F4C2
:1074D00041C0809132089091330897FF03C0909586
:1074E00081959F4F6CE070E00E94628B9B017093CE
:1074F0003F0360933E03809142089091430897FFB9
:1075000003C0909581959F4F6CE070E00E94628B64
:1075100070933D0360933C038091E4059091E505F1
:107520009093390380933803B90184E090E00E947E
:107530000A2E60913C0370913D0386E090E00E942A
:107540000A2E609138037091390388E090E00E9420
:107550000A2E65C084E090E00E94052E90933F03C0
:1075600080933E0386E090E00E94052E90933D03B9
:1075700080933C0388E090E00E94052E9C0190934C
:1075800039038093380380913E0390913F038150EB
:10759000984050F480913C0390913D038150984075
:1075A00018F421503440D8F18DE199E09F938F93E6
:1075B0008FEB94E19F938F93E091FC03F091FD0397
:1075C0000995809132089091330897FF03C09095F8
:1075D00081959F4F6CE070E00E94628B70933F0337
:1075E00060933E03809142089091430897FF03C047
:1075F000909581959F4F6CE070E00E94628B709334
:107600003D0360933C038091E4059091E5059093E0
:107610003903809338030F900F900F900F901092C2
:10762000F7071092F6071092E7071092E6071092FC
:1076300038081092370884E690E00E94F018809194
:10764000F4019091F5019C01220F331F220F331F8B
:10765000280F391F280F391F309333082093320821
:107660008091F6019091F7018C01000F111F000F1E
:10767000111F080F191F080F191F109343080093BB
:10768000420880915E06C82EDD24EE24FF244427A4
:1076900037FD4095542FC701B6010E94238B4B0143
:1076A0005C016093330370933403809335039093AC
:1076B00036039801442737FD4095542FC701B60182
:1076C0000E94238BDC01CB0180932B0390932C032E
:1076D000A0932D03B0932E03809213039092140372
:1076E000A0921503B092160380930B0390930C03A2
:1076F000A0930D03B0930E031092030310920403A2
:1077000010920503109206038091150190911601C5
:10771000A0911701B09118019093E7058093E605B9
:107720001092EC011092EB011092F3021092F4020D
:107730001092F5021092F60200918E0110918F01C5
:107740001093F2020093F10284E690E090938B0193
:1077500080938A0182E390E09093DB018093DA01C9
:10776000809183069927AA27BB27BC01CD0124EC71
:1077700039E040E050E00E94238BDC01CB018856C9
:10778000954CAF4FBF4F8093860190938701A09394
:107790008801B0938901809184069927AA27BB2785
:1077A000BC01CD010E94238BDC01CB018856954C96
:1077B000AF4FBF4F8093820190938301A0938401C8
:1077C000B09385011092470110924601C801AA2783
:1077D00097FDA095BA2F209142013091430140912D
:1077E000440150914501BC01CD010E94238BDC0175
:1077F000CB0180933E0890933F08A0934008B0933C
:1078000041081092EE021092ED020E94CA6B809124
:10781000A10284608093A1028FEF8093BE08109232
:10782000BF0880E28093C008CAEDD2E0A7E4B6E0CA
:1078300007E08D91E82FFF27EE0FFF1FEB58F84F61
:107840008081918181588993015007FFF2CF84E6AE
:107850008093D9028091D801882311F0469A579AD3
:10786000809148039091490380569940815C9B42E6
:1078700028F080911504816080931504809146035F
:107880009091470380569940815C9B4228F08091FB
:107890001504826080931504809144039091450300
:1078A0008C5291408957954028F08091150484604E
:1078B0008093150480913E0390913F038C52914038
:1078C000835C914028F080911504886080931504B2
:1078D00080913C0390913D038C529140835C914098
:1078E00028F08091150480618093150480913803FD
:1078F00090913903805092408355914028F08091B7
:10790000150480628093150486E480937D010E94B3
:107910008685ECE0CDB7DEB70C94D48BA3E1B0E064
:10792000E4E9FCE30C94B28B80914403909145030D
:107930002091F8013091F901821B930B9093380844
:1079400080933708809102029091030297FD079679
:107950009C0113E0359527951A95E1F73093F707C9
:107960002093F607809100029091010297FD0796FF
:10797000B3E095958795BA95E1F79093E7078093E3
:10798000E60730930208209301089093FA0780934A
:10799000F9078091320890913308AC01440F551FCC
:1079A000480F591F2091F4013091F501C901880F4A
:1079B000991F880F991F820F931F820F931F480FE3
:1079C000591F57FF02C04D5F5F4F5595479555951D
:1079D0004795509333084093320880914208909124
:1079E0004308AC01440F551F480F591F2091F60161
:1079F0003091F701C901880F991F880F991F820FD5
:107A0000931F820F931F480F591F57FF02C04D5FEE
:107A10005F4F55954795559547955093430840932B
:107A200042082091F4013091F501C901880F991F96
:107A3000880F991F820F931F820F931F9C01442769
:107A400037FD4095542F8091230390912403A091FA
:107A50002503B0912603820F931FA41FB51F8093A7
:107A6000230390932403A0932503B093260320912E
:107A7000F6013091F701C901880F991F880F991FEE
:107A8000820F931F820F931F9C01442737FD40955F
:107A9000542F80911F0390912003A0912103B09156
:107AA0002203820F931FA41FB51F80931F0390937F
:107AB0002003A0932103B093220380910B0890919F
:107AC0000C082091F4013091F501820F931F9093DF
:107AD0000C0880930B0880913A0890913B08209104
:107AE000F6013091F701820F931F90933B0880932A
:107AF0003A0880913A0390913B03019690933B039F
:107B000080933A038091E4059091E5052091380334
:107B100030913903821B930B9C01442737FD40951C
:107B2000542F80911B0390911C03A0911D03B091D1
:107B30001E03820F931FA41FB51F80931B039093F6
:107B40001C03A0931D03B0931E038FEC80937A0057
:107B500010920F0120910B0330910C0340910D0303
:107B600050910E0329873A874B875C8729543B46FF
:107B7000414050402CF028E43BE641E050E00DC08D
:107B800089859A85AB85BC85885B9449AE4FBF4F8C
:107B90004CF428EB34E94EEF5FEF2D833E834F83A7
:107BA000588708C089859A85AB85BC858D839E835F
:107BB000AF83B887209113033091140340911503CC
:107BC000509116032D873E874F87588B29543B468B
:107BD000414050402CF028E43BE641E050E00DC02D
:107BE0008D859E85AF85B889885B9449AE4FBF4F20
:107BF0004CF428EB34E94EEF5FEF29833A834B8353
:107C00005C8308C08D859E85AF85B88989839A83FA
:107C1000AB83BC83A0913708B0913808BB8BAA8B8B
:107C2000FD01CF01AA2797FDA095BA2FA0900303CD
:107C3000B0900403C0900503D0900603A80EB91EAF
:107C4000CA1EDB1EA0920303B0920403C092050378
:107C5000D0920603E0903E08F0903F080091400863
:107C600010914108E80EF91E0A1F1B1FE0923E0802
:107C7000F0923F080093400810934108F091BC0235
:107C8000F98BFF2309F098C18091BB02882309F08A
:107C900093C180912E0886FF8FC18091E607909155
:107CA000E707AA2797FDA095BA2FBC01CD0129812E
:107CB0003A814B815C810E94238B9B01AC0197FF31
:107CC00004C02150384F4F4F5F4FBBE0559547954B
:107CD00037952795BA95D1F780916901682E772459
:107CE00088249924CA01B901A40193010E94238B1D
:107CF000DC01CB018093540390935503A09356036A
:107D0000B0935703B7FF04C08150904FAF4FBF4FA0
:107D10001C012D01ACE05594479437942794AA9503
:107D2000D1F720925403309255034092560350925B
:107D300057038091F6079091F707AA2797FDA09522
:107D4000BA2FBC01CD012D813E814F8158850E9403
:107D5000238B97FF04C06150784F8F4F9F4FFBE0FC
:107D60009595879577956795FA95D1F7A401930135
:107D70000E94238BDC01CB0180935803909359031D
:107D8000A0935A03B0935B03B7FF04C08150904F98
:107D9000AF4FBF4F9C01AD01ECE05595479537952E
:107DA0002795EA95D1F720935803309359034093D0
:107DB0005A0350935B038091540390915503909321
:107DC000DE078093DD0780915803909159039093CB
:107DD000E2078093E10722193309440955092093EA
:107DE00058033093590340935A0350935B03E20EB8
:107DF000F31E041F151FE0923E08F0923F08009307
:107E0000400810934108809168018823B1F457FF1E
:107E100004C02F5F3F4F4F4F5F4F559547953795A4
:107E20002795A21AB30AC40AD50AA0920303B092F6
:107E30000403C0920503D09206032A893B89790185
:107E40000027F7FC0095102F80915803909159035B
:107E5000A0915A03B0915B03E80EF91E0A1F1B1F85
:107E6000C801B70129813A814B815C810E94238B33
:107E70009B01AC0197FF04C02150384F4F4F5F4F1B
:107E80006BE055954795379527956A95D1F7809181
:107E90006A01A82EBB24CC24DD24CA01B901A601A5
:107EA00095010E94238BDC01CB0180934C039093BE
:107EB0004D03A0934E03B0934F03B7FF04C081500E
:107EC000904FAF4FBF4F3C014D013CE095948794DC
:107ED000779467943A95D1F760924C0370924D0372
:107EE00080924E0390924F03C801B7012D813E81CD
:107EF0004F8158850E94238B97FF04C06150784FB3
:107F00008F4F9F4F2BE095958795779567952A958D
:107F1000D1F7A60195010E94238BDC01CB01809350
:107F2000500390935103A0935203B0935303B7FFB0
:107F300004C08150904FAF4FBF4FAC01BD018CE0EA
:107F400075956795579547958A95D1F74093500356
:107F50005093510360935203709353032A893B89D2
:107F600037FF03C0309521953F4F21343105E4F1AF
:107F7000D401C30197FE07C0B095A0959095819557
:107F80009F4FAF4FBF4F81389105A105B10584F4D4
:107F9000DB01CA0177FF07C0B095A0959095819548
:107FA0009F4FAF4FBF4F81389105A105B105E4F058
:107FB00081E08093EF0218C01092E2071092E1076F
:107FC0001092DE071092DD071092500310925103B9
:107FD000109252031092530310924C0310924D03CF
:107FE00010924E0310924F038091500390915103D1
:107FF000A0915203B0915303BC01CD0124E630E0BF
:1080000040E050E00E94978BE0904C03F0904D03CD
:10801000E21AF30AF092F507E092F40780914C031C
:1080200090914D03A0914E03B0914F03BC01CD013F
:1080300024E630E040E050E00E94978BDA01C9016D
:1080400020915003309151038C01021B130B1093AC
:10805000E9070093E8078091420190914301A091C4
:108060004401B0914501BC01CD0128E631E040E07A
:1080700050E00E94238B20913E0830913F084091B0
:10808000400850914108261737074807590764F000
:10809000261B370B480B590B20933E0830933F08A3
:1080A000409340085093410820913E0830913F088A
:1080B000409140085091410857FF0CC0260F371FD0
:1080C000481F591F20933E0830933F0840934008B3
:1080D000509341086091E6077091E7076E0D7F1D90
:1080E0009B01442737FD4095542F809107039091C1
:1080F0000803A0910903B0910A03820F931FA41FE4
:10810000B51F8093070390930803A0930903B093CE
:108110000A038091C1029091C202681B790BCB01C6
:10812000AA2797FDA095BA2F29853A854B855C85AE
:10813000820F931FA41FB51F80930B0390930C0312
:10814000A0930D03B0930E03C0908201D0908301E1
:10815000E0908401F0908501C816D906EA06FB0676
:10816000C4F488EA91E6A0E0B0E08C199D09AE095C
:10817000BF0980930B0390930C03A0930D03B0935E
:108180000E038093070390930803A0930903B09311
:108190000A0322273327A9012C193D094E095F093B
:1081A00080910B0390910C03A0910D03B0910E03ED
:1081B00082179307A407B507B4F4D701C601885AFC
:1081C0009146A040B04080930B0390930C03A09382
:1081D0000D03B0930E038093070390930803A093BD
:1081E0000903B0930A036091F6077091F707600FD7
:1081F000711F9B01442737FD4095542F80910F0339
:1082000090911003A0911103B0911203820F931F5C
:10821000A41FB51F80930F0390931003A093110325
:10822000B09312038091BF029091C002681B790B3A
:10823000CB01AA2797FDA095BA2F2D853E854F85A6
:108240005889820F931FA41FB51F80931303909327
:108250001403A0931503B0931603E0908601F090E9
:1082600087010091880110918901E816F9060A0733
:108270001B07C4F488EA91E6A0E0B0E08E199F09DC
:10828000A00BB10B8093130390931403A0931503D9
:10829000B093160380930F0390931003A0931103E0
:1082A000B093120322273327A9012E193F09400B4F
:1082B000510B8091130390911403A0911503B09179
:1082C000160382179307A407B507B4F4D801C701B2
:1082D000885A9146A040B0408093130390931403B2
:1082E000A0931503B093160380930F03909310038C
:1082F000A0931103B09312038091030390910403A0
:10830000A0910503B091060380931703909318037F
:10831000A0931903B0931A0380911303909114034F
:10832000A0911503B0911603809333039093340307
:10833000A0933503B093360380910B0390910C0307
:10834000A0910D03B0910E0380932B0390932C0307
:10835000A0932D03B0932E0380910F0390911003EF
:10836000A0911103B091120380932F0390933003D7
:10837000A0933103B09332038091070390910803D7
:10838000A0910903B0910A038093270390932803D7
:10839000A0932903B0932A0380911B0190911C01A3
:1083A00097FD079603E0959587950A95E1F79093D9
:1083B000F7078093F6078091190190911A0197FDB4
:1083C000079613E0959587951A95E1F79093E7073F
:1083D0008093E6078091FC019091FD010F9734F4A2
:1083E00088E19CEF9093F7078093F6078091FC015A
:1083F0009091FD01079734F480E398EF9093F7078D
:108400008093F607209101012A30A9F48091FC01A4
:108410009091FD01835F934034F088EE93E0909358
:10842000F7078093F6078091FC019091FD018A5F28
:108430009340DCF014C08091FC019091FD01815DBE
:10844000974034F088EE93E09093F7078093F60717
:108450008091FC019091FD01805E974034F080EDA9
:1084600097E09093F7078093F6078091FA01909137
:10847000FB010F9734F488E19CEF9093E70780931A
:10848000E6078091FA019091FB01079734F480E3AD
:1084900098EF9093E7078093E6072A30A9F480913C
:1084A000FA019091FB01835F934034F088EE93E0F2
:1084B0009093E7078093E6078091FA019091FB0182
:1084C0008A5F9340DCF014C08091FA019091FB0127
:1084D000815D974034F088EE93E09093E7078093B6
:1084E000E6078091FA019091FB01805E974034F09D
:1084F00080ED97E09093E7078093E6076091740121
:10850000662309F4AFC040911B0150911C0180917A
:108510005C0390915D03481B590B50936303409398
:10852000620320911B0130911C01280F391F37FF76
:1085300002C02F5F3F4F3595279530935D03209301
:108540005C03413851051CF080E890E005C04058BC
:108550005F4F34F480E89FEF90936303809362034E
:108560004091190150911A0180915E0390915F032F
:10857000481B590B509361034093600320911901EC
:1085800030911A01280F391F37FF02C02F5F3F4F6C
:108590003595279530935F0320935E03413851054D
:1085A0001CF080E890E005C040585F4F34F480E84C
:1085B0009FEF9093610380936003462F552780912E
:1085C000620390916303849FB001859F700D949F17
:1085D000700D11249B0177FF02C0215F3F4FF4E033
:1085E00035952795FA95E1F78091F6079091F70771
:1085F000820F931F9093F7078093F6078091600393
:1086000090916103849FD001859FB00D949FB00D20
:108610001124AD019D01B7FF02C0215F3F4FE4E08F
:1086200035952795EA95E1F78091E6079091E70760
:10863000820F931F9093E7078093E60780911B01B9
:1086400090911C01860F971F90931C0180931B0132
:108650008091190190911A01840F951F90931A012E
:10866000809319010091F9071091FA078091DD07B5
:108670009091DE07101611065CF59C0197FF04C06F
:1086800022273327281B390BC901AA2797FDA0955C
:10869000BA2F20916801332744275527BC01CD010B
:1086A0000E94238B9B01AC0197FF04C0215C3F4FCC
:1086B0004F4F5F4F76E055954795379527957A95BB
:1086C000D1F78091F4079091F507820F931F27C08F
:1086D00097FF03C0909581959F4FAA2797FDA0957E
:1086E000BA2F20916801332744275527BC01CD01BB
:1086F0000E94238B9B01AC0197FF04C0215C3F4F7C
:108700004F4F5F4F66E055954795379527956A958A
:10871000D1F78091F4079091F507821B930B90930A
:10872000F5078093F407E0900108F090020880912B
:10873000E1079091E2071E141F045CF59C0197FF6E
:1087400004C022273327281B390BC901AA2797FD0C
:10875000A095BA2F20916801332744275527BC01E3
:10876000CD010E94238B9B01AC0197FF04C0215CCB
:108770003F4F4F4F5F4F96E055954795379527955B
:108780009A95D1F78091E8079091E907820F931F9E
:1087900027C097FF03C0909581959F4FAA2797FD0B
:1087A000A095BA2F20916801332744275527BC0193
:1087B000CD010E94238B9B01AC0197FF04C0215C7B
:1087C0003F4F4F4F5F4F86E055954795379527951B
:1087D0008A95D1F78091E8079091E907821B930B66
:1087E0009093E9078093E80780912E0887FF44C0A3
:1087F000B989BB2309F040C08091BB028823E1F511
:10880000E1E0EE16E1E0FE064CF08091F607909173
:10881000F7078E0D9F1D805091400DC0F0E0EF16C0
:10882000FFEFFF0664F48091F6079091F7078E0D35
:108830009F1D80509F4F9093F7078093F60721E08C
:10884000013012074CF08091E6079091E707800F06
:10885000911F805091400CC03FEF0030130764F42B
:108860008091E6079091E707800F911F80509F4FFE
:108870009093E7078093E607E2E1CD5E0C94CE8B00
:108880008091D802882301F58091A1028C7F80938A
:10889000A102AAE1B4E0E4E1F7E09BE08091B90134
:1088A000882309F48C938D9181831282915038969C
:1088B00097FFF4CF8091B901882359F08091B901D5
:1088C00081508093B90105C08091A102816080939D
:1088D000A10280912302882319F0109223020895A7
:1088E0008093250280932702809121028E7F8093BE
:1088F000210285EA8093BC000895CF93DF93AAED0F
:10890000B2E0C7E4D6E057E09991E92FFF27EE0FD8
:10891000FF1FEB58F84F0190F081E02DE158FF4F19
:10892000EF3FF10521F01CF0EFEFF0E004C0F7FF9E
:1089300002C0E0E0F0E0993111F4EC931BC04C91DF
:10894000242F3327E217F307A9F0CF01821B930BE3
:1089500097FD03969595879595958795242F280FD4
:108960002C93822F9927E817F90714F4215001C09E
:108970002F5F2C935150119657FFC6CF809151060F
:10898000883F38F0EFEFF0E0E81BF109E652FD4FC9
:10899000808180937A0180917A01882329F084363E
:1089A00018F084E680937A0180915306883F38F06E
:1089B000EFEFF0E0E81BF109E652FD4F8081809374
:1089C000780180917801882329F0843618F084E6B4
:1089D0008093780180916006883F38F0EFEFF0E0F7
:1089E000E81BF109E652FD4F80818093730180916D
:1089F00073018B3010F48AE002C08F3F11F4809332
:108A0000730180918D06883F38F0EFEFF0E0E81BAE
:108A1000F109E652FD4F808180930D0880910D0889
:108A2000863010F485E002C08F3F11F480930D086A
:108A300080918F06883F38F0EFEFF0E0E81BF109F6
:108A4000E652FD4F8081809335088091350886304D
:108A500010F485E002C08F3F11F4809335088091B7
:108A60007A06873F19F4429905C006C0863F31F463
:108A7000439B02C08CE80BC086E409C0883F38F0F5
:108A8000EFEFF0E0E81BF109E652FD4F80818093A3
:108A90000A0880917B06873F19F4429905C006C0F9
:108AA000863F31F4439B02C08CE80BC086E409C0CA
:108AB000883F38F0EFEFF0E0E81BF109E652FD4F98
:108AC00080818093E30780917C06883F38F0EFEF48
:108AD000F0E0E81BF109E652FD4F80818093130816
:108AE00080915206883F38F0EFEFF0E0E81BF10983
:108AF000E652FD4F80818093790180915506883F31
:108B000038F0EFEFF0E0E81BF109E652FD4F80810D
:108B10008093770180915706883F38F0EFEFF0E0BF
:108B2000E81BF109E652FD4F808180937501809129
:108B30005F06883F38F0EFEFF0E0E81BF109E652FE
:108B4000FD4F80818093760180916106883F38F0E7
:108B5000EFEFF0E0E81BF109E652FD4F80818093D2
:108B6000720180916206883F38F0EFEFF0E0E81B79
:108B7000F109E652FD4F8081809374018091630674
:108B8000883F38F0EFEFF0E0E81BF109E652FD4FC7
:108B900080818093710180916406883F38F0EFEF07
:108BA000F0E0E81BF109E652FD4F808180937001EF
:108BB00080916A06883F38F0EFEFF0E0E81BF1099A
:108BC000E652FD4F808180936E0180916B06883F55
:108BD00038F0EFEFF0E0E81BF109E652FD4F80813D
:108BE0008093B60280916C06883F38F0EFEFF0E09A
:108BF000E81BF109E652FD4F80818093B502809118
:108C00006D06883F38F0EFEFF0E0E81BF109E6521F
:108C1000FD4F80818093B40280916E06883F38F0CA
:108C2000EFEFF0E0E81BF109E652FD4F8081809301
:108C3000B30280918806883F38F0EFEFF0E0E81B40
:108C4000F109E652FD4F80818093B202809189063E
:108C5000883F38F0EFEFF0E0E81BF109E652FD4FF6
:108C600080818093B10280918A06883F38F0EFEFCF
:108C7000F0E0E81BF109E652FD4F80818093B002DD
:108C800080918B06883F38F0EFEFF0E0E81BF109A8
:108C9000E652FD4F80818093AF0280916F06883F3E
:108CA00038F0EFEFF0E0E81BF109E652FD4F80816C
:108CB00080936D0180917306883F38F0EFEFF0E00C
:108CC000E81BF109E652FD4F808180936C01809191
:108CD0007D06883F38F0EFEFF0E0E81BF109E6523F
:108CE000FD4F808180936B0180918006883F38F032
:108CF000EFEFF0E0E81BF109E652FD4F8081809331
:108D00006A0180918106883F38F0EFEFF0E0E81BC0
:108D1000F109E652FD4F80818093690180918206BE
:108D2000883F38F0EFEFF0E0E81BF109E652FD4F25
:108D30008081809368018091A906883F38F0EFEF29
:108D4000F0E0E81BF109E652FD4F80818093F207C5
:108D50009091AE03992321F08091F207981720F0AB
:108D60008091F207882311F49093F20780914F06C7
:108D700080932E088091AF06809312088091870619
:108D8000883F38F0EFEFF0E0E81BF109E652FD4FC5
:108D90008081809367018091A206883F38F0EFEFD1
:108DA000F0E0E81BF109E652FD4F80818093450811
:108DB00080916E01282F33272F5F3F4F8CE398E27D
:108DC000B9010E94628B70937C0160937B0180915A
:108DD0005D068093360880915C068093FB07909136
:108DE000A4069333E0F181E08093AE02983F58F0FF
:108DF000EFEFF0E0E91BF109E652FD4F808182338D
:108E000010F41092AE0280917D012091AE02821783
:108E1000B1F0833088F4222319F08CED95E002C084
:108E200088EC90E09093DB018093DA0185E08093F9
:108E3000C30220937D0103C0815080937D01809106
:108E400085089091860897FF0FC08091AE02882315
:108E500059F08091150480688093150405C0109224
:108E6000AE028AE080937D0180918508909186080A
:108E700097FF1DC08091D8028823C9F08091AE026F
:108E80008823A9F080910701909108018F5F9F4F7F
:108E900071F488E99AE39093DB018093DA0180E032
:108EA00094EA90930801809307011092AE0280919A
:108EB000AE02882369F08091A00281608093A002B5
:108EC00080916A01823D48F4825E80936A0105C008
:108ED0008091A0028E7F8093A002DF91CF910895B0
:108EE000A7E1B0E0E6E7F7E40C94B28B0E948E3C79
:108EF0008091B00682FF27C08091BD029091BE0292
:108F00000097F1F002E088359007D4F49C0197FFB8
:108F100002C02D5F3F4F3595279535952795809158
:108F200067069927289FA001299F500D389F500D53
:108F30001124CA0164E670E00E94628BCB0106C076
:108F40008DE290E003C080916706992790939F027D
:108F500080939E026091E3027091E4027A836983B8
:108F60008091FB0799270A966817790714F49A836A
:108F700089838091D902843608F06AC08091A0026A
:108F800082FD66C08091780390917903009731F05B
:108F9000019790937903809378030BC01092D802C5
:108FA0009093A3028093A2028091A1028D7E809370
:108FB000A102809101018A3011F0843110F0289AC9
:108FC00001C028988091A2029091A302895E9340EB
:108FD000E0F18091D4088536C0F180919E02909195
:108FE0009F029A8389838091A10280618093A1026C
:108FF00080914306A82FBB27AA0FBB1FFD01E75591
:10900000F84F1182108280914406282F3327220FB7
:10901000331FC9018755984FFC0111821082AB584C
:10902000B84F11961C921E922B58384FD9011196A9
:109030001C921E9280914606E82FFF27EE0FFF1F1D
:10904000EB58F84F11821082ABC21092D802A8C21E
:109050008091D9028D3808F4A3C28091A1028F7E3D
:109060008093A1029091680682E3989FC001112429
:109070009093790380937803E981FA81B9978CF012
:109080008091D802882369F08091A2029091A30276
:10909000FFEF8F3F9F0729F001969093A3028093E3
:1090A000A2028091A2029091A3028F3F910509F044
:1090B00008F51092FB021092FC021092FD02109231
:1090C000FE021092F7021092F8021092F90210922A
:1090D000FA021092640310926503109266031092D4
:1090E0006703109203031092040310920503109279
:1090F000060305C08091A10282608093A102809145
:109100004506E82FFF27EE0FFF1FEB58F84F808131
:109110009181813591050CF437C12091D802222329
:1091200009F032C180914606E82FFF27EE0FFF1F9E
:10913000EB58F84F808191818C3491050CF401C17A
:1091400080917A038F5F80937A03893C08F41CC175
:1091500020937A031092A3021092A2023091430648
:10916000E32FFF27EE0FFF1FEB58F84F808191810F
:1091700087349105B4F480914406E82FFF27EE0F61
:10918000FF1FEB58F84F808191810190F081E02D15
:10919000F7FF03C0F095E195FF4FE734F1050CF4BC
:1091A00078C041E020914406A22FBB27AA0FBB1F25
:1091B000AB58B84F8D919C9111978734910544F02D
:1091C000E32FFF27EE0FFF1FEB58F84F80819181AF
:1091D0008D919C918734910574F080914306E82F1E
:1091E000FF27EE0FFF1FEB58F84F808191818734E6
:1091F00091050CF042E0E22FFF27EE0FFF1FEB5826
:10920000F84F808191818634910574F480914306F2
:10921000E82FFF27EE0FFF1FEB58F84F8081918159
:10922000873491050CF043E0E22FFF27EE0FFF1F7C
:10923000EB58F84F808191818A5B9F4F74F4809145
:109240004306E82FFF27EE0FFF1FEB58F84F8081F2
:109250009181873491050CF044E0E22FFF27EE0F57
:10926000FF1FEB58F84F808191818A5B9F4F74F408
:1092700080914306E82FFF27EE0FFF1FEB58F84FB2
:1092800080819181863491050CF445E0842F0E9401
:10929000642E80914406E82FFF27EE0FFF1FEB5846
:1092A000F84F808191810190F081E02DF7FF03C09C
:1092B000F095E195FF4F7E97CCF480914306E82F1F
:1092C000FF27EE0FFF1FEB58F84F808191818A5BDB
:1092D0009F4F64F481E0809330041092C40288EEC2
:1092E00093E09093DB018093DA014EC00E946D2FD2
:1092F0000E940F2E80E00E941309809169060E944F
:10930000288780912E0880FF10C0809113019091D2
:109310001401875B934038F48091130190911401FC
:109320008E5E924010F40E94EB1C1092D80180E0F7
:109330000E94DD3981E08093C4028093D801579A5E
:109340001AC080819181855B9F4FE4F480917A03FC
:109350008F5F80937A03893CB8F02093D8022093E2
:109360007A031092A3021092A20281E00E94DD39DA
:1093700081E08093C4020E946D2F68E770E00E9434
:109380000E3902C020937A0380914506E82FFF270B
:10939000EE0FFF1FEB58F84F808191818B5A9F4F42
:1093A0000CF0FEC03091D802E0914606332309F05C
:1093B000CCC0FF27EE0FFF1FEB58F84F8081918143
:1093C000855B9F4F0CF0BEC02091A506E22FFF27C2
:1093D000EE0FFF1FEB58F84F80819181855B9F4F07
:1093E0001CF0222309F0AEC080917B038F5F809335
:1093F0007B03893C08F4D4C030937B03809115042F
:10940000882309F098C08091C402882309F493C08E
:109410008091B303882309F08EC081E090E090939F
:10942000A3028093A20281E08093D8021092640389
:109430001092650310926603109267031092030363
:109440001092040310920503109206031092FF027B
:1094500010920003109201031092020380915E06A5
:10946000E82EFF24002711278091320890913308BD
:109470009C01442737FD4095542FC801B7010E9435
:10948000238BDC01CB018093130390931403A093EF
:109490001503B093160380914208909143089C01F4
:1094A000442737FD4095542FC801B7010E94238BF4
:1094B000DC01CB0180930B0390930C03A0930D036D
:1094C000B0930E038091330390913403A091350340
:1094D000B091360380930F0390931003A093110370
:1094E000B093120380912B0390912C03A0912D0334
:1094F000B0912E038093070390930803A093090370
:10950000B0930A031092FB021092FC021092FD022B
:109510001092FE021092F7021092F8021092F902D5
:109520001092FA028091A10288608093A10284E6E1
:109530008093C30235C08CED95E09093DB0180935E
:10954000DA012EC010927B032BC0FF27EE0FFF1F06
:10955000EB58F84F808191818C349105FCF020917B
:10956000A506E22FFF27EE0FFF1FEB58F84F808173
:109570009181855B9F4F14F0222381F480917C03BD
:109580008F5F80937C03893C58F01092D802109230
:109590007C031092A3021092A20202C010927C03DC
:1095A00080914001815080934001809140018F3F24
:1095B00021F08091A10284FFA9C30E947D44B09054
:1095C000590680918503909186039C01220F331FD9
:1095D000280F391FC0904306AC2DBB27AA0FBB1F15
:1095E000FD01EB58F84F4B2D552780819181849FC9
:1095F000F001859FF00D949FF00D11242E0F3F1F59
:1096000037FF02C02D5F3F4FB9017595679575957E
:109610006795A755B84F80915A06082F11278D914D
:109620009C91809F7001819FF00C909FF00C112401
:109630006E0D7F1D70938603609385038091870371
:10964000909188039C01220F331F280F391FD0905F
:109650004406AD2DBB27AA0FBB1FFD01EB58F84FE9
:1096600080819181849FF001859FF00D949FF00D82
:1096700011242E0F3F1F37FF02C02D5F3F4FA9015E
:109680005595479555954795A755B84F8D919C9100
:10969000809F7001819FF00C909FF00C11244E0D63
:1096A0005F1D50938803409387038091AE02882307
:1096B00009F448C0CB0177FD0396DC01B595A79569
:1096C000B595A795CA0157FD0396FC01F595E79559
:1096D000F595E79580919C01682F772767FD709538
:1096E0006A9F90016B9F300D7A9F300D11248091FD
:1096F000B503482F552747FD50954E9FC0014F9FFA
:10970000900D5E9F900D1124280F391F37FF02C066
:10971000295F3F4F93E0359527959A95E1F7309370
:10972000EA022093E9026E9F90016F9F300D7E9FA9
:10973000300D11244A9FC0014B9F900D5A9F900DF0
:1097400011243FC08091A306E82FFF27E85BFE4F5E
:10975000868180939C0190819093B503A82FBB27AD
:10976000A7FDB095A69F9001A79F300DB69F300D25
:109770001124E92FFF27E7FDF095E49FC001E59F45
:10978000900DF49F900D1124280F391F37FF02C050
:10979000295F3F4F83E0359527958A95E1F7309310
:1097A000EA022093E902A49F9001A59F300DB49F87
:1097B000300D1124E69FC001E79F900DF69F900D9C
:1097C0001124281B390B37FF02C0295F3F4F03E0EC
:1097D000359527950A95E1F73093E8022093E70243
:1097E00080914606E82FFF27EE0FFF1FEB58F84F3A
:1097F00080819181909581959F4F9093E60280930F
:10980000E5028530910514F0049705C00FEF8C3FF9
:10981000900734F404969093E6028093E50204C026
:109820001092E6021092E5028091A103882309F4C8
:109830003EC0282F33278091E9029091EA0297FDDC
:10984000079613E0959587951A95E1F7289FA00153
:10985000299F500D389F500D1124CA0157FD0F96B6
:10986000B4E095958795BA95E1F79093EA028093D5
:10987000E9028091E7029091E80297FD0796A3E044
:1098800095958795AA95E1F7289FB001299F700DBE
:10989000389F700D1124CB0177FD0F96F4E095955C
:1098A0008795FA95E1F79093E8028093E70280901C
:1098B000E9029090EA028091A4039091A503881A8E
:1098C000990A9092EA028092E9020091E7021091CF
:1098D000E8028091A2039091A303081B190B109337
:1098E000E8020093E70280914506E82FFF27EE0F7C
:1098F000FF1FEB58F84FE080F1808FE790E0E80E13
:10990000F91EF092E402E092E3028091730199273C
:10991000AA2797FDA095BA2FBC01CD010E94978A76
:10992000DC01CB0120E030E040E251E4BC01CD019C
:109930000E94058ADC01CB01BC01CD010E94698A2D
:10994000DC01CB0180933C08809172018093140864
:10995000809171019927AA2797FDA095BA2FBC0184
:10996000CD010E94978ADC01CB0120E030E040E28B
:1099700051E4BC01CD010E94058ADC01CB01BC0190
:10998000CD010E94698ADC01CB018093ED078091B3
:1099900070018093030880913C0480FF59C080913E
:1099A0004508813808F454C080913504992787FD13
:1099B00090952B2D3327829FD001839FB00D929FCE
:1099C000B00D11248A0E9B1E9092EA028092E90249
:1099D00080913604992787FD9095829FF001839F9F
:1099E000F00D929FF00D11240E0F1F1F1093E8022F
:1099F0000093E70280913704282F332727FD309505
:109A00008091E5029091E602820F931F9093E60207
:109A10008093E50280913904282F332727FD309564
:109A2000809154069927289F8001299F100D389F07
:109A3000100D1124109347010093460180913804C2
:109A400099278E159F0524F49093E4028093E302F6
:109A50008091E3029091E40297FF04C01092E40227
:109A60001092E30280912E0882FF02C01092140827
:109A70004091E9025091EA02CA0157FD03969C0108
:109A8000359527953595279537FF03C03095219556
:109A90003F4F8091A6029091A70282179307B4F4DA
:109AA000CA0157FF03C0909581959F4F97FD03967C
:109AB00095958795959587959093A7028093A60293
:109AC0008536910544F084E690E001C001979093BB
:109AD000A7028093A6024091E7025091E802CA01D2
:109AE00057FD03969C01359527953595279537FFAA
:109AF00003C0309521953F4F8091A4029091A5021B
:109B000082179307B4F4CA0157FF03C0909581955B
:109B10009F4F97FD0396959587959595879590937B
:109B2000A5028093A4028536910544F084E690E076
:109B300001C001979093A5028093A4028091A10295
:109B400084FF08C01092A7021092A6021092A502EC
:109B50001092A402ED2DFF27EE0FFF1FEB58F84FD8
:109B600040917E06242F3327808191812817390761
:109B700044F48091AD0682FF04C081E08093BA0274
:109B800013C0ED2DFF27EE0FFF1FEB58F84F842F6A
:109B9000992720917F06821B910920813181281706
:109BA000390714F41092BA0240914406E42FFF27BB
:109BB000EE0FFF1FEB58F84F50917E06852F992727
:109BC00022273327281B390B808191818217930725
:109BD00044F48091AD0683FF04C081E08093B90214
:109BE00016C08091B902882391F0E42FFF27EE0F71
:109BF000FF1FEB58F84F80917F069927851B91092D
:109C0000208131818217930714F41092B902EC2D50
:109C1000FF27EE0FFF1FEB58F84F40917E06242FD1
:109C20003327808191812817390744F48091AD064C
:109C300080FF04C081E08093B70217C08091B70213
:109C4000882399F0EC2DFF27EE0FFF1FEB58F84FFC
:109C5000842F992720917F06821B910920813181D1
:109C60002817390714F41092B70240914306E42FE5
:109C7000FF27EE0FFF1FEB58F84F50917E06852F00
:109C8000992722273327281B390B8081918182173E
:109C9000930744F48091AD0681FF04C081E0809376
:109CA000B80216C08091B802882391F0E42FFF27F4
:109CB000EE0FFF1FEB58F84F80917F069927851B09
:109CC0009109208131818217930714F41092B80210
:109CD0008091BA02882319F48091B902811181E040
:109CE0008093BB028091B702882321F48091B8024F
:109CF000882351F081E08093BC021092BB02109245
:109D0000BA021092B90202C08093BC028091BB02D9
:109D1000882321F48091BC02882369F080917D061C
:109D2000992729813A818217930714F49A838983AA
:109D300081E08093EF028091A00299279C0124701A
:109D4000307082FF2DC08091A4039091A50390955F
:109D500081959F4F9093EA028093E9028091A2033C
:109D60009091A303909581959F4F9093E8028093E3
:109D7000E70280918001909181019093E4028093A9
:109D8000E30280912E088B778B6680932E0880915A
:109D900012088C7B8093120888EC809379011EC096
:109DA0008091A10284FF1AC03093E6022093E5025D
:109DB0003093EA022093E9023093E8022093E7020D
:109DC0009AE590933C0888E7809314089093ED07F8
:109DD000809303081092BB021092BC028091060887
:109DE00090910708A0910808B091090820913303C9
:109DF000309134034091350350913603820F931F05
:109E0000A41FB51F8093060890930708A093080825
:109E1000B093090880910E0890910F08A091100846
:109E2000B0911108E0902B03F0902C0300912D03CA
:109E300010912E03EB82FC820D831E838E0D9F1DDD
:109E4000A01FB11F80930E0890930F08A0931008D5
:109E5000B09311088091FD079091FE07A091FF0734
:109E6000B0910008E0902F03F0903003009131038F
:109E700010913203EF82F88609871A878E0D9F1D95
:109E8000A01FB11F8093FD079093FE07A093FF07CB
:109E9000B09300088091EE079091EF07A091F00732
:109EA000B091F107E0902703F09028030091290377
:109EB00010912A03EB86FC860D871E878E0D9F1D51
:109EC000A01FB11F8093EE079093EF07A093F007B8
:109ED000B093F107F090BC02FF86FF2029F4809137
:109EE000BB02882309F460C010922303109224035C
:109EF000109225031092260310921F031092200344
:109F00001092210310922203109206081092070863
:109F1000109208081092090810920E0810920F086B
:109F200010921008109211081092FD071092FE076F
:109F30001092FF07109200081092EE071092EF07A0
:109F40001092F0071092F10780911303909114037F
:109F5000A0911503B091160380930F039093100303
:109F6000A0931103B093120380910B0390910C0303
:109F7000A0910D03B0910E03809307039093080303
:109F8000A0930903B0930A031092EA011092E90129
:109F90001092C0021092BF021092C2021092C1022F
:109FA0000F85002309F0F8C18091BB02882309F0D6
:109FB000F3C18091E4059091E505815092402CF425
:109FC0008091D802882309F4E7C19090BE08A09040
:109FD0005E0620903208309033084090420850903E
:109FE000430819140CF0E3C0BB24CC24DD24CA01BF
:109FF000B901A60195010E94978B79018A01809190
:10A00000870890918808281A390AC101AA2797FD64
:10A01000A095BA2FE81AF90A0A0B1B0B6B817C81F9
:10A020008D819E81A60195010E94978B59016A013D
:10A030008091890890918A08481A590AC201AA2772
:10A0400097FDA095BA2FA81AB90ACA0ADB0A292CCB
:10A05000332427FC3094432C532CC801B701A201B0
:10A0600091010E94238B97FF04C061507E4F8F4F58
:10A070009F4F3B014C0109E0959487947794679436
:10A080000A95D1F7C601B501A20191010E94238B67
:10A0900097FF04C061507E4F8F4F9F4F5B016C0153
:10A0A00019E0D594C794B794A7941A95D1F78091E5
:10A0B000A6029091A702813491053CF48091A402FC
:10A0C0009091A50281349105D4F0D401C30197FE8B
:10A0D00003C00196A11DB11D3C014D0195948794CB
:10A0E00077946794D601C501D7FE03C00196A11DE0
:10A0F000B11D5C016D01D594C794B794A79480916C
:10A100004606E82FFF27EE0FFF1FEB58F84F808120
:10A1100091810190F081E02DF7FF03C0F095E1956A
:10A12000FF4F7A97A4F0C401B30123E030E040E090
:10A1300050E00E94978B39014A01C601B50123E026
:10A1400030E040E050E00E94978B59016A01809115
:10A15000C008282F332727FD3095432F532F26156E
:10A1600037054805590514F439014A01992787FD37
:10A170009095909581959F4FAA2797FDA095BA2F0E
:10A18000681679068A069B0614F43C014D012A15CF
:10A190003B054C055D0514F459016A01A816B90682
:10A1A000CA06DB060CF0D0C05C016D01CDC0EA2C04
:10A1B000FF2400271127CA01B901A80197010E94B5
:10A1C000978B39014A01C101AA2797FDA095BA2FA3
:10A1D000681A790A8A0A9B0A6B817C818D819E812B
:10A1E000A80197010E94978B59016A01C201AA2711
:10A1F00097FDA095BA2FA81AB90ACA0ADB0AD4019A
:10A20000C30197FE03C00F96A11DB11D3C014D0176
:10A21000F4E09594879477946794FA95D1F7D601F2
:10A22000C501D7FE03C00F96A11DB11D5C016D01D4
:10A23000E4E0D594C794B794A794EA95D1F78091B8
:10A24000A6029091A702813491053CF48091A4026A
:10A250009091A50281349105A4F0C401B30123E0DB
:10A2600030E040E050E00E94978B39014A01C6017E
:10A27000B50123E030E040E050E00E94978B5901A7
:10A280006A0180914606E82FFF27EE0FFF1FEB586B
:10A29000F84F808191810190F081E02DF7FF03C09C
:10A2A000F095E195FF4F7A97A4F0C401B30123E044
:10A2B00030E040E050E00E94978B39014A01C6012E
:10A2C000B50123E030E040E050E00E94978B590157
:10A2D0006A0189E180938C0121E262167104810494
:10A2E00091042CF070E2672E712C812C912C30EEB1
:10A2F00063163FEF73063FEF83063FEF930644F488
:10A3000060EE662E6FEF762E6FEF862E6FEF962E35
:10A3100041E2A416B104C104D1042CF050E2A52EF0
:10A32000B12CC12CD12C50EEA5165FEFB5065FEF16
:10A33000C5065FEFD50644F440EEA42E4FEFB42ED1
:10A340004FEFC42E4FEFD42E80911303909114033E
:10A35000A0911503B091160386199709A809B909A8
:10A360008093130390931403A0931503B0931603E3
:10A3700080910B0390910C03A0910D03B0910E03FB
:10A380008A199B09AC09BD0980930B0390930C03B8
:10A39000A0930D03B0930E038091E9019091EA011F
:10A3A0008F3F910509F008F4C4C56F85662309F055
:10A3B0004EC58091BB02882309F049C58091EF0208
:10A3C000882309F044C570918606788B772309F4B9
:10A3D0003EC58091060890910708A0910808B091A9
:10A3E0000908B7FF04C081509F4FAF4FBF4FE92E00
:10A3F000FA2E0B2F112707FD1A95E0920608F0920E
:10A400000708009308081093090880910E0890919E
:10A410000F08A0911008B0911108B7FF04C0815037
:10A420009F4FAF4FBF4F892F9A2FAB2FBB27A7FD51
:10A43000BA95898B9A8BAB8BBC8B80930E089093CB
:10A440000F08A0931008B093110880915E06A82E03
:10A45000BB24CC24DD24209123033091240340919C
:10A46000250350912603C601B5010E94238B97FF57
:10A4700004C061507F4F8F4F9F4F672E782E892EDB
:10A48000992487FC9A94609223037092240380920B
:10A4900025039092260320911F03309120034091C1
:10A4A000210350912203C601B5010E94238B97FF1F
:10A4B00004C061507F4F8F4F9F4F272E382E492E5B
:10A4C000552447FC5A9420921F0330922003409257
:10A4D00021035092220380911B0390911C03A091B1
:10A4E0001D03B0911E03B7FF04C081509F4FAF4FB3
:10A4F000BF4F892F9A2FAB2FBB27A7FDBA9580930B
:10A500001B0390931C03A0931D03B0931E03D8015B
:10A51000C70186199709A809B90980937003909318
:10A520007103A0937203B093730320918506E22E0A
:10A53000FF2400271127BC01CD01A80197010E942B
:10A54000978B59016A0120937D0330937E034093DA
:10A550007F035093800389899A89AB89BC898219CA
:10A560009309A409B5098093740390937503A0938C
:10A570007603B0937703BC01CD01A80197010E9437
:10A58000978B2093810330938203409383035093EE
:10A590008403D601C501D7FE04C081509F4FAF4F41
:10A5A000BF4F892F9A2FAB2FBB27A7FDBA9590934A
:10A5B000C0028093BF0257FF04C021503F4F4F4F4E
:10A5C0005F4FBB2757FDBA95A52F942F832F9093EC
:10A5D000C2028093C1028091A6029091A7028134A9
:10A5E0009105DCF48091A4029091A502813491053B
:10A5F000A4F480914606E82FFF27EE0FFF1FEB58CB
:10A60000F84F808191810190F081E02DF7FF03C028
:10A61000F095E195FF4F7A97E4F08091BE088F3F67
:10A62000C1F48091BF029091C00297FD019695956B
:10A6300087959093C0028093BF028091C102909150
:10A64000C20297FD0196959587959093C2028093DB
:10A65000C1028091FD079091FE07A091FF07B09184
:10A660000008B7FF04C081509F4FAF4FBF4F892FE5
:10A670009A2FAB2FBB27A7FDBA958093FD07909328
:10A68000FE07A093FF07B09300088091EE0790911A
:10A69000EF07A091F007B091F107B7FF04C0815018
:10A6A0009F4FAF4FBF4F892F9A2FAB2FBB27A7FDCF
:10A6B000BA958093EE079093EF07A093F007B093BD
:10A6C000F1078091330390913403A0913503B09149
:10A6D00036032F81388549855A85281B390B4A0B4B
:10A6E0005B0B209368033093690340936A03509394
:10A6F0006B0380912B0390912C03A0912D03B091BB
:10A700002E03EB84FC840D851E85E81AF90A0A0BDA
:10A710001B0BE0926C03F0926D0300936E03109399
:10A720006F0320937003309371034093720350932F
:10A730007303E0927403F092750300937603109311
:10A74000770380910F0390911003A0911103B091B2
:10A750001203821B930BA40BB50B80930F039093F2
:10A760001003A0931103B0931203809107039091FB
:10A770000803A0910903B0910A038E199F09A00B49
:10A78000B10B8093070390930803A0930903B09340
:10A790000A0388898823E1F02091ED023091EE02CE
:10A7A000213831054CF08091440390914503019686
:10A7B000909345038093440320583F4F4CF480917D
:10A7C000440390914503019790934503809344037C
:10A7D0001092EE021092ED0281E090E090938A03D5
:10A7E00080938903E0907003F090710300917203ED
:10A7F00010917303D801C70117FF07C08827992755
:10A80000DC018E199F09A00BB10B81509240A04032
:10A81000B04034F084E090E090938A038093890301
:10A8200080918F0390919003A0919103B091920336
:10A8300020910608309107084091080850910908B6
:10A84000821B930BA40BB50B815E914BAF4FBF4F97
:10A850008F539C49A040B04028F08091BF088931B7
:10A860000CF4FFC021E0E21620E1F20620E002072E
:10A8700020E012070CF473C080918B03882309F445
:10A880006AC0D801C70117FF07C088279927DC01D4
:10A890008E199F09A00BB10B9C01AD01B7FF04C03D
:10A8A00021503E4F4F4F5F4FF9E0559547953795F3
:10A8B0002795FA95D1F78091890390918A03820FA9
:10A8C000931F90938A0380938903D801C70117FFD0
:10A8D00003C00796A11DB11DE3E0B595A795979517
:10A8E0008795EA95D1F780937D0390937E03A0939B
:10A8F0007F03B093800389589341A040B04064F037
:10A9000088E893E1A0E0B0E080937D0390937E031C
:10A91000A0937F03B093800320917D0330917E0349
:10A9200040917F035091800357FF04C021503F4F57
:10A930004F4F5F4F232F342F452F552747FD5A95F3
:10A940008091BF029091C002820F931F9093C0022A
:10A950008093BF0206C081E080938B0302C01092F7
:10A960008B0340E0E41640EFF4064FEF04074FEF8F
:10A9700014070CF073C080918C03882309F46AC01B
:10A98000D801C70117FF07C088279927DC018E1956
:10A990009F09A00BB10B9C01AD01B7FF04C0215072
:10A9A0003E4F4F4F5F4F69E0559547953795279537
:10A9B0006A95D1F78091890390918A03820F931F42
:10A9C00090938A0380938903D801C70117FF03C0BE
:10A9D0000796A11DB11D23E0B595A795979587957D
:10A9E0002A95D1F780937D0390937E03A0937F03F4
:10A9F000B093800388579C4EAF4FBF4F64F488E7F5
:10AA00009CEEAFEFBFEF80937D0390937E03A09306
:10AA10007F03B093800320917D0330917E034091AA
:10AA20007F035091800357FF04C021503F4F4F4F89
:10AA30005F4F232F342F452F552747FD5A9580917F
:10AA4000BF029091C002820F931F9093C002809327
:10AA5000BF0211C081E080938C030DC010928C0363
:10AA60000AC010928A031092890384E690E09093C2
:10AA70008B0180938A016889262F3327809189036F
:10AA800090918A032817390724F430938A0320937E
:10AA900089031091BF08112379F0212F332727FD57
:10AAA00030958091890390918A032817390724F4FF
:10AAB00030938A032093890340917003509171036E
:10AAC00060917203709173034138510561057105FE
:10AAD00074F080914803909149032091890330914B
:10AAE0008A03820F931F9093490380934803405831
:10AAF0005F4F6F4F7F4F74F48091480390914903EB
:10AB00002091890330918A03821B930B9093490310
:10AB10008093480381E090E090938A0380938903B7
:10AB2000C0907403D0907503E0907603F0907703A3
:10AB3000D701C601F7FE07C088279927DC018C19C9
:10AB40009D09AE09BF0981509240A040B04034F049
:10AB500084E090E090938A0380938903809193032B
:10AB600090919403A0919503B091960320910E08C3
:10AB700030910F084091100850911108821B930BDF
:10AB8000A40BB50B815E914BAF4FBF4F8F539C49C8
:10AB9000A040B04018F019310CF4FFC001E0C0161D
:10ABA00000E1D00600E0E00600E0F0060CF473C01F
:10ABB00080918D03882309F46AC0D701C601F7FE8E
:10ABC00007C088279927DC018C199D09AE09BF09A8
:10ABD0009C01AD01B7FF04C021503E4F4F4F5F4F66
:10ABE00009E055954795379527950A95D1F78091B6
:10ABF000890390918A03820F931F90938A03809315
:10AC00008903D701C601F7FE03C00796A11DB11D38
:10AC100013E0B595A795979587951A95D1F78093E9
:10AC2000810390938203A0938303B0938403895894
:10AC30009341A040B04064F088E893E1A0E0B0E028
:10AC40008093810390938203A0938303B093840342
:10AC500020918103309182034091830350918403BA
:10AC600057FF04C021503F4F4F4F5F4F232F342FCA
:10AC7000452F552747FD5A958091C1029091C202F8
:10AC8000820F931F9093C2028093C10206C081E09D
:10AC900080938D0302C010928D0320E0C21620EF36
:10ACA000D2062FEFE2062FEFF2060CF073C0809170
:10ACB0008E03882309F46AC0D701C601F7FE07C0D6
:10ACC00088279927DC018C199D09AE09BF099C01D1
:10ACD000AD01B7FF04C021503E4F4F4F5F4FE9E039
:10ACE0005595479537952795EA95D1F78091890332
:10ACF00090918A03820F931F90938A038093890314
:10AD0000D701C601F7FE03C00796A11DB11D73E070
:10AD1000B595A795979587957A95D1F780938103F7
:10AD200090938203A0938303B093840388579C4E2F
:10AD3000AF4FBF4F64F488E79CEEAFEFBFEF809357
:10AD4000810390938203A0938303B09384032091A3
:10AD5000810330918203409183035091840357FF14
:10AD600004C021503F4F4F4F5F4F232F342F452FAB
:10AD7000552747FD5A958091C1029091C202820FDA
:10AD8000931F9093C2028093C10211C081E080930F
:10AD90008E030DC010928E030AC010928A03109287
:10ADA000890384E690E090938B0180938A0148891F
:10ADB000242F33278091890390918A03281739071C
:10ADC00024F430938A03209389038091BF08882359
:10ADD00079F0282F332727FD3095809189039091B2
:10ADE0008A032817390724F430938A0320938903B0
:10ADF00040917403509175036091760370917703CD
:10AE0000413851056105710574F0809146039091B8
:10AE100047032091890330918A03820F931F9093F7
:10AE200047038093460340585F4F6F4F7F4FCCF4EA
:10AE300080914603909147032091890330918A03C2
:10AE4000821B930B90934703809346030AC0109292
:10AE5000C2021092C1021092C0021092BF02109260
:10AE6000EF0280911408882341F41092C2021092DC
:10AE7000C1021092C0021092BF0280910608909108
:10AE80000708A0910808B091090880938F03909358
:10AE90009003A0939103B093920380910E08909138
:10AEA0000F08A0911008B09111088093930390931C
:10AEB0009403A0939503B0939603109223031092EA
:10AEC0002403109225031092260310921F03109260
:10AED0002003109221031092220310921B03109260
:10AEE0001C0310921D0310921E031092060810926C
:10AEF0000708109208081092090810920E08109284
:10AF00000F0810921008109211081092FD0710926D
:10AF1000FE071092FF07109200081092EE071092A1
:10AF2000EF071092F0071092F1071092EA011092C9
:10AF3000E901E090E502F090E602C701F7FE04C0E7
:10AF4000882799278E199F0904973CF080912E0835
:10AF500084FD03C082E38093C30210915B06A12E9F
:10AF6000BB24CC24DD24B701882777FD8095982F5A
:10AF70009701F7FE04C0222733272E193F094427E3
:10AF800037FD4095542F0E94238B9B01AC01C601D5
:10AF9000B5010E94238B97FF04C061507E4F8F4FF5
:10AFA0009F4F59E095958795779567955A95D1F775
:10AFB0009B01812F99278E9DD0018F9DB00D9E9D65
:10AFC000B00D1124CD01B7FD039695958795959504
:10AFD0008795280F391F8091C5029091C602280FCE
:10AFE000391F442737FD4095542F20936403309335
:10AFF0006503409366035093670380910303909128
:10B000000403A0910503B0910603821B930BA40BCC
:10B01000B50B8093030390930403A0930503B093AF
:10B0200006038155934CA040B04064F080E593EC5A
:10B03000A0E0B0E08093030390930403A093050382
:10B04000B09306038091030390910403A09105033C
:10B05000B0910603805B9C43AF4FBF4F64F480EB1D
:10B060009CE3AFEFBFEF8093030390930403A0939F
:10B070000503B093060300918E0110918F0117FD17
:10B08000FCC080912E0883FFF8C080918D01815013
:10B0900080938D01882309F0F4C08DE080938D01A9
:10B0A0008091330390913403A0913503B09136031E
:10B0B000B7FF04C081509E4FAF4FBF4F39E0B595E9
:10B0C000A795979587953A95D1F77C0197FF04C08E
:10B0D000F094E194F108F39480912B0390912C0368
:10B0E000A0912D03B0912E03B7FF04C081509E4F55
:10B0F000AF4FBF4F29E0B595A795979587952A95AE
:10B10000D1F79C0197FF03C0309521953F4FE21680
:10B11000F3060CF47901B701F7FE02C0695F7F4FB7
:10B120002B01A3E055944794AA95E1F722E030E083
:10B13000420E531E60903E0870903F088090400879
:10B140009090410820914201309143014091440187
:10B1500050914501C401B3010E94978B59016A01C6
:10B160003093EC072093EB07021B130BC801845E9E
:10B170009D4F68E671E00E94628B9C01245B304029
:10B1800080918A0190918B01009731F00197909303
:10B190008B0180938A011BC049E1E416F104BCF4E1
:10B1A0008091ED029091EE02820F931F9093EE0238
:10B1B0008093ED028091C302882349F081508093EF
:10B1C000C302882321F4B092F202A092F10280918E
:10B1D0008A0190918B01892BF9F480918C01992738
:10B1E000289FB001299F700D389F700D1124CB014D
:10B1F000B2010E94628BCB01AA2797FDA095BA2FBE
:10B20000680E791E8A1E9B1E60923E0870923F084F
:10B2100080924008909241088091C302882369F58A
:10B220008091F1029091F2022091EB073091EC07AE
:10B23000821B930B845E9D4F68E671E00E94628BD7
:10B240009C01245B30408091760186959927289F48
:10B25000D001299FB00D389FB00D11249D01B7FF7B
:10B2600002C0215F3F4FF4E035952795FA95E1F74D
:10B270003093C6022093C50204C01092C6021092F9
:10B28000C5028091EF02882381F01092F70210929C
:10B29000F8021092F9021092FA021092FB02109238
:10B2A000FC021092FD021092FE02F090BC02FF2000
:10B2B000F1F480911408282F3327442755278091D3
:10B2C000330390913403A0913503B0913603BC0150
:10B2D000CD010E94238BDC01CB01BC01CD0128EF05
:10B2E0003AE240E050E00E94978B390102C06624A8
:10B2F0007724E090BB02EE20F1F480911408282F0F
:10B3000033274427552780912B0390912C03A0913C
:10B310002D03B0912E03BC01CD010E94238BDC01D3
:10B32000CB01BC01CD0128EF3AE240E050E00E94A1
:10B33000978B290102C0442455248091E8079091FD
:10B34000E907893C91051CF088EC90E005C0885322
:10B350009F4F34F488E39FEF9093E9078093E807C9
:10B360008091F4079091F507893C91051CF088ECD9
:10B3700090E005C088539F4F34F488E39FEF90938B
:10B38000F5078093F4078091F6079091F707AA27B5
:10B3900097FDA095BA2F20913C08A22EBB24CC2467
:10B3A000DD24BC01CD01A60195010E94238B9B01E8
:10B3B000AC018091E8079091E907AA2797FDA09535
:10B3C000BA2FE7E0880F991FAA1FBB1FEA95D1F794
:10B3D000280F391F4A1F5B1F57FF04C0215C3F4FD6
:10B3E0004F4F5F4F76E055954795379527957A955E
:10B3F000D1F78301020F131F1093F7070093F6078D
:10B400008091E6079091E707AA2797FDA095BA2FAC
:10B41000BC01CD01A60195010E94238B9B01AC01CB
:10B420008091F4079091F507AA2797FDA095BA2F70
:10B4300067E0880F991FAA1FBB1F6A95D1F7280FD5
:10B44000391F4A1F5B1F57FF04C0215C3F4F4F4FFE
:10B450005F4FF6E05595479537952795FA95D1F7C3
:10B460004201820E931E9092E7078092E607809138
:10B47000370890913808880F991FAA2797FDA09543
:10B48000BA2F2091ED07332744275527BC01CD0162
:10B490000E94238B5B016C0197FF08C02FE330E013
:10B4A00040E050E0A20EB31EC41ED51EE6E0D594C7
:10B4B000C794B794A794EA95D1F780910308282FF1
:10B4C0003327442755278091170390911803A091A3
:10B4D0001903B0911A03BC01CD010E94238BDC013A
:10B4E000CB01BC01CD0120EF35E540E050E00E94EA
:10B4F000978BB501620F731F7093380860933708FC
:10B500000150104134F080E090E19093F707809370
:10B51000F6078091F6079091F7078050904F34F42A
:10B5200080E090EF9093F7078093F60751E085163F
:10B5300050E1950634F080E090E19093E707809326
:10B54000E6078091E6079091E7078050904F34F42A
:10B5500080E090EF9093E7078093E6076150704199
:10B5600034F080E090E19093380880933708809120
:10B570003708909138088050904F34F480E090EF75
:10B58000909338088093370880910001482F552701
:10B5900080911D0190911E014817590794F4209144
:10B5A0001D0130911E0109811A81049FC001059F70
:10B5B000900D149F900D1124B9010E944E8B7A8337
:10B5C000698329813A81220F331F220F331F3A8367
:10B5D000298340912E0840FD02C00C94DD62EE20CC
:10B5E00009F0EBC7FF2009F0E8C700E010E04801D0
:10B5F0008091BD029091BE029093CC058093CB05C3
:10B6000020914A0330914B032115310509F03FC0C9
:10B6100080911301909114018959934058F087B596
:10B62000803F20F48091ED01815011C081E0809332
:10B63000A0034EC0809113019091140184369105AE
:10B6400008F587B58031D0F08091ED018F5F809350
:10B65000ED019FE08902900111248091EE05821B8B
:10B6600087BD8CE291E09093DB018093DA018EE557
:10B6700091E090934B0380934A032AC081E080932A
:10B680009F0326C0F0929F03F092A00321C08091F7
:10B69000D3029091D402A091D502B091D60264E079
:10B6A000880F991FAA1FBB1F6A95D1F78093EE01DF
:10B6B0009093EF01A093F001B093F1011093EC018E
:10B6C0000093EB012150304030934B0320934A0309
:10B6D0002091790141FF24C02233D8F48091900158
:10B6E0008150809390018F3FD9F51092F0028091A4
:10B6F000D3029091D402A091D502B091D60280934A
:10B70000CF029093D002A093D102B093D20281E0F5
:10B7100004C081E08093F00288EC8093900120C007
:10B720008091460190914701820F911D209154060E
:10B730003327829FA001839F500D929F500D1124AB
:10B74000CA01AA2797FDA095BA2F8093CF029093A4
:10B75000D002A093D102B093D20281E08093F00294
:10B760008091330390913403A0913503B091360357
:10B77000E0904201F0904301009144011091450195
:10B78000BC01CD01A80197010E94978B59016A0164
:10B7900080912B0390912C03A0912D03B0912E0347
:10B7A000BC01CD01A80197010E94978BB901C50189
:10B7B0000E944C7F5C01CC971CF05CE3A52EB12C61
:10B7C000C5010E94F36F5C0180E2809341011092F9
:10B7D000CE021092CD028091F002882309F45FC559
:10B7E0008091A10299279C012071307084FD57C57A
:10B7F0008091A00282608093A00270911208872F2E
:10B80000992741E0C42ED12CC822D92280FD04C042
:10B8100080912E0881FD10C0C980DA803093980392
:10B82000209397033093CE022093CD028091A10202
:10B83000806C8093A102ABC28091A10281FF7AC289
:10B840000091800110918101C8010F962090E302C0
:10B850003090E402821593050CF058C080919F034C
:10B86000882309F053C08091A10287FF15C0809101
:10B87000A1028F778093A1028091D3029091D4028C
:10B88000A091D502B091D6028093CF029093D002BE
:10B89000A093D102B093D2028091A10280648093E0
:10B8A000A102E090F207EE20F1F08091CF0290919A
:10B8B000D002A091D102B091D202BC01CD0124E608
:10B8C00030E040E050E00E94978B8E2D9927AA2708
:10B8D000BB2782179307A407B5072CF4D092CE029A
:10B8E000C092CD0210C0C101801B910B0F9797FF32
:10B8F00003C0909581959F4F9093CE028093CD0287
:10B900008BE2809341011092C70216C1C8010F97C4
:10B9100028163906C4F52091A0032223A1F58091B1
:10B92000A10286FF15C08091A1028F7B8093A102A6
:10B930008091D3029091D402A091D502B091D60209
:10B940008093CF029093D002A093D102B093D20201
:10B950008091A10280688093A102C101801B910B9C
:10B960000F9697FF03C0909581959F4F9095819575
:10B970009F4F9093CE028093CD028DE28093410140
:10B980002093C702D9C08DE3809341016091C80222
:10B99000662371F12091C9023091CA024091CB0215
:10B9A0005091CC028091CF029091D002A091D1020F
:10B9B000B091D20282179307A407B507CCF4809107
:10B9C000A10280648093A102862F99279093CE02D2
:10B9D0008093CD028AE08093C7028EE58093410177
:10B9E0008091A10287FFA8C08091A1028F7733C008
:10B9F000662309F443C02091C9023091CA024091E4
:10BA0000CB025091CC028091CF029091D002A091B4
:10BA1000D102B091D202281739074A075B0774F5A3
:10BA20008091A10280688093A102862F992790952A
:10BA300081959F4F9093CE028093CD0286EF8093A5
:10BA4000C70286E7809341018091A10286FF74C0FE
:10BA50008091A1028F7B8093A1028091D30290916B
:10BA6000D402A091D502B091D6028093CF029093D8
:10BA7000D002A093D102B093D2025EC08091A10205
:10BA8000807C09F459C08091C702882379F5E09041
:10BA9000D302F090D4020091D5021091D602D801C1
:10BAA000C70180589040A040B0402091CF02309113
:10BAB000D0024091D1025091D20282179307A4077D
:10BAC000B5075CF4D801C70180589F4FAF4FBF4FF7
:10BAD000281739074A075B075CF08093CF029093E1
:10BAE000D002A093D102B093D20202C01092C7023A
:10BAF0008091A1028F738093A102109298031092FB
:10BB0000970371FF06C084EF91E09093DB0180936F
:10BB1000DA018091D702882379F48091D302909141
:10BB2000D402A091D502B091D602C397A105B10568
:10BB30001CF081E08093D702609197037091980385
:10BB40008091CD029091CE02680F791F7093980377
:10BB500060939703CB0177FF04C088279927861B42
:10BB6000970B855F91400CF4CEC04091C7024423EF
:10BB700089F18091C9029091CA022091CF0230913F
:10BB8000D002821B930B0996439748F48091C90217
:10BB90009091CA02A091CB02B091CC0212C0242F86
:10BBA000332727FD3095432F532F8091CF0290915B
:10BBB000D002A091D102B091D202820F931FA41F94
:10BBC000B51F8093CF029093D002A093D102B0937F
:10BBD000D20224C0809154062091CF023091D0022D
:10BBE0004091D1025091D2021616170644F463E038
:10BBF0000E94428B280F311D411D511D07C063E07B
:10BC00000E94428B281B3109410951092093CF0220
:10BC10003093D0024093D1025093D20210929803F5
:10BC200010929703E090D302F090D4020091D502D5
:10BC30001091D602D801C70180509440A040B04076
:10BC40002091CF023091D0024091D1025091D20286
:10BC500082179307A407B5075CF4D801C701805089
:10BC60009C4FAF4FBF4F281739074A075B0744F077
:10BC70008093CF029093D002A093D102B093D202CE
:10BC80008091120881FF06C084E690E09093DB016A
:10BC90008093DA01809158068823A9F58091C80223
:10BCA000882389F54091BD025091BE0257FF02C022
:10BCB0004D5F5F4F559547955595479580911D016F
:10BCC00090911E01209100013327489FF001499F68
:10BCD000F00D589FF00D1124CF01B9010E94628B25
:10BCE0007093810160938001663471051CF486E4D1
:10BCF00090E005C06739710534F086E990E09093D3
:10BD000081018093800180914A0390914B03892B9C
:10BD1000D1F18091D3029091D402A091D502B0913B
:10BD2000D6028093CF029093D002A093D102B09319
:10BD3000D20229C08091D3029091D402A091D50261
:10BD4000B091D60280599140A040B0408093CF027C
:10BD50009093D002A093D102B093D2028091580662
:10BD6000882311F0992702C088E790E09093810121
:10BD700080938001E980FA80F092BE02E092BD02D9
:10BD80008EE280934101C090BD02D090BE02E0904F
:10BD9000D302F090D4020091D5021091D6022091E6
:10BDA000CF023091D0024091D1025091D2022E1593
:10BDB0003F054007510724F08091120880FDBBC267
:10BDC00080914A0390914B03892B39F0C090BD02BA
:10BDD000D090BE0200E010E0D7C0D801C701821B9E
:10BDE000930BA40BB50B8093680390936903A09306
:10BDF0006A03B0936B03823000E890070FEFA0074F
:10BE00000FEFB0072CF481E090E8AFEFBFEF09C06F
:10BE10008F5F9F47A040B04064F08FEF9FE7A0E0A6
:10BE2000B0E08093680390936903A0936A03B09392
:10BE30006B03009168031091690380917801282FAA
:10BE40003327442755278091680390916903A09177
:10BE50006A03B0916B03BC01CD010E94238B97FF55
:10BE600004C0615E7F4F8F4F9F4F25E0959587956A
:10BE7000779567952A95D1F7609368037093690366
:10BE800080936A0390936B0365302EEF72072FEF58
:10BE900082072FEF92072CF484E09EEFAFEFBFEF05
:10BEA00009C0605074408040904064F080E094E0AD
:10BEB000A0E0B0E08093680390936903A0936A03C5
:10BEC000B0936B0380906803909069032091EB011D
:10BED0003091EC0137FF02C0295F3F4F83E0359579
:10BEE00027958A95E1F74FEF223834071CF421E8B3
:10BEF0003FEF05C02038310514F020E830E0C901DB
:10BF0000AA2797FDA095BA2F20917A0133274427BD
:10BF10005527BC01CD010E94238B97FF04C06D5FA4
:10BF20007F4F8F4F9F4FB2E0959587957795679597
:10BF3000BA95D1F79B015FEF613075071CF420E0E3
:10BF40003FEF06C06F3F710519F014F020E031E0BB
:10BF50008091A102807C49F0C90137FD03969C01C4
:10BF600035952795359527950DC08091120880FF4E
:10BF700009C0C90137FD07969C01F3E03595279567
:10BF8000FA95E1F7820E931E20917701222309F49E
:10BF900054C06091F3027091F4028091F502909187
:10BFA000F60297FF04C061587F4F8F4F9F4FE7E025
:10BFB0009595879577956795EA95D1F73327442727
:10BFC00055270E94238B97FF04C0615E7F4F8F4FE0
:10BFD0009F4F55E095958795779567955A95D1F739
:10BFE000609368037093690380936A0390936B0373
:10BFF0006138AFEF7A07AFEF8A07AFEF9A072CF4FB
:10C0000080E89FEFAFEFBFEF0AC06F3F710581057A
:10C01000910569F064F080E091E0A0E0B0E08093E9
:10C02000680390936903A0936A03B0936B038091B4
:10C03000680390916903880E991E80917501282FDD
:10C0400033278091C208992787FD9095289FF0019A
:10C05000299FF00D389FF00D11249F01F7FF02C0BA
:10C0600021583F4F220F232F221F330BFFEF213880
:10C070003F071CF420E83FEF06C02F3F310519F0C1
:10C0800014F020E031E0820E931EC401AA2797FD30
:10C09000A095BA2FE090BD02F090BE029701442710
:10C0A00037FD4095542FBC01CD010E94238B97FF93
:10C0B00004C061507E4F8F4F9F4F29E09595879523
:10C0C000779567952A95D1F7C61AD70A8091CD0240
:10C0D0009091CE02892B09F060C01E141F040CF051
:10C0E0005CC0980117FF03C0309521953F4F2D3359
:10C0F000310540F48091EB029091EC028C159D0586
:10C1000074F526C02C53304085E0369527958A95E6
:10C11000E1F72031310510F02FE030E04091EB02E3
:10C120005091EC0210161106E4F480E190E0821BBD
:10C13000930B489F9001499F300D589F300D11245B
:10C14000B4E036952795BA95E1F72C153D0520F515
:10C1500080917E0190917F01C816D906F4F06C01A0
:10C160001CC0205F3F4F80917E0190917F01829F94
:10C170008001839F100D929F100D11249801A4E05F
:10C1800036952795AA95E1F74C155D0514F06A01DF
:10C1900004C0C216D30608F06901C601AA2797FD9C
:10C1A000A095BA2FFDE0880F991FAA1FBB1FFA9513
:10C1B000D1F79501442737FD4095542FBC01CD019F
:10C1C0000E94978B20936C0330936D0340936E0312
:10C1D00050936F03C0906C03D0906D0380919903CE
:10C1E00090919A039C01220F331F280F391F2C0DA9
:10C1F0003D1D37FF02C02D5F3F4FA9015595479563
:10C200005595479550939A03409399038091500612
:10C21000282F3327220F331F220F331F24173507F0
:10C220006CF480913608282F3327220F331F220FFA
:10C23000331F205530404217530724F030939A03A0
:10C24000209399038091120880FF14C08091990374
:10C2500090919A0329813A818217930724F03093B1
:10C260009A03209399034091990350919A035A831A
:10C27000498361C029813A812E193F0937FF02C0E5
:10C280002D5F3F4F359527953595279560919903FB
:10C2900070919A03620F731F7A8369834CC08091F7
:10C2A0005806882301F56091BD027091BE0277FFA8
:10C2B00002C06D5F7F4F7595679575956795409145
:10C2C0001D0150911E0180910001282F3327649F8A
:10C2D000C001659F900D749F900D1124B9010E94BB
:10C2E000628BCB0101C099279093810180938001DB
:10C2F0008091800190918101873491051CF486E43E
:10C3000090E005C08639910534F086E990E090937D
:10C3100081018093800189819A8190939A0380930F
:10C3200099038091A102806C8093A1028091A00268
:10C330008D7F8093A0028091A10299279C01227099
:10C34000307081FF2BC180919B0390919C03A09141
:10C350009D03B0919E030097A105B10521F0809146
:10C36000D7028130B1F4E981FA81CF01AA2797FD84
:10C37000A095BA2F1EE0880F991FAA1FBB1F1A9500
:10C38000D1F780939B0390939C03A0939D03B0935C
:10C390009E038091D702813019F482E08093D70206
:10C3A000E980FA80C701AA2797FDA095BA2F9501C9
:10C3B000442737FD4095542FBC01CD010E94238BAB
:10C3C000DC01CB0180936C0390936D03A0936E030B
:10C3D000B0936F03B7FF04C08150904EAF4FBF4F73
:10C3E0007C018D01ADE015950795F794E794AA952A
:10C3F000D1F7E0926C03F0926D0300936E031093FB
:10C400006F036091A2027091A3022FE0603A72075D
:10C4100050F580919B0390919C03A0919D03B09156
:10C420009E039C01AD01FAE05695479537952795F7
:10C43000FA95D1F7821B930BA40BB50BA8019701BA
:10C44000E4E0220F331F441F551FEA95D1F7820FF6
:10C45000931FA41FB51F80939B0390939C03A093ED
:10C460009D03B0939E0360547F4118F580919B0318
:10C4700090919C03A0919D03B0919E039C01AD01FE
:10C480006CE056954795379527956A95D1F7821BAD
:10C49000930BA40BB50BA8019701F2E0220F331FF9
:10C4A000441F551FFA95D1F7820F931FA41FB51F84
:10C4B00038C08091EB019091EC018091EB0190915B
:10C4C000EC0197FF03C0909581959F4F84369105AD
:10C4D00084F58091D3029091D4022091CF023091C3
:10C4E000D002821B930B81509F4F8F5F914008F5C4
:10C4F00080919B0390919C03A0919D03B0919E031A
:10C500009C01AD01EEE05695479537952795EA9544
:10C51000D1F7821B930BA40BB50B8E0D9F1DA01F93
:10C52000B11F80939B0390939C03A0939D03B093B2
:10C530009E0380919B0390919C03A0919D03B091D9
:10C540009E037EE0B695A795979587957A95D1F746
:10C550009093BE028093BD0240915606442399F009
:10C5600055279C01BA010E94628BC901861B970B5B
:10C570009093EC028093EB02260F371F30937F01DC
:10C5800020937E011FC01092EC021092EB028FEFFD
:10C5900093E090937F0180937E0114C01092D702A4
:10C5A00010929B0310929C0310929D0310929E0385
:10C5B0003093BE022093BD0205C08091A102806C21
:10C5C0008093A1028091AF0381FF37C089819A8156
:10C5D00097FD0396959587959595879520919E0251
:10C5E00030919F022817390760F48091BD02909125
:10C5F000BE02892B31F0220F331F220F331F3A83E3
:10C6000029838091D3029091D402A091D502B09158
:10C61000D6028093CF029093D002A093D102B09320
:10C62000D20288E99AE39093DB018093DA0180E0FB
:10C630009EE090930801809307012091FB07822FD1
:10C640009927880F991F880F991F889669817A8189
:10C650008617970714F09A838983709136087D8B2B
:10C66000872F9927880F991F880F991F8055904011
:10C67000A981BA818A179B0714F49A8389838091D0
:10C680002202882341F48091D4088F3F21F48091C5
:10C69000B3038823E9F08091A2029091A30202974C
:10C6A000C097B0F4E981FA811E161F068CF481E070
:10C6B00090E09093A3028093A202E22EFF24EE0C5E
:10C6C000FF1CEE0CFF1C8701085D1F4F1A830983B6
:10C6D00029813A813093B0052093AF05809164039E
:10C6E00090916503A0916603B091670312E0880FF3
:10C6F000991FAA1FBB1F1A95D1F7009137081091F7
:10C700003808081B190B213A31058CF0C90137FD97
:10C71000019695958795801791070CF48C0190955B
:10C7200081959F4F081719076CF48C010BC00135D8
:10C73000110514F000E510E03FEF003B130714F47F
:10C7400000EB1FEF4D89242F3327220F331F220FB9
:10C75000331FC90169817A81861B970B8017910766
:10C760000CF48C0189819A81821B930B081719079D
:10C770000CF48C018091F6079091F7076091E90223
:10C780007091EA02861B970B90930508809304082A
:10C79000D09014082091FB023091FC024091FD02E0
:10C7A0005091FE02DD2041F0661A770AC301AA27E4
:10C7B00097FDA095BA2F04C0AA2797FDA095BA2F80
:10C7C000280F391F4A1F5B1F2093FB023093FC0286
:10C7D0004093FD025093FE028091FB029091FC0277
:10C7E000A091FD02B091FE0281509A4FA040B0404E
:10C7F00064F080E09AEFA0E0B0E08093FB029093B9
:10C80000FC02A093FD02B093FE028091FB02909186
:10C81000FC02A091FD02B091FE0280509640AF4F05
:10C82000BF4F64F480E096E0AFEFBFEF8093FB0270
:10C830009093FC02A093FD02B093FE02C0906506A7
:10C84000209104083091050878E0E72EEC1498F068
:10C850008C2D9927829FA001839F500D929F500D90
:10C860001124CA0157FD07967C0163E0F594E79413
:10C870006A95E1F712C08C2D86959927829FB001A9
:10C88000839F700D929F700D1124CB0177FD03964D
:10C890007C01F594E794F594E794A0907B01B09027
:10C8A0007C019501442737FD4095542F8091FB0270
:10C8B0009091FC02A091FD02B091FE02BC01CD015D
:10C8C0000E94978BE20EF31E90906701692D7727E7
:10C8D00088279927980117FF04C022273327201B98
:10C8E000310B37FF02C02F5F3F4F35952795A98148
:10C8F000BA812A0F3B1F442737FD4095542F0E94D1
:10C90000238B97FF04C0615C7F4F8F4F9F4F26E0C2
:10C9100095958795779567952A95D1F79B016E1523
:10C920007F050CF47B01309521953F4FE216F3060D
:10C930000CF479018091E6079091E7076091E70296
:10C940007091E802861B970B9093E5078093E407AC
:10C950002091F7023091F8024091F9025091FA02C9
:10C96000DD2041F0461A570AC201AA2797FDA0957B
:10C97000BA2F04C0AA2797FDA095BA2F280F391FF8
:10C980004A1F5B1F2093F7023093F8024093F9028D
:10C990005093FA028091F7029091F802A091F90267
:10C9A000B091FA0281509A4FA040B04064F080E00C
:10C9B0009AEFA0E0B0E08093F7029093F802A09382
:10C9C000F902B093FA028091F7029091F802A091D7
:10C9D000F902B091FA0280509640AF4FBF4F64F415
:10C9E00080E096E0AFEFBFEF8093F7029093F802FC
:10C9F000A093F902B093FA022091E4073091E50781
:10CA000048E04C1598F08C2D9927829FB001839FA8
:10CA1000700D929F700D1124CB0177FD07966C016C
:10CA2000B3E0D594C794BA95E1F712C0C6948C2DA3
:10CA30009927829FD001839FB00D929FB00D112442
:10CA4000CD01B7FD03966C01D594C794D594C794D6
:10CA50009501442737FD4095542F8091F70290911E
:10CA6000F802A091F902B091FA02BC01CD010E9436
:10CA7000978BC20ED31E692D772788279927980197
:10CA800017FF04C022273327201B310B37FF02C0BA
:10CA90002F5F3F4F35952795E981FA812E0F3F1F74
:10CAA000442737FD4095542F0E94238B97FF04C0E5
:10CAB000615C7F4F8F4F9F4FE6E095958795779507
:10CAC0006795EA95D1F79B016C157D050CF46B0118
:10CAD000309521953F4FC216D3060CF46901809121
:10CAE000FB07282E33245090A60664E1862E67E0CB
:10CAF000962E5BECA52E56E0B52E4BE0442E35E18C
:10CB0000632E38E0732ED5012C9112160CF029C13A
:10CB1000203429F4E981FA81FF8BEE8B1FC0498113
:10CB20005A81CA01AA2797FDA095BA2F332727FD5E
:10CB30003095432F532FBC01CD010E94238B97FFCB
:10CB400004C0615C7F4F8F4F9F4F26E0959587957E
:10CB5000779567952A95D1F77F8B6E8BF5012181AB
:10CB6000203439F42E893F892E0D3F1D3F8B2E8BAB
:10CB70002AC0203C39F44E895F894E195F095F8BCA
:10CB80004E8B21C0C701AA2797FDA095BA2F332746
:10CB900027FD3095432F532FBC01CD010E94238BDD
:10CBA00097FF04C0615C7F4F8F4F9F4FB6E0959514
:10CBB000879577956795BA95D1F7AE89BF89A60F06
:10CBC000B71FBF8BAE8BF5012281203439F42E893B
:10CBD0003F892C0D3D1D3F8B2E8B2AC0203C39F404
:10CBE0004E895F894C195D095F8B4E8B21C0C60150
:10CBF000AA2797FDA095BA2F332727FD3095432FFD
:10CC0000532FBC01CD010E94238B97FF04C0615CB0
:10CC10007F4F8F4F9F4FA6E09595879577956795A6
:10CC2000AA95D1F7AE89BF89A60FB71FBF8BAE8B70
:10CC3000F5012381203439F42E893F89200F311FDB
:10CC40003F8B2E8B2AC0203C39F44E895F89401BD4
:10CC5000510B5F8B4E8B21C0C801AA2797FDA09571
:10CC6000BA2F332727FD3095432F532FBC01CD0119
:10CC70000E94238B97FF04C0615C7F4F8F4F9F4FB3
:10CC8000F6E09595879577956795FA95D1F7AE89F2
:10CC9000BF89A60FB71FBF8BAE8BF3018081918137
:10CCA0002E893F898217930764F4B901680F791FB1
:10CCB00077FF02C06F5F7F4F759567957F8B6E8B97
:10CCC0001DC0552049F44E895F89440F551F481BEC
:10CCD000590B5F8B4E8B12C051E0551578F4252D02
:10CCE00033276E897F89861B970BB9010E94628B5F
:10CCF000AE89BF89A60FB71FBF8BAE8BC101880F4E
:10CD0000991F880F991FEE89FF898E179F0764F47A
:10CD1000FD898F2F9927880F991F880F991F2E89BA
:10CD20003F892817390714F09F8B8E8B8E899F8936
:10CD300097FD03969595879595958795F401818341
:10CD4000880F991F880F991F2E893F89281B390B3F
:10CD5000C901880F8283EE89FF89D301ED93FC938B
:10CD600003C0F401118212824A9422E030E0620E84
:10CD7000731E44E050E0A40EB51E68E070E0860E1D
:10CD8000971E47FEC0CEE2E1C95E0C94CE8B84B103
:10CD9000806A84B93D9A82E58CBD1DBC459A81E0CC
:10CDA000809348088AEA8093590883E880935A0858
:10CDB0008AE080935B0810925D0810925C081092E4
:10CDC0005F0810925E081092C10810927D080895C5
:10CDD00030914808332309F085C00DB407FE82C0A6
:10CDE00084E08093D901459A2EB58091B6039927A6
:10CDF0008130910589F0823091051CF4892B21F056
:10CE00003EC00297B9F03BC030937C082093B70333
:10CE10002138A9F581E008C0253549F48091B70390
:10CE2000820F8093B70382E08093B60328C03093CB
:10CE3000B60325C080917C08E82FFF27E256F74F04
:10CE400020838F5F80937C089091B7038032A0F09D
:10CE5000291769F480E2AEE9B8E0EEE7F8E00D905A
:10CE600001928A95E1F781E080937D0802C03093BA
:10CE70007D081092B60303C0920F9093B7032091E0
:10CE80005808223208F028C0459800000000000031
:10CE90000000000000000000000000000000000092
:10CEA0000000000000000000000000000000000082
:10CEB00000000000000000000000E0915108F09127
:10CEC0005208E20FF11D80818EBD80917A08908119
:10CED000890F80937A0803C081E0809348082F5F10
:10CEE000209358080895EF92FF920F931F9380911B
:10CEF0005E069927880F991F880F991F7C010027CC
:10CF0000F7FC0095102F8091330390913403A0918A
:10CF10003503B0913603BC01CD01A80197010E94F1
:10CF2000978B30935D0820935C0880912B03909140
:10CF30002C03A0912D03B0912E03BC01CD01A801BB
:10CF400097010E94978B30935F0820935E08209191
:10CF50003E0830913F084091400850914108DA0165
:10CF6000C90163E0880F991FAA1FBB1F6A95D1F7FB
:10CF7000820F931FA41FB51F820F931FA41FB51FFD
:10CF8000209142013091430140914401509145016B
:10CF9000BC01CD010E94978B3093650820936408F3
:10CFA00080914403909145032091F8013091F9015B
:10CFB000821B930B90936B0880936A08E0913A036D
:10CFC000F0913B0380910B0890910C08BF010E94E7
:10CFD000628B9B01220F331F220F331F260F371F37
:10CFE000260F371F37FF02C02D5F3F4F359527951E
:10CFF00035952795309361082093600880913A0811
:10D0000090913B08BF010E94628B9B01220F331F4E
:10D01000220F331F260F371F260F371F37FF02C07F
:10D020002D5F3F4F359527953595279530936308AC
:10D030002093620810923B0310923A0310920C085E
:10D0400010920B0810923B0810923A0880915B08EE
:10D0500099278D30910509F48CC08E3091055CF4D0
:10D060008B30910509F4B4C08C3091050CF035C1BA
:10D070000A9761F0E7C18F30910509F4B3C18F3091
:10D0800091050CF480C14097A9F1DCC18091B602F2
:10D0900080936E088091B50280936F088091B402EE
:10D0A000809370088091B302809371088091B202DE
:10D0B000809372088091B102809373088091B002CE
:10D0C000809374088091AF02809375088091A102CB
:10D0D000809376088091A102837F8093A1020E94B1
:10D0E0006D2F809377088091A706809378088091B0
:10D0F000A002A6C18091CE089091CF0890936F08AE
:10D1000080936E088091D2089091D3089093710813
:10D110008093700880911D0190911E018093720888
:10D12000809100018093730880914101809374087D
:10D130009091B80390937508E92FFF27A3E0EE0FB5
:10D14000FF1FAA95E1F7EC5EF84F86818093760881
:10D150008381809377088781809378088581809385
:10D160007908892F8F5F6CE00E94428B9093B803FF
:10D1700069C18091920680936E0880919306809396
:10D180006F08809194068093700880919506809333
:10D190007108809196068093720880919A06809318
:10D1A000730880919B068093740880919C068093FD
:10D1B000750880919F068093760880919D068093E4
:10D1C000770880919E06809378088091A00638C1E8
:10D1D000F89480914506E82FFF27EE0FFF1FEB58CC
:10D1E000F84F0190F081E02DE038F1051CF0EFE7F9
:10D1F000F0E006C02FEFE138F20714F4E1E8FFEFAA
:10D20000E0936E0880914606E82FFF27EE0FFF1F80
:10D21000EB58F84F0190F081E02DE038F1051CF05B
:10D22000EFE7F0E006C06FEFE138F60714F4E1E84D
:10D23000FFEFE0936F0880914406E82FFF27EE0F81
:10D24000FF1FEB58F84F0190F081E02DE038F10519
:10D250001CF0EFE7F0E006C08FEFE138F80714F4B8
:10D26000E1E8FFEFE093700880914306E82FFF2785
:10D27000EE0FFF1FEB58F84F0190F081E02DE038E2
:10D28000F1051CF0EFE7F0E006C02FEFE138F20700
:10D2900014F4E1E8FFEF7894E09371088091DA02EA
:10D2A000809372088091DB02809373088091DC0286
:10D2B000809374088091DD02809375088091DE026E
:10D2C000809376088091DF02809377088091E00256
:10D2D000809378088091E102B3C080913004863059
:10D2E00018F01092300485E080936E088091A106BA
:10D2F00080936F088091D3029091D402A091D502BF
:10D30000B091D602BC01CD0125E030E040E050E014
:10D310000E94978B30937108209370088091CF0200
:10D320009091D002A091D102B091D202BC01CD0166
:10D3300025E030E040E050E00E94978B3093730886
:10D3400020937208809197068093740880919806C4
:10D350008093750880919906809376088091D90210
:10D36000809377088091750790917607809378086D
:10D370008091AF059091B00597FD0396959587959F
:10D38000959587955DC010926E0888E580936F082B
:10D3900084E0809370088FE180937108809101018F
:10D3A000809372088091150480937308809116040D
:10D3B00080937408109215048071809316048091F4
:10D3C00017048093750880912E08809376088091C9
:10D3D0001208809377088091A30680937808809143
:10D3E000B0062EC08091770680936E088091AE06BD
:10D3F00080936F0880916D01809370088091700612
:10D4000080937108809171068093720880917206F2
:10D410008093730880916C018093740880917406E6
:10D4200080937508809175068093760880917606C2
:10D43000809377088091D408809378088091D905EB
:10D440008093790880917D08882309F455C18AEF7B
:10D4500080939B0181E080938D0140917F085091E2
:10D460008008CA0181509E4F8F5F9340B0F4209195
:10D47000810830918208C90181509E4F8F5F93408F
:10D4800060F480914F0685FF08C05093A503409338
:10D49000A4033093A3032093A20380918508909165
:10D4A000860821E08936920724F490938F018093B7
:10D4B0008E0120918F08309190088091DA0190912F
:10D4C000DB018217930740F48091AE01882321F499
:10D4D0003093DB012093DA0180917E089927893609
:10D4E000910509F4A5C08A36910544F48736910563
:10D4F00071F08836910509F462C006C18A3691053B
:10D5000009F4F3C08B36910509F4E2C0FDC08091A7
:10D5100091088093BE08809192088093C008809102
:10D5200093088093BF088091940880938C01809128
:10D5300095088093C2088091960880939C01809101
:10D5400097088093B503809198088093A1038091F8
:10D55000AE028823F9F02091990830919A0837FD9E
:10D5600019C03093F2022093F10290917906992329
:10D5700089F08FE0989FC0011124281B390BC90145
:10D5800088599E4F68E671E00E94628B9093F20288
:10D590008093F1022091AC033091AD0380919B0800
:10D5A00090919C08280F391F37FF02C02F5F3F4F13
:10D5B000359527953093AD032093AC03A5C080919A
:10D5C0009108809353088091920880935408809129
:10D5D0009308809355088091940880935608809111
:10D5E00095088093570880919F0590919608892B04
:10D5F00080939F059091A0059370809197088C70FF
:10D60000982B9093A005809198088093B303809104
:10D6100099088093910180919A088093C108809124
:10D620009B088093AF0380919C088093AE036CC0ED
:10D6300080919108809349088091920880934A08CC
:10D640008091930880934B088091940880934C08B4
:10D65000809195089091960890934E0880934D087C
:10D6600080919708909198089093500880934F0864
:10D6700080919908992787FD90959093A8078093AA
:10D68000A70780919A088093C80280919B08909187
:10D690009C089C01442737FD4095542FDA01C901AD
:10D6A00063E0880F991FAA1FBB1F6A95D1F7820FED
:10D6B000931FA41FB51F820F931FA41FB51F809334
:10D6C000C9029093CA02A093CB02B093CC021CC0B3
:10D6D000809191088093B203809192088093B10366
:10D6E000809193088093B0030FC0809169068630C3
:10D6F00059F40E944A7108C01092A5031092A40325
:10D700001092A3031092A2031F910F91FF90EF902C
:10D71000089580914808882309F43BC0459889E51D
:10D7200098E090935208809351089091B403E92FA8
:10D73000FF27EE56FE4F9F5F9093B4038081809346
:10D740005B08993010F01092B403109248080E94C0
:10D75000736781E08093580800000000000000001B
:10D7600000000000000000000000000000000000B9
:10D7700000000000000000000000000000000000A9
:10D7800000000000000000008091590880937A0892
:10D790008EBD089587B18C6087B9429843981092E6
:10D7A000BA0380E880939E011092B90380939D0193
:10D7B00008958091BF0381508093BF038F3F09F08C
:10D7C00019C189E08093BF038091A10299278073DA
:10D7D0009070892B21F48091160480FF1DC08091E8
:10D7E0009006882351F08091C203882319F484E0C5
:10D7F0008093BA0381E08093C203809191068823CD
:10D80000B9F08091C303882319F484E08093B903AD
:10D8100081E08093C3030CC01092C2031092C30333
:10D8200080918C068093C00380918E068093C10303
:10D830008091C203882309F045C08091AD06282F4E
:10D84000332724FF07C08091D802882319F425FDCF
:10D8500052C053C090918D06983F48F080910D08BA
:10D860008D3D28F08091C00388236CF00AC0983F5A
:10D8700078F080910D08853059F48091C00387FFBE
:10D8800002C0429801C0429A81E080939E0136C056
:10D890008091BA0381508093BA038F3F79F58091CC
:10D8A0000D0886958093BA0380919E01813011F412
:10D8B00080E801C0869580939E0180919E019091A1
:10D8C000C00317C08091BA0381508093BA038F3F81
:10D8D000A9F489E08093BA0380919E01813011F40C
:10D8E00080E801C0869580939E0180919E01909171
:10D8F0009006892311F0429A01C042988091C30397
:10D90000882309F043C09091AD0697FF07C080912E
:10D91000D802882319F496FD52C053C090918F0607
:10D92000983F48F0809135088D3D28F08091C103E3
:10D9300088236CF00AC0983F78F0809135088530D4
:10D9400059F48091C10387FF02C0439801C0439AF4
:10D9500081E080939D0136C08091B903815080930E
:10D96000B9038F3F79F58091350886958093B90387
:10D9700080919D01813011F480E801C086958093EB
:10D980009D0180919D019091C10317C08091B903C1
:10D9900081508093B9038F3FA9F489E08093B90344
:10D9A00080919D01813011F480E801C086958093BB
:10D9B0009D0180919D0190919106892311F0439AD8
:10D9C00001C04398429B04C08091A002886003C0BC
:10D9D0008091A002877F8093A002439B06C0809124
:10D9E000A00280618093A00208958091A0028F7EA2
:10D9F0008093A00208954FB724E130E0F89480911D
:10DA0000C9008F778093C9008091C9008F7B809374
:10DA1000C9008091C9008F7D8093C9005A9A52989D
:10DA20005B9A539A832F99278093CD002093CC0043
:10DA30008091C80082608093C80080E18093C90013
:10DA40008091CA008F778093CA008091CA008F7B33
:10DA50008093CA008091CA008F7D8093CA00809114
:10DA6000CA008F7E8093CA008091CA00877F80930E
:10DA7000CA008091C9008B7F8093C9008091CA0041
:10DA800084608093CA008091CA0082608093CA003B
:10DA90008091C80087FF03C08091CE00F9CF8091AC
:10DAA000C90080688093C9004FBF0895A0E0B0E02E
:10DAB000ECE5FDE60C94BC8B482F00E010E0809173
:10DAC0009F01813061F410929F0184E48093C6032A
:10DAD0001092C8031092C7031092C90333C28091F9
:10DAE000C603882319F421E030E001C09801909129
:10DAF000C703992371F4232B11F081E010C084E453
:10DB00008093C6039093C8039093C7039093C9036F
:10DB100002C2913069F4232B09F0F3C182E08093B3
:10DB2000C7038091C8038F5F8093C80383E0F1C16E
:10DB30009230D1F4232B09F0E4C183E08093C60333
:10DB40004093C9039091C803923039F41092CA03EC
:10DB500047FF03C081E08093CA0383E08093C7033B
:10DB60009F5F9093C803D7C1933009F0CAC1232B9C
:10DB700009F0C7C19093C60382E08093C7038091E8
:10DB8000C8038F5F8093C8032091C903822F992710
:10DB9000782F6627842F9927682B792B8091690627
:10DBA000813051F47370CB018050924063E070E09B
:10DBB0000E94628BEB0119C0823069F47770CB014F
:10DBC0008050944066E070E00E94628BEB012695E5
:10DBD000269526950CC0EB01D370C856D140CE01D6
:10DBE000D7FD0196EC01D595C79526952695022F70
:10DBF00011270F7010700F5F1F4F0D30110508F0C7
:10DC000079C10230110519F404E010E005C00430B8
:10DC1000110511F402E010E06801C00ED11EF601FA
:10DC2000EB58F84F808191819E01281B390BC90167
:10DC300037FF03C0909581959F4F069704F5E091BB
:10DC4000AA06EE2351F0FF27EE0FFF1FEB58F84F07
:10DC5000808191818436910594F48091D902883C29
:10DC600030F48091D902865F8093D90208C088EC95
:10DC70008093D90280916F008F7D80936F00F601B1
:10DC8000EB58F84F808191819C01220F331F280FA0
:10DC9000391F2C0F3D1F37FF02C02D5F3F4F790109
:10DCA000F594E794F594E794CE0101968E159F05BF
:10DCB00024F40894E108F10808C0CE010197E816A1
:10DCC000F9061CF40894E11CF11C0630110509F05A
:10DCD000D1C0C536D1050CF4A8C09091C503E92F79
:10DCE000FF27ED53F74FE081ED3729F48091C4030E
:10DCF00080958093C403963061F48091C403882397
:10DD000011F0E338B9F0882309F08BC0ED3791F0BA
:10DD100088C0993009F085C08091C403882329F414
:10DD20008091CC08833831F07CC08091CC088D374D
:10DD300009F077C08091C4088D3739F48091C50807
:10DD40008338B1F483E89FEF0FC0833889F4809162
:10DD5000C508833829F41092800710927F0708C005
:10DD60008D3731F48DE790E09093800780937F07A3
:10DD70008091C608992787FD90959093820780939C
:10DD800081078091C708992787FD909590938C070C
:10DD900080938B078091C808992787FD9095909371
:10DDA0008E0780938D078091C5038930D1F58091CE
:10DDB000CA088D3749F480918507909186070596AA
:10DDC00090938607809385078091CB088D3749F41F
:10DDD0008091850790918607059790938607809399
:10DDE0008507809185079091860783589F4F1CF483
:10DDF00083E89FEF09C080918507909186078E3751
:10DE0000910534F08DE790E0909386078093850725
:10DE10008091C908992787FD909590938A078093F0
:10DE200089071092C5031092C403CA30D1055CF46F
:10DE30008091C5038F5F8093C503E82FFF27ED53C3
:10DE4000F74F83E880838091C5038A3011F41092E4
:10DE5000C5038FEFCC39D8076CF48091C503E82F48
:10DE6000FF27ED53F74F8DE780838091C4038095A2
:10DE70008093C4038091D902843BD0F0F601EB5823
:10DE8000F84F80819181F701E81BF90BCF0163E026
:10DE900070E00E94628BCB01880F991F860F971F3D
:10DEA00029EA37E0C20ED31EF6019183808307C0B2
:10DEB00029EA37E0C20ED31EF60111821082053026
:10DEC000110540F4000F111F0B58184FF801F18293
:10DED000E08221C00530110529F4D0938407C09356
:10DEE000830719C007301105B1F4D0938807C09398
:10DEF000870711C00231110570F081E080939F0106
:10DF00000AC081E080939F011092C8031092CA0357
:10DF100084E48093C6038091C803803198F0809197
:10DF2000CA03882331F480919F01882311F48093E0
:10DF300040011092C8031092CA031092C70384E4F0
:10DF40008093C603E8E0CDB7DEB70C94D88BCF93AF
:10DF5000FC0197FF05C0CFEFF095E195FF4F01C0A1
:10DF6000C1E028E631E0CF01B9010E94628BFC01DB
:10DF70008B35910554F08B5590408A35910538F4D6
:10DF800084EB90E08E1B9F0BFC0141E00DC0CF01A4
:10DF9000855B90408A35910518F4E45BF04003C03E
:10DFA0002E1B3F0BF9014FEFEE0FFF1FEB5CF64FFF
:10DFB000259134918C2F992787FD9095289FB0014A
:10DFC000299F700D389F700D1124842F992787FD8C
:10DFD0009095689FA001699F500D789F500D112466
:10DFE000CA01CF9108952AE530E0281B390BC901F9
:10DFF0000E94A76F089508950895089508950895BB
:10E0000080E090E008951092CF081092CE08109210
:10E01000D3081092D2081092D1081092D008109212
:10E02000D4088AE090E00E94CE189093CC038093AD
:10E03000CB030895CF93DF938091CB039091CC03D2
:10E040000E94D718882309F4AFC08091CB03909128
:10E05000CC030A969093CC038093CB03E0E0F0E0EE
:10E060009F0190E05FEFA4E1B7E04BE0ED018B8111
:10E0700087FF0BC09F5F8D81E80FF11D8981280FFD
:10E08000311D8E81851708F4582F4150189647FF8F
:10E09000EDCF5093D408232B41F52091D10330913B
:10E0A000D2034091D3035091D403BB27A52F942FC3
:10E0B000832F9093D0038093CF03AA27BB27281BDD
:10E0C000390B4A0B5B0BCF01AA27BB27280F391F3F
:10E0D0004A1F5B1F2093D1033093D2034093D30395
:10E0E0005093D403E5E0F0E013C02091CF033091CA
:10E0F000D0032E173F0718F4E21BF30B02C0E0E039
:10E10000F0E0892F9927880F991FE80FF91F35969E
:10E11000F093CF08E093CE08EF3FF10578F48091BB
:10E120001D0190911E018E9F90018F9F300D9E9F2B
:10E13000300D1124C90164E670E013C0CF0196953B
:10E1400087959695879520911D0130911E01289FF6
:10E15000A001299F500D389F500D1124CA0169E17B
:10E1600070E00E944E8B7093D1086093D00820918C
:10E17000CD033091CE032E0F3F1F3093CE0320935B
:10E18000CD035EE02131350778F08091D20890917F
:10E19000D30801969093D3088093D20820513E4033
:10E1A0003093CE032093CD03DF91CF91089530912A
:10E1B000DA03E32FFF2783E0EE0FFF1F8A95E1F7D5
:10E1C000EC5EF84F2781422F552747FD50958091EF
:10E1D000DB039927841795072CF42093DB033093F6
:10E1E000DD030AC0222341F08091DC039927481700
:10E1F000590714F42093DC03832F8F5F8093DA0395
:10E200008D30D0F01092DA038091DC038F3F19F04B
:10E210008093D60302C01092D6038091DB038093D3
:10E22000D7038091DD038093D5038FEF8093DC03C8
:10E230001092DB031092DD03089595E1899F802DF4
:10E2400011240E94818589EE9BE09F938F9383E543
:10E2500095E89F938F93E091FC03F091FD0309955E
:10E260000F900F900F900F9008958091A10285FF5D
:10E2700003C080E190E008958091D802882339F0AE
:10E280008091B303882319F085E090E0089580E041
:10E2900090E0089540E050E030E080919C0899279C
:10E2A0008A38910591F08B38910524F489389105CD
:10E2B00041F016C08D38910581F08E38910549F0F6
:10E2C0000FC04DE159E031E10BC04AED59E03DE1AD
:10E2D00007C045ED58E036E203C04BEF58E032E2AC
:10E2E0009091910820E080919208281770F493177C
:10E2F00060F4DA01A90FB11DE22FFF27E258F74FB2
:10E3000085898C939F5F2F5FEECF089520E335E7DB
:10E31000809141018B3211F08D32F9F480915406D5
:10E32000282F33278091CD029091CE02829FA001A9
:10E33000839F500D929F500D1124CA0163E070E03D
:10E340000E94628BCB019B01205D3A48C196C19728
:10E3500008F03FC02EEF34E73CC0803229F58091B1
:10E36000A10281FF36C02091D8033091D903205DEE
:10E370003A4855E72133350748F085E7243938070F
:10E3800018F420E335E702C02456304045E7203337
:10E390003407F8F454E72D3C350718F020E335E74F
:10E3A00018C02C593F4F15C08E3549F49091C802C2
:10E3B0008AE0989F90011124205D3A480AC0863770
:10E3C00041F49091C8028AE0989FC0011124281B53
:10E3D000390BC9010895EF92FF920F931F9399276C
:10E3E0008A38910509F45DC08B38910524F4893889
:10E3F000910551F0D2C18D38910509F416C18E38BE
:10E40000910509F483C0C9C18091D3029091D402CF
:10E41000A091D502B091D602BC01CD0124E630E036
:10E4200040E050E00E94978BDA01C9018C509E4F6A
:10E4300090932109809320090E9486719093270967
:10E4400080932609909329098093280990932B099A
:10E4500080932A0920912009309121098091240973
:10E46000909125092817390724F430932509209322
:10E47000240980912209909123098217930724F49B
:10E4800030932309209322090E94357180931F093C
:10E490008DE199E09093EC038093EB0381E190E0B0
:10E4A0007EC18091D3029091D402A091D502B09107
:10E4B000D602BC01CD0124E630E040E050E00E94ED
:10E4C000978BDA01C9018C509E4F9093ED09809390
:10E4D000EC090E9486719093EF098093EE0988E71A
:10E4E00090E09093F1098093F0091092F309109253
:10E4F000F2090E9435718093DC098AED99E09093CE
:10E50000EC038093EB038DE190E049C10E94D7704A
:10E510008091D3029091D402A091D502B091D602FD
:10E52000BC01CD0124E630E040E050E00E94978B32
:10E53000DA01C9018C509E4F9093ED088093EC084E
:10E5400080911D0190911E019093E7088093E60849
:10E5500080911D0190911E019093E9088093E80835
:10E560008091EB079091EC0797FD01969595879523
:10E570008093D8088093DF0820914F08309150088D
:10E5800037FF02C02F5F3F4F359527952093DD0859
:10E5900080914D0890914E0864E170E00E944E8B8E
:10E5A0006093DE082093E4086093E5080E9486717A
:10E5B0009093F5088093F40888E790E09093F7082B
:10E5C0008093F60880911D0190911E019093F108AF
:10E5D0008093F0088091D6038C5E8093EA08809146
:10E5E000D7038C5E8093EB088091D2089091D3087A
:10E5F0006AE070E00E944E8B7093F3086093F2081B
:10E600000E9435718093D7088091CE089091CF08F1
:10E610009093EF088093EE0885ED98E09093EC03DB
:10E620008093EB0386E290E0BAC00E94D77080919D
:10E630004D0890914E0864E670E00E944E8B7093F6
:10E640000E0960930D098091EB079091EC0797FDFF
:10E650000196959587958093FE0880914F0890913B
:10E66000500897FD019695958795809303098091B1
:10E670000001482F55279A012B5F3F4F80911D01C4
:10E6800090911E012817390784F480911D01909103
:10E690001E01841B950B9C01220F331F280F391F6D
:10E6A000822F825180930A0902C010920A09E090D9
:10E6B000D302F090D4020091D5021091D602C80185
:10E6C000B70124E630E040E050E00E94978B3093A1
:10E6D0000C0920930B0937FF04C010920C0910920B
:10E6E0000B09C801B70124E630E040E050E00E9489
:10E6F000978BDA01C9018C509E4F9093100980933B
:10E700000F0980911D0190911E019093050980933E
:10E71000040980911D0190911E0190930709809337
:10E7200006090E948671909312098093110988E767
:10E730008093130980911D0190911E0190931709F8
:10E74000809316098091D6038C5E8093080980918E
:10E75000D7038C5E809309098091D2089091D308E9
:10E760006AE070E00E944E8B70931909609318095B
:10E770000E9435718093FD088091CE089091CF085A
:10E7800090931509809314098BEF98E09093EC0314
:10E790008093EB0382E290E002C080E090E01F9162
:10E7A0000F91FF90EF900895EF92FF920F931F93B8
:10E7B000CF93DF938091D8039091D9039C0103E01C
:10E7C000220F331F0A95E1F7281B390B8091EB01CB
:10E7D0009091EC01280F391F37FF02C0295F3F4F8E
:10E7E00013E0359527951A95E1F73093D9032093D7
:10E7F000D8039091DF03992309F011C38091DE03C0
:10E80000282F3327442755278F5F8093DE03F90194
:10E810002131310508F000C3E058FF4F0C94E98B1B
:10E820008091A10285FF2AC080E00E9481858091AD
:10E830001D0190911E016AE070E00E94628B9F931F
:10E840008F9380911D0190911E016AE070E00E94FB
:10E85000628B7F936F938FEF9BE09F938F9384E7FF
:10E8600095E89F938F93E091FC03F091FD03099548
:10E870002DB73EB7285F3F4F2DBF28C080E00E94D4
:10E88000818580911D0190911E016AE070E00E94D7
:10E89000628B9F938F9380911D0190911E016AE07E
:10E8A00070E00E94628B7F936F938CE09CE09F935B
:10E8B0008F9383E595E89F938F93E091FC03F0910C
:10E8C000FD0309958DB79EB708968DBF80912E08E0
:10E8D00080FF39C08091F0028823E9F08AE00E942D
:10E8E00081858091410199279F938F938091D302D5
:10E8F0009091D402A091D502B091D602BC01CD0175
:10E9000024E630E040E050E00E94978B3F932F9345
:10E9100089E19CE084C68AE00E9481858091D302CF
:10E920009091D402A091D502B091D602BC01CD0144
:10E9300024E630E040E050E00E94978B3F932F9315
:10E9400085E29CE098C78AE00E94818580E39CE094
:10E9500017C68091A10285FF2AC085E10E948185AA
:10E960008091A8019091A9016CE370E00E944E8B08
:10E970009F938F938091A8019091A9016CE370E01F
:10E980000E944E8B7F936F938AE39CE09F938F93BB
:10E9900084E795E89F938F93E091FC03F091FD034A
:10E9A00009952DB73EB7285F3F4F2DBF28C085E1A1
:10E9B0000E9481858091A8019091A9016CE370E08B
:10E9C0000E944E8B9F938F938091A8019091A901F3
:10E9D0006CE370E00E944E8B7F936F9387E49CE022
:10E9E0009F938F9383E595E89F938F93E091FC032A
:10E9F000F091FD0309958DB79EB708968DBF8FE105
:10EA00000E94818580E690E09F938F938091EB0731
:10EA10009091EC079F938F9384E59CE09F938F9355
:10EA2000C3E5D5E8DF93CF93E091FC03F091FD03BC
:10EA300009958091A0022DB73EB7285F3F4F2DBFAB
:10EA400080FF06C089E20E9481858FE59CE069C352
:10EA500089E20E94818581E69CE0A9C68091A1029D
:10EA600085FF1BC08AE20E9481858091D208909127
:10EA7000D3089F938F9383E69CE09F938F9384E7C3
:10EA800095E89F938F93E091FC03F091FD03099526
:10EA90008DB79EB706968DBF1BC08AE20E94818506
:10EAA0008091D2089091D3089F938F938BE69CE03E
:10EAB0009F938F9383E595E89F938F93E091FC0359
:10EAC000F091FD0309952DB73EB72A5F3F4F2DBF4B
:10EAD00086E30E9481858091CE089091CF086AE0FC
:10EAE00070E00E944E8B9F938F938091CE089091FF
:10EAF000CF086AE070E00E944E8B7F936F9383E7AC
:10EB00009CE09F938F9383E595E89F938F93E0918B
:10EB1000FC03F091FD0309958DB79EB70896B9C621
:10EB200089E00E9481858FE79CE09F938F9303E5A6
:10EB300015E81F930F93E091FC03F091FD030995F5
:10EB40008EE10E9481850F900F900F900F9081E8C9
:10EB50009CE09F938F931F930F93E091FC03F091A0
:10EB6000FD03099583E30E9481850F900F900F901C
:10EB70000F9083E89CE09F938F931F930F93E091F6
:10EB8000FC03F091FD0309958FE30E9481850F90AE
:10EB90000F900F900F9085E89CE09F938F931F93A9
:10EBA0000F93E091FC03F091FD0309958EE70E941D
:10EBB00081850F900F900F900F908BE99CE09F93B1
:10EBC0008F931F930F938AC780919B01882309F429
:10EBD00062C08DE50E94818581EB9CE09F938F93BD
:10EBE000C3E5D5E8DF93CF93E091FC03F091FD03FB
:10EBF000099584E50E9481850F900F900F900F90EA
:10EC000080914A0899279F938F9383EB9CE09F9371
:10EC10008F93DF93CF93E091FC03F091FD0309956F
:10EC20008EE50E9481852DB73EB72A5F3F4F2DBFED
:10EC300080914D0890914E086AE070E00E944E8BE2
:10EC40007F936F938CEB9CE09F938F93DF93CF9395
:10EC5000E091FC03F091FD0309958DB79EB70696F0
:10EC60008DBF80914B08833081F48091490881FFEA
:10EC700006C08BE50E94818586EC9CE098C58BE5FB
:10EC80000E94818589EC9CE092C58BE50E9481857C
:10EC90008CEC9CE01DC784E0CDC380919B01882350
:10ECA00009F47AC08091E103C3E5EC2EC5E8FC2E9F
:10ECB000882309F44BC089E60E9481858091B203C4
:10ECC00099279F938F938FEC9CE09F938F93FF9254
:10ECD000EF92E091FC03F091FD03099585E70E9416
:10ECE00081852DB73EB72A5F3F4F2DBF809191019F
:10ECF00099279F938F9300E610E01F930F938091C5
:10ED00004F08909150089F938F938AED9CE09F93BA
:10ED10008F93FF92EF92E091FC03F091FD03099530
:10ED200082E70E9481858DB79EB70A968DBF80913C
:10ED3000B00399279F938F931F930F938091B103F3
:10ED400099279F938F9386EE9CE063C689E60E9485
:10ED500081858091910199279F938F9380E690E020
:10ED60009F938F9380914F08909150089F938F931A
:10ED700080914C0899279F938F9386EF9CE09F93F7
:10ED80008F93FF92EF92E091FC03F091FD030995C0
:10ED90008DB79EB70C967DC585E04CC39091B303AB
:10EDA0009923D1F08091E803882381F09E3170F49B
:10EDB00087E00E941D7183E90E9481858091B303E1
:10EDC00099279F938F938FE09DE09EC383E90E94D4
:10EDD00081858AE19DE0ADC383E90E94818580E25F
:10EDE0009DE0CEC30E943571809330098091100A56
:10EDF000863059F48091E103882319F01092E103E1
:10EE000099C681E08093E10395C6883009F092C6E7
:10EE10000E94868581E0D5C39093DE0393C691302E
:10EE200009F0DAC38091DE03282F332744275527C2
:10EE30008F5F8093DE03F9012131310508F07DC633
:10EE4000EF56FF4F0C94E98B8091A10285FF43C0E0
:10EE500080E00E9481858091D2089091D3089F9391
:10EE60008F9380911D0190911E016AE070E00E94D5
:10EE7000628B9F938F9380911D0190911E016AE098
:10EE800070E00E94628B7F936F938091A8019091B4
:10EE9000A9016CE370E00E944E8B9F938F93809149
:10EEA000A8019091A9016CE370E00E944E8B7F93C2
:10EEB0006F9386E39DE09F938F9384E795E89F93FC
:10EEC0008F93E091FC03F091FD0309952DB73EB7B8
:10EED000225F3F4FABC580E00E9481858091D208C0
:10EEE0009091D3089F938F9380911D0190911E0163
:10EEF0006AE070E00E94628B9F938F9380911D0166
:10EF000090911E016AE070E00E94628B7F936F9384
:10EF10008091A8019091A9016CE370E00E944E8B52
:10EF20009F938F938091A8019091A9016CE370E069
:10EF30000E944E8B7F936F9381E59DE0C6C285E171
:10EF40000E94818580E690E09F938F9380918E014F
:10EF500090918F019F938F938CE69DE09F938F9369
:10EF6000C3E5D5E8DF93CF93E091FC03F091FD0377
:10EF7000099580912E082DB73EB7285F3F4F2DBFD2
:10EF800080FF51C08091F002882339F18FE10E9407
:10EF900081858091D3029091D402A091D502B09145
:10EFA000D602BC01CD0124E630E040E050E00E94F2
:10EFB000978B3F932F9386E79DE09F938F9383E6F4
:10EFC00095E89F938F93E091FC03F091FD030995E1
:10EFD0008DB79EB706968DBF38C08FE10E948185A0
:10EFE0008091D3029091D402A091D502B091D60223
:10EFF000BC01CD0124E630E040E050E00E94978B58
:10F000003F932F938FE79DE09F938F93DF93CF9351
:10F01000E091FC03F091FD0309952DB73EB72A5FFF
:10F020003F4F2DBF12C08FE10E94818588E89DE08F
:10F030009F938F93DF93CF93E091FC03F091FD03B7
:10F0400009950F900F900F900F9089E20E94818593
:10F050008091410199279F938F9382E99DE09F932F
:10F060008F93DF93CF930DC480919B018823F9F098
:10F070008BE20E9481858091910199279F938F93C4
:10F0800080914D0890914E086AE070E00E944E8B8E
:10F090007F936F9380E690E09F938F9380914F08CA
:10F0A000909150089F938F9385E99DE05CC182E029
:10F0B000C1C18FE30E9481858091D0089091D108D1
:10F0C0009F938F938091CE089091CF086AE070E073
:10F0D0000E944E8B9F938F938091CE089091CF0882
:10F0E0006AE070E00E944E8B7F936F938CEA9DE004
:10F0F0009F938F93C3E5D5E8DF93CF93E091FC0313
:10F10000F091FD0309958091A0022DB73EB7265FCF
:10F110003F4F2DBF80FF0AC082E50E94818580ECB1
:10F120009DE09F938F9383E695E8D6C482E50E9485
:10F13000818583EC9DE03BC380919B01B3E5EB2E81
:10F14000B5E8FB2E882309F449C084E50E94818537
:10F1500080914A0899279F938F9380914C08992713
:10F160009F938F9386EC9DE09F938F93E701FF928F
:10F17000EF92E091FC03F091FD0309958DB79EB7E6
:10F1800008968DBF80914B08833051F484E60E942D
:10F19000818589ED9DE09F938F93FF92EF920BC045
:10F1A00084E60E9481858FED9DE09F938F9384E795
:10F1B00095E89F938F93E091FC03F091FD030995EF
:10F1C0000F900F900F900F908091490881FFBAC463
:10F1D00084E60E94818585EE9DE0E9C284E50E9477
:10F1E00081858BEE9DE09F938F93FF92EF9276C483
:10F1F0008091E003A3E5EA2EA5E8FA2E882309F41E
:10F2000050C089E60E948185809131076AE00E94A2
:10F21000428B892F99279F938F93809131070E946A
:10F22000428B99279F938F93809129070E94428B4D
:10F23000892F99279F938F93809129070E94428B52
:10F2400099279F938F93809121070E94428B892F4A
:10F2500099279F938F93809121070E94428B992732
:10F260009F938F93809119070E94428B892F992732
:10F270009F938F93809119070E94428B99279F93A8
:10F280008F9381E09EE09F938F93FF92EF92E091A6
:10F29000FC03F091FD0309952DB73EB72C5E3F4F5F
:10F2A000C5C389E60E94818580E690E09F938F9395
:10F2B00080913307992787FD90959F938F93809135
:10F2C0002B07992787FD90959F938F938091230714
:10F2D000992787FD90959F938F9380911B0799277E
:10F2E00087FD90959F938F938EE19EE09F938F93E0
:10F2F000FF92EF92E091FC03F091FD0309958DB729
:10F300009EB70E96C6C28091E00390914106882375
:10F3100009F48DC0943009F48CC09630A1F58EE7C5
:10F320000E948185809141076AE00E94428B892F6B
:10F3300099279F938F93809141070E94428B992731
:10F340009F938F93809139070E94428B892F992731
:10F350009F938F93809139070E94428B99279F93A7
:10F360008F9381E39EE09F938F9383E595E89F932E
:10F370008F93E091FC03F091FD0309952DB73EB703
:10F38000245F3F4F53C3973008F4DCC38EE70E94DD
:10F390008185809151076AE00E94428B892F9927CD
:10F3A0009F938F93809151070E94428B99279F933F
:10F3B0008F93809149070E94428B892F99279F93B1
:10F3C0008F93809149070E94428B99279F938F9337
:10F3D000809141070E94428B892F99279F938F9399
:10F3E000809141070E94428B99279F938F93809130
:10F3F00039070E94428B892F99279F938F93809181
:10F4000039070E94428B99279F938F9380E49EE057
:10F410009F938F9383E595E89F938F93E091FC03EF
:10F42000F091FD0309958DB79EB7449632C2943092
:10F4300021F486E00E941D7185C39630F1F48EE7B9
:10F440000E94818580E690E09F938F93809143078F
:10F45000992787FD90959F938F9380913B079927DC
:10F4600087FD90959F938F938DE59EE09F938F935B
:10F4700083E595E89F938F93D0C2973008F462C3D9
:10F480008EE70E94818580E690E09F938F93809124
:10F490005307992787FD90959F938F9380914B07F2
:10F4A000992787FD90959F938F9380914307992784
:10F4B00087FD90959F938F9380913B07992787FDB8
:10F4C00090959F938F9380E79EE09F938F9383E522
:10F4D00095E89F938F930ECF9091B303992309F4EE
:10F4E0004AC08091E8038823F9F09E31E8F487E070
:10F4F0000E941D7183E90E9481858091B303992741
:10F500009F938F9383E89EE09F938F9383E695E884
:10F510009F938F93E091FC03F091FD0309952DB724
:10F520003EB72A5F3F4F82C283E90E9481858EE801
:10F530009EE09F938F9303E515E81F930F93E0914F
:10F54000FC03F091FD0309951F921F929091B30364
:10F5500081E1989FC00111248551964F9F938F930D
:10F560001F930F93E091FC03F091FD0309958DB774
:10F570009EB70A968EC183E90E94818584E99EE048
:10F580009F938F9383E595E8A7C20E94357180937E
:10F5900030098091100A863079F48091E003882345
:10F5A00019F01092E00303C081E08093E00385E04E
:10F5B0000E941D7186E0B3C2883031F40E948685B6
:10F5C00082E08093DF03B4C2813009F0B3C20E94AD
:10F5D00086851092DF03ACC2923009F0B1C28091EF
:10F5E000DE03282F3327442755278F5F8093DE03C0
:10F5F000F9012131310508F0A0C2EE55FF4F0C94FE
:10F60000E98B80E00E94818581EB96E09F938F9348
:10F610000E946D2F99279F938F938AEA9EE09F9374
:10F620008F9383E695E89F938F93E091FC03F0918D
:10F63000FD0309952DB73EB7285F3F4FF7C185E120
:10F640000E9481858FEB96E09F938F9380910001BC
:10F650006AE00E94428B892F99279F938F93809114
:10F6600000010E94428B99279F938F9389EB9EE024
:10F670009F938F9383E595E89F938F93E091FC038D
:10F68000F091FD03099573CF8AE20E9481858AEC8F
:10F690009EE09F938F93C3E5D5E8DF93CF93E091EE
:10F6A000FC03F091FD03099580912E080F900F90B7
:10F6B0000F900F9080FF41C080914F06909179018B
:10F6C00081FD0BC0892F99279F938F938FEC9EE02C
:10F6D0009F938F93DF93CF931DCFE091FC03F09125
:10F6E000FD03933318F089ED9EE002C080EE9EE0AA
:10F6F0009F938F93DF93CF9309950F900F900F9067
:10F700000F9080911208E091FC03F091FD0390911D
:10F71000790180FF0BC0892F99279F938F9387EEE4
:10F720009EE09F938F93DF93CF93AFC0892F99274C
:10F730009F938F938DEE9EE0CFC083EF9EE037C006
:10F740008FE30E9481858CEF9EE09F938F93C3E5AA
:10F75000D5E8DF93CF93E091FC03F091FD03099589
:10F760000F900F900F900F908091A406882319F4AA
:10F7700080E09FE01CC08091AE02E091FC03F0911C
:10F78000FD03882319F089E09FE002C080E19FE03B
:10F790009F938F93DF93CF9309950F900F900F90C6
:10F7A0000F908091AF0686FFCDC187E19FE09F93C8
:10F7B0008F93DF93CF9392C184E50E9481858EE180
:10F7C0009FE09F938F93C3E5D5E8DF93CF93E091BC
:10F7D000FC03F091FD03099580912E080F900F9086
:10F7E0000F900F9085FD03C083E29FE011C08091D0
:10F7F0009206883F10F4E82F07C0EFEFF0E0E81B17
:10F80000F109E652FD4FE081E23358F48CE29FE0CB
:10F810009F938F93DF93CF93E091FC03F091FD03CF
:10F8200016C0E43B18F083E39FE0F2CF8091AF066F
:10F83000E091FC03F091FD0385FF03C08AE39FE0A4
:10F8400002C081E49FE09F938F93DF93CF9309954C
:10F850000F900F900F900F908091A806882309F4C5
:10F8600071C18EE50E9481858091A80699279F939A
:10F870008F9388E49FE09F938F9383E595E89F9310
:10F880008F93E091FC03F091FD0309958DB79EB72E
:10F8900006968DBF57C189E60E94818583E59FE06A
:10F8A0009F938F93C3E5D5E8DF93CF93E091FC035B
:10F8B000F091FD0309950F900F900F900F9080919C
:10F8C000A706E091FC03F091FD03882351F09927EE
:10F8D0009F938F938DE59FE09F938F93DF93CF93BB
:10F8E0001DCE81E69FE09F938F93DF93CF93FAC065
:10F8F0008091E203F3E5EF2EF5E8FF2E882309F06F
:10F9000053C08EE70E94818580916D0199279F9356
:10F910008F9380914406E82FFF27EE0FFF1FEB58CF
:10F92000F84F808191819F938F9380914306E82FB8
:10F93000FF27EE0FFF1FEB58F84F808191819F93B7
:10F940008F9387E69FE09F938F93FF92EF92E091D2
:10F95000FC03F091FD03099583E90E9481858DB731
:10F960009EB70A968DBF80914606E82FFF27EE0FBF
:10F97000FF1FEB58F84F808191819F938F93809167
:10F980004506E82FFF27EE0FFF1FEB58F84F808149
:10F99000918181589F4F9F938F938BE79FE09F9317
:10F9A0008F93FF92EF9241CE8EE70E9481858091E6
:10F9B000DC0299279F938F938091DB0299279F9375
:10F9C0008F938091DA0299279F938F938AE89FE023
:10F9D0009F938F93FF92EF92E091FC03F091FD03D0
:10F9E000099583E90E9481858DB79EB70A968DBFE0
:10F9F0008091DF0299279F938F938091DE02992750
:10FA00009F938F938091DD0299279F938F938EE927
:10FA10009FE09F938F93FF92EF92E091FC03F09110
:10FA2000FD0309952DB73EB7265F3F4F2DBF8AC016
:10FA30008091E803882309F485C08EE70E948185C0
:10FA400080912E0886FD11C082EB9FE09F938F93DB
:10FA500084E795E89F938F93E091FC03F091FD0379
:10FA600009950F900F900F900F908091AD069927F8
:10FA70008F709070892B89F081EC9FE09F938F931A
:10FA800084E795E89F938F93E091FC03F091FD0349
:10FA900009950F900F900F900F9080912E0882FF84
:10FAA00011C08BEC9FE09F938F9384E795E89F9321
:10FAB0008F93E091FC03F091FD0309950F900F9057
:10FAC0000F900F9080912E0883FD3CC080ED9FE049
:10FAD0009F938F9384E795E89F938F93E091FC0326
:10FAE000F091FD0309950F900F900F900F902AC091
:10FAF0000E9435718093300925C00091100A0630AC
:10FB000089F48091E203882319F01092E20303C084
:10FB100081E08093E20386E00E941D7187E00E94ED
:10FB20001D7108C0013031F40E9486850093DF0307
:10FB30001092DE031092100A05C01092DE0302C07C
:10FB40001092DF03E6E0CDB7DEB70C94DA8B4FB747
:10FB500028E130E0F8948091C9008F778093C90044
:10FB60008091C9008F7B8093C9008091C9008F7DEF
:10FB70008093C9005A9A52985B9A539A832F992777
:10FB80008093CD002093CC008091C8008260809348
:10FB9000C80080E18093C9008091CA008F7780936C
:10FBA000CA008091CA008F7B8093CA008091CA00EE
:10FBB0008091CA008F7E8093CA008091CA008860BD
:10FBC0008093CA008091C9008B7F8093C900809187
:10FBD000CA0084608093CA008091CA0082608093CA
:10FBE000CA008091C80087FF03C08091CE00F9CF82
:10FBF0008091C90080688093C90080910E0A84605A
:10FC000080930E0A4FBF08959091C603992341F443
:10FC10008F3031F49093E40380E58093C603089518
:10FC2000E091E403EF5FE093E403E83121F481E045
:10FC30008093E3030895E93120F089E18093E403A0
:10FC40000895FF27E950F64F80830895A0E0B0E0C3
:10FC5000ECE2FEE70C94BA8B91E0D92E82E0A82E5C
:10FC6000BD2CE12C01E0F02E80910E0A82FDB5C082
:10FC700080916F008F7D80936F00E091AA06EE2344
:10FC800051F0FF27EE0FFF1FEB58F84F8081918155
:10FC9000843691055CF48091D902883C20F48091EF
:10FCA000D9028C5E01C088EC8093D9028091F8095A
:10FCB000682F77278091E50381508093E5038F3F7C
:10FCC00031F41CE7C12E82E08093E50302C0C4E258
:10FCD000CC2E40E04C1508F07EC0EA2DFF27E950FD
:10FCE000F64F80818D2111F06E297F298D2D992766
:10FCF000880F991FD82E882319F4B1E0DB2EAD0CA4
:10FD0000EE0CFF1C20E0E21628E0F20609F061C0CC
:10FD1000A1E0EA2EF12CCB018050944065E070E028
:10FD20000E94628BAB2DBB27FD01EA0FFB1FEB5836
:10FD3000F84F808191819C01220F331F280F391FBA
:10FD4000260F371F37FF02C02D5F3F4FE901D595C2
:10FD5000C795D595C795CB0101968C179D0714F4CF
:10FD6000219706C061507040C617D7070CF4219642
:10FD70008091D902833CD8F08D010A0F1B1FF80136
:10FD8000EB58F84F80819181FE01E81BF90BCF0100
:10FD900063E070E00E94628BCB01880F991F860F91
:10FDA000971F0755184FF8019183808307C0AA0F4A
:10FDB000BB1FA755B84F11961C921E92EB2DFF2723
:10FDC000EE0FFF1FEB58F84FD183C08360E070E067
:10FDD000B3944F5F7FCF109240011092E303EAE0AB
:10FDE000CDB7DEB70C94D68B089508950024222752
:10FDF0003327442751E0BB27EE27FF27A0E1660FFA
:10FE0000771F881F991F001C221F331F441F660F76
:10FE1000771F881F991F001C221F331F441F2AF4BD
:10FE2000050E2B1F3E1F4F1F04C0051A2B0B3E0B48
:10FE30004F0B550FBB1FEE1F587F556047FD5250AB
:10FE4000AA95E9F6E695B7955795E695B79557952E
:10FE5000852F9B2F08952227332741E0552768E0FF
:10FE6000880F991F221F331F880F991F221F331FCE
:10FE70001AF4240F351F02C0241B350B440F551FE5
:10FE8000487F456037FD42506A9551F75695479532
:10FE900056954795842F0895AA2797FF04C080950B
:10FEA00090958A1F9A1F77FF04C0609570956A1F0E
:10FEB0007A1F669F9001779FA001679F300D411DBB
:10FEC0005A1F300D411D5A1F889FF001999F2E0F18
:10FED0003F1F401D511D899F300D411D5A1F300D80
:10FEE000411D5A1FCA01B901112480CF4FB720E428
:10FEF00030E0F8948091C9008F778093C900809199
:10FF0000C9008F7B8093C9008091C9008F7D809349
:10FF1000C9005A9A52985B9A539A832F99278093D3
:10FF2000CD002093CC008091C80082608093C800EF
:10FF300088E18093C9008091CA008F778093CA00BE
:10FF40008091CA008F7B8093CA008091CA008F7D08
:10FF50008093CA008091CA008F7E8093CA008091EE
:10FF6000CA00877F8093CA008091C9008B7F8093ED
:10FF7000C9008091CA0084608093CA008091CA0041
:10FF800082608093CA008091C80087FF03C080917F
:10FF9000CE00F9CF8091C90080688093C9004FBF1F
:10FFA00008950F931F93CF93DF93482F4F5F8931AD
:10FFB00008F08BC080917407841720F44F5F409342
:10FFC00074074150CB0183539B4268E170E00E946B
:10FFD000628BA42FBB27FD01EA0FFB1FEB58F84FE4
:10FFE000808191819B01281B390BC90137FF03C018
:10FFF000909581959F4F069794F48091D902883C03
:020000021000EC
:1000000030F48091D902865F8093D90208C088ECD1
:100010008093D90280916F008F7D80936F00FD01E6
:10002000EA0FFB1FEB58F84F808191819C01220F52
:10003000331F280F391F260F371F37FF02C02D5FD0
:100040003F4FE901D595C795D595C795CB01019649
:100050008C179D0714F4219706C061507040C61795
:10006000D7070CF421968091D902843BD8F08D01FA
:100070000A0F1B1FF801EB58F84F80819181FE0198
:10008000E81BF90BCF0163E070E00E94628BCB01AB
:10009000880F991F860F971F0755184FF8019183F6
:1000A000808307C0AA0FBB1FA755B84F11961C929B
:1000B0001E92E42FFF27EE0FFF1FEB58F84FD1835E
:1000C000C083443011F410924001DF91CF911F9111
:1000D0000F910895CF93DF932091110A822F9927D2
:1000E000807F9070409709F06CC02F3109F046C0B6
:1000F0008091120A8093EF032091140A2093F10358
:100100008091150A8093F003822F992790937607A8
:1001100080937507222309F054C080914306282F4D
:100120003327220F331FF901E755F84F1182108250
:1001300080914406A82FBB27AA0FBB1FFD01E755DE
:10014000F84F1182108280914606E82FFF27EE0FAC
:10015000FF1FCF018755984FEC01198218822B5849
:10016000384FE90119821882AB58B84F11961C928A
:100170001E92EB58F84F1182108223C0C22FCF700D
:10018000CA30F8F48091120A80933D0A8091130AD4
:1001900080933C0A8091140A80933F0A8091150A4B
:1001A00080933E0A60913C0A70913D0A8C2F0E9418
:1001B000D17F60913E0A70913F0A8C2F8F5F0E9421
:1001C000D17FDF91CF910895CF93C82F8F3F49F40E
:1001D0008091F2038F3F29F41092F4031092F303FD
:1001E00032C02091F403222339F4CF3111F485E099
:1001F00001C084E08093F5038091F5039091F303AF
:100200008217A0F4892F80958093F3038F3F19F410
:100210008EEF8093F3038091F303C81711F40E94CB
:100220006A801092F4031092F3030BC0E22FFF27B1
:10023000EF5EF54FC0832F5F2093F4039C0F9093E4
:10024000F303C093F203CF9108959091EE0393329C
:1002500040F4E92FFF27E75EF54F80839F5F90937F
:10026000EE030895833218F48D5F8093EE030895B2
:1002700090E2ECE1FAE08FE19193815087FFFCCFAF
:100280000895CF93CFB723E031E0F8948091C9006F
:100290008F778093C9008091C9008F7B8093C900BC
:1002A0008091C9008F7D8093C9005A9A52985B9AB9
:1002B000539A832F99278093CD002093CC0080916F
:1002C000C80082608093C80088E18093C900809153
:1002D000CA008F778093CA008091CA008F7B809379
:1002E000CA008091CA0080628093CA008091CA00CF
:1002F00080618093CA008091CA0088608093CA00A0
:100300008091C90084608093C9008091CA00846094
:100310008093CA008091CA0082608093CA00809155
:10032000C80087FF03C08091CE00F9CF8091C9003B
:1003300080688093C9008091C90080648093C9005F
:100340000E943881CFBFCF910895282F99278F70B1
:100350009070892B31F420958091ED03822B80934E
:10036000ED0308958091A201882309F44BC0809188
:10037000A10285FD04C08091A601882381F082E955
:100380008093190A83E280931A0A8091A601882338
:1003900009F485E580931B0A1092A60102C08093A0
:1003A000190A8091A3018F3071F48091ED030E94AE
:1003B0000070882341F081E98093190A80931A0A1A
:1003C00081E380931B0A1092A2018091C80085FFEF
:1003D000FCCF8091C9008F7E8093C9008091C900B5
:1003E0008E7F8093C9008091190A882311F48EEFC3
:1003F00001C08EE78093CE008091ED038093A3012E
:100400001092ED0308951F920F920FB60F921124D0
:100410008F939F93EF93FF939091A201992309F0FB
:1004200040C08091F603882361F48091190A8823E3
:1004300011F483E003C0813999F481E08093F603DD
:100440000FC0833099F48091190A882349F0909362
:10045000190A8091C9008E7F8093C9008EEF1EC05B
:100460008091C90081608093C9000EC0833261F41D
:100470008091C9008E7F8093C9008FEF8093CE005A
:1004800081E08093A20114C08091F603E82FFF273A
:10049000E75EF54F8F5F8093F60380818093CE00F7
:1004A00007C01092F6038091C90080618093C90053
:1004B000FF91EF919F918F910F900FBE0F901F9022
:1004C0001895EF92FF920F931F93CF93DF937C01C8
:1004D0008B01EA01452B39F0F80181918F01F70179
:1004E00009952197C9F7E6E0CDB7DEB70C94DA8B12
:1004F000EF92FF920F931F93CF93DF937C018B01B9
:10050000EA01452B41F0F8010F5F1F4F8491F7017D
:1005100009952197C1F7E6E0CDB7DEB70C94DA8BE9
:100520000F931F93CF938C01C62F161634F480E2DD
:10053000F8010995C1501C16D4F3CF911F910F916A
:1005400008950F931F93CF938C01C62F161634F482
:1005500080E3F8010995C1501C16D4F3CF911F9187
:100560000F910895A5E3B0E0E8EBF2E80C94B28BAC
:100570002E96EEADFFAD2E978824992454018091DC
:10058000E703882321F42C961FAE1EAE2C975EE461
:10059000452E512C4C0E5D1E6F01B60105C0153263
:1005A00039F00894C11CD11CF60114911123B9F73C
:1005B000A601461B570B31F02C968EAD9FAD2C97A4
:1005C0000E947882112309F46AC20894C11CD11CCC
:1005D000FF24FDA6FCA64FEFE42EF9A6F601089431
:1005E000C11CD11C1491153721F0812F80628837EE
:1005F000B1F4F0FE0AC0F20124E030E0420E531ED6
:1006000080809180A280B3800AC0F20142E050E075
:10061000440E551E808191814C01AA24BB241032C6
:1006200021F489A58823D1F61DC0133219F458E0AE
:10063000F52AD4CF1A3211F01D3291F41A3259F43E
:10064000F20182E090E0480E591EE081ECA7EE2313
:100650002CF6E195ECA790E1F92AAFEDFA22BECF96
:100660001B3211F419A7BACF1E32C1F5F601089456
:10067000C11CD11C14911A3279F4F20122E030E04D
:10068000420E531E408151813FEF4F3F530714F4F8
:100690004FEF5FEFE42EA2CF40E050E0812F805378
:1006A0008A30A0F4CA0133E0880F991F3A95E1F728
:1006B000840F951F480F591F410F511D4053504043
:1006C000F6010894C11CD11C1491E8CF8FEF4F3F65
:1006D000580714F44FEF5FEFE42E85CF103329F461
:1006E000F4FC7CCF90E2F92A79CF812F81538930B5
:1006F000D8F440E050E0CA0123E0880F991F2A9502
:10070000E1F7840F951F480F591F410F511D4053AA
:100710005040F6010894C11CD11C1491812F8053C4
:100720008A3048F34CA75FCF183619F4A4E0FA2AB0
:1007300055CF1C3619F4B1E0FB2A50CF133661F4C3
:100740003E010894611C711CF20122E030E0420E6F
:10075000531E808189833CC1143421F0143611F07A
:10076000193651F5143411F431E0F32AF0FE0AC0C1
:10077000F20144E050E0440E551E80809180A2803A
:10078000B3800CC0F20182E090E0480E591E8081D7
:1007900091814C01AA2497FCA094BA2CB7FE0AC000
:1007A000B094A09490948094811C911CA11CB11CC5
:1007B0008DE289A70AE06FC01F3411F01F3631F4B3
:1007C0001F3411F491E0F92A08E064C0103779F47D
:1007D000F201A2E0B0E04A0E5B1E808191814C01E3
:1007E000AA24BB2400E1B0E4FB2A18E753C0133766
:1007F000C1F5F20122E030E0420E531E60807180AC
:100800006114710489F43E010894611C711C88E232
:1008100089838EE6F301818385E78B838CE68C8365
:100820008D8389E28E831F82E7FC13C08E2D99276A
:1008300087FD9095AC0160E070E0C3010E947F8964
:10084000009729F0382E3618E3140CF0C3C03E2C64
:10085000C1C0F30101900020E9F731973E2E361810
:10086000B9C0153511F0153731F4153511F4F1E033
:10087000FF2A0AE00FC0183519F0183709F0A0C098
:1008800000E1F3FE07C081149104A104B10411F04A
:1008900020E4F22A19A6EDA6E7FC02C03FEDF32200
:1008A00089E2682E712C6C0E7D1E81149104A104C6
:1008B000B10421F44DA5442309F47BC0802F99276E
:1008C000AA27BB278EA79FA7A8ABB9AB202E33249E
:1008D00090E0891690E0990691E0A90690E0B906AB
:1008E00048F0C501B4012EA53FA548A959A90E9409
:1008F000758B17C0AFEF8A169104A104B10449F0BB
:1009000040F0C401B1010E944E8B9B014427552742
:1009100008C0882D602F0E94428B282F3327442740
:1009200055272AAB3BAB4CAB5DAB0A3059F48AA9D7
:10093000880F880F880F9AA9990F890F382D381BB7
:10094000832F10C0003139F48AA98295807F482D09
:10095000481B842F07C08AA9880F880F880F582D3D
:10096000581B852F90E02EA53FA548A959A98216AE
:100970009306A406B50608F091E08AA89BA8ACA847
:10098000BDA88A3010F4805D04C0895A183509F476
:100990008F7DD3018E933D01992309F099CF0830C3
:1009A00041F4F3FE06C0803321F080E3FD01829321
:1009B0003F01CE010196382E3618F8E23F0E0BC0EB
:1009C000112309F46CC03E010894611C711C198349
:1009D000B1E03B2E19A6032D2DA4231827FC2224B9
:1009E00089A5882311F00F5F02C0F6FC0E5F020D8F
:1009F000EF2CFF24C70180739070892B49F48CA5DC
:100A0000801B682F2C968EAD9FAD2C970E949082F4
:100A100089A5882331F041E050E0BE01675D7F4F3A
:100A20000AC0E6FE0EC080E38AA71BA742E050E0A2
:100A3000BE01665D7F4F2C968EAD9FAD2C970E94B8
:100A40006182C70180739070809749F48CA5801BE8
:100A5000682F2C968EAD9FAD2C970E94A182622D9F
:100A60002C968EAD9FAD2C970E94A182832D992745
:100A700087FD9095AC01B3012C968EAD9FAD2C9760
:100A80000E946182E4FE89CD2CA5201B2CA7622F39
:100A90002C968EAD9FAD2C970E9490827ECDE2E188
:100AA000CB5C0C94CE8B982F8091180A883A50F426
:100AB0008091180AE82FFF27E25DF64F93838F5F3E
:100AC0008093180A0895982F8091180A883A58F44C
:100AD0008091180AE82FFF27E25DF64F9068938314
:100AE0008F5F8093180A0895982F8091E8038823D8
:100AF00021F0892F0E9463850895892F0E945385D4
:100B00000895883A10F48093180A089580E090E2DE
:100B1000E1E3F9E091938F5F883AE0F308954FB7EE
:100B200021E830E0F8948091C9008F778093C90064
:100B30008091C9008F7B8093C9008091C9008F7D0F
:100B40008093C9005A9A52985B9A539A832F992797
:100B50008093CD002093CC008091C8008260809368
:100B6000C80088E18093C9008091CA008F77809384
:100B7000CA008091CA008F7B8093CA008091CA000E
:100B80008F7D8093CA008091CA008F7E8093CA00B7
:100B90008091CA00877F8093CA008091C9008460D9
:100BA0008093C9008091CA0084608093CA008091BC
:100BB000CA0082608093CA008091C90081608093DE
:100BC000C9008091C80087FF03C08091CE00F9CF93
:100BD0008091C90080688093C9004FBF3CE7309383
:100BE000D5082DE72093FA088EE88093D608109256
:100BF000EF081092EE081092D80830931D09209348
:100C00002D09109227091092260910922909109295
:100C1000280910922B0910922A0984EF91E09093F1
:100C200025098093240990932309809322099093A6
:100C300021098093200910921F0989E880931E09D9
:100C400010922C093093DA092093F6091092DC09EE
:100C50008AE88093DB091092DF091092DE09109276
:100C6000DD091092E1091092E2091092E309109255
:100C7000E4091092E6091092E7091092E80910922F
:100C8000E9091092ED091092EC091092EB0910920B
:100C9000EA093093FB0820931C091092FD088DE8A7
:100CA0008093FC088BE780932E0980E880932F09BE
:100CB000109230098091D80890E2E1E3F9E0919335
:100CC0008F5F883AE0F38DE78093D9090895CF9339
:100CD000C82F8091F703803879F48C2F0E94EB7134
:100CE0008093EA038091EA03882311F1C093170AE5
:100CF0008091EA038F5F12C08F37D1F48091100A80
:100D0000882329F48C2F80958F708093100A8EE2AF
:100D100099E09093EC038093EB038DEA8093EA03D0
:100D20008091C9008F7E8093C90082E08093E9039F
:100D3000C093F703CF9108953091E903332331F045
:100D40008091E90381508093E90308958091EA033B
:100D5000882381F14091EA039091F803413091F4A6
:100D6000292F3093F8038091C90080618093C900D6
:100D70008091E803882319F03093E80310C0409372
:100D8000E8030DC0E091EB03F091EC038191F09347
:100D9000EC03E093EB03282F980F9093F8038091D6
:100DA000C80085FFFCCF2093CE008091EA038150DC
:100DB0008093EA0308952FB740E0F894E0E0F0E074
:100DC00081E2809357009491E2E0F0E08093570035
:100DD0003491E4E0F0E08093570084912FBF9E317E
:100DE00099F4363941F4893011F441E00DC08A306C
:100DF00059F442E009C0373939F4863011F443E040
:100E000003C0853009F444E0842F992708959FB7E3
:100E1000F8948091C900877F8093C9008091C900B0
:100E20008F7E8093C9008091C9008F778093C9001D
:100E30008091C9008F7B8093C9008091C9008F7D0C
:100E40008093C90052985A9A53985B9A9FBF08950D
:100E50001F93CF93DF93182F8091E703882309F422
:100E6000A7C08091A101181709F4A2C08091E603E0
:100E7000882321F40E94DB868093E60382ED91E0D3
:100E800090933F0180933E018DE790E19F938F9374
:100E9000CFEBD4E1DF93CF93E091FC03F091FD031E
:100EA00009950F900F900F900F90812F9927AA27E7
:100EB000BB27FC01099778F5ED54FF4F2091FC0307
:100EC0003091FD030C94E98B89E790E102C080E743
:100ED00090E19F938F93DF93CF93F901099527C0FA
:100EE0008BE690E1F6CF83E690E1F3CF8BE590E1DE
:100EF0009F938F93DF93CF93F901099588ED91E04C
:100F000090933F0180933E0112C086E590E1E1CFCE
:100F10008AE890E1DECF80E990E19F938F93DF93A1
:100F2000CF93E091FC03F091FD03099510E00F9041
:100F30000F900F900F908091E603843011F0823073
:100F400011F50E940787812F8150833018F40E9489
:100F5000FB6C2CC0143019F40E94418127C015305D
:100F600019F40E94767F22C0183019F40E94F47E92
:100F70001DC0163019F40E948F8518C01730B1F4C7
:100F80000E94A77D13C0112389F086EA90E19F9308
:100F90008F938FEB94E19F938F93E091FC03F091FB
:100FA000FD0309950F900F900F900F901093A101E2
:100FB000DF91CF911F9108950F931F9381E080934C
:100FC000E7034091A001E6E0F0E120E030E05FE4DB
:100FD000849199272F5F3F4F829FB001839F700DAF
:100FE000929F700D112446275150319657FFF0CF34
:100FF0004093A001EEEDFFE020E030E057E2849165
:1010000099272F5F3F4F829FB001839F700D929F62
:10101000700D112446275150319657FFF0CF409361
:10102000A0018091E603882321F40E94DB8680934F
:10103000E6038091A001833459F088E190E029E231
:101040000FB6F894A895809360000FBE20936000BF
:1010500082EB92E89093FD038093FC030E94CC08FE
:1010600085E690E09F938F9388E590E09F938F9320
:101070001F921F92809101016AE00E94428B892F8A
:1010800099279F938F93809101010E94428B99270A
:101090009F938F9381EC90E19F938F930FEB14E1DB
:1010A0001F930F93E091FC03F091FD03099586E0F7
:1010B00090E19F938F931F930F93E091FC03F09126
:1010C000FD0309958EED9FE09F938F931F930F93E0
:1010D000E091FC03F091FD0309950E94CC0883EC9C
:1010E0008093810080916F00806280936F008DB744
:1010F0009EB746968DBF1F910F9108958091A806C7
:101100008D3338F08091490887FD03C08CE38093CC
:10111000A80680915806882331F08055853618F04E
:101120008FE78093580608958091E703882309F498
:1011300077C08091F90381508093F903882309F0E7
:1011400053C089E18093F9038091A8068E3338F06B
:101150008091490887FD03C08DE38093A8068091A4
:10116000D902823820F58091A2029091A302885E74
:10117000934020F08091D408843620F41092FB0331
:101180001092FA038091FA039091FB03009739F1D2
:1011900001979093FB038093FA03419728F1809184
:1011A000490884FF21C08091A00284601BC0809107
:1011B000D902853BC8F09091A80684E1989FC001B0
:1011C000112440962091FA033091FB032817390728
:1011D00030F42F5F3F4F3093FB032093FA0380914D
:1011E000A0028B7F8093A0029091A101963019F408
:1011F0000E949C860FC08091A401882321F0815019
:101200008093A401089586E98093A401943011F499
:101210000E94B2818091A001833411F01092E70303
:1012200008951F920F920FB60F9211242F933F93A0
:101230004F935F936F937F938F939F93AF93BF93DE
:10124000EF93FF932091CE008091B0018823B1F0FD
:101250002093C6008091B0018230B9F52F3FA9F5E7
:101260008FEF94E3ACE0B0E0C297A109B109B7FFFA
:10127000FBCF80913F048093CE0027C09091A101C5
:10128000892F8150833020F4822F0E94566D1DC01B
:10129000943021F4822F0E94A58117C0953021F44B
:1012A000822F0E94E48011C0983021F4822F0E9486
:1012B000F57E0BC0963021F4822F0E94678605C010
:1012C000973019F4822F0E94047EFF91EF91BF9115
:1012D000AF919F918F917F916F915F914F913F91CE
:1012E0002F910F900FBE0F901F901895FB01DC01FE
:1012F00002C005900D9241505040D8F70895FC016E
:101300004150504030F001900616D1F73197CF018F
:101310000895882799270895A0E0B0E0E2E9F9E868
:101320000C94BA8B6C017B01EA01590121978FEF74
:10133000CF3FD80789F086010894C11CD11CC70192
:101340000894E11CF11CF5010995F80180832197AF
:10135000FFEFCF3FDF0779F7EAE0CDB7DEB70C94B8
:10136000D68BCF92DF92EF92FF920F931F937C0167
:101370006B01FB010995082FC7010196F60109953C
:10138000182FC8011F910F91FF90EF90DF90CF9021
:101390000895A0E0B0E0EFECF9E80C94BC8B8C0170
:1013A0007B01EA01690121978FEFCF3FD80771F0E8
:1013B000F70121917F01C8010F5F1F4F622FF601D6
:1013C00009952197FFEFCF3FDF0791F7E8E0CDB711
:1013D000DEB70C94D88BCF92DF92EF92FF920F93EF
:1013E0001F936C018B017A01FA010995812F9927CE
:1013F000682FC6010196F70109951F910F91FF9083
:10140000EF90DF90CF9008955058BB27AA270ED0B9
:10141000E0C0D1D030F0D6D020F031F49F3F11F4AD
:101420001EF4C6C00EF4E095E7FBBCC0E92FE2D085
:1014300080F3BA17620773078407950718F071F4F1
:101440009EF5FAC00EF4E0950B2EBA2FA02D0B01DD
:10145000B90190010C01CA01A0011124FF27591BF9
:1014600099F0593F50F4503E68F11A16F040A22FFF
:10147000232F342F4427585FF3CF46953795279570
:10148000A795F0405395C9F77EF41F16BA0B620B6F
:10149000730B840BBAF09150A1F0FF0FBB1F661FB6
:1014A000771F881FC2F70EC0BA0F621F731F841FF9
:1014B00048F4879577956795B795F7959E3F08F01F
:1014C000B3CF9395880F08F09927EE0F97958795DE
:1014D000089598D088F09F5790F0B92F9927B75169
:1014E000A0F0D1F0660F771F881F991F1AF0BA95E8
:1014F000C9F712C0B13081F09FD0B1E008959CC00F
:10150000672F782F8827B85F39F0B93FCCF38695DD
:1015100077956795B395D9F73EF49095809570953A
:1015200061957F4F8F4F9F4F0895E89409C097FBB7
:101530003EF490958095709561957F4F8F4F9F4FAA
:101540009923A9F0F92F96E9BB279395F6958795EE
:1015500077956795B795F111F8CFFAF4BB0F11F4B1
:1015600060FF1BC06F5F7F4F8F4F9F4F16C0882358
:1015700011F096E911C0772321F09EE8872F762F8E
:1015800005C0662371F096E8862F70E060E02AF0CF
:101590009A95660F771F881FDAF7880F96958795BB
:1015A00097F9089597F99F6780E870E060E00895E3
:1015B0009FEF80EC089500240A941616170618066B
:1015C0000906089500240A94121613061406050647
:1015D0000895092E0394000C11F4882352F0BB0FD8
:1015E00040F4BF2B11F460FF04C06F5F7F4F8F4F3B
:1015F0009F4F089557FD9058440F551F59F05F3F76
:1016000071F04795880F97FB991F61F09F3F79F024
:1016100087950895121613061406551FF2CF4695A6
:10162000F1DF08C0161617061806991FF1CF869528
:101630007105610508940895E894BB27662777270C
:10164000CB0197F90895629FD001739FF001829FAB
:10165000E00DF11D649FE00DF11D929FF00D839F41
:10166000F00D749FF00D659FF00D9927729FB00DDE
:10167000E11DF91F639FB00DE11DF91FBD01CF01F1
:1016800011240895991B79E004C0991F961708F05A
:10169000961B881F7A95C9F780950895AA1BBB1BD6
:1016A00051E107C0AA1FBB1FA617B70710F0A61B62
:1016B000B70B881F991F5A95A9F780959095BC0183
:1016C000CD01089597FB092E07260AD077FD04D097
:1016D000E5DF06D000201AF4709561957F4F0895DC
:1016E000F6F7909581959F4F0895A1E21A2EAA1BB7
:1016F000BB1BFD010DC0AA1FBB1FEE1FFF1FA217C2
:10170000B307E407F50720F0A21BB30BE40BF50BBE
:10171000661F771F881F991F1A9469F76095709547
:10172000809590959B01AC01BD01CF01089597FB79
:10173000092E05260ED057FD04D0D7DF0AD0001C95
:1017400038F450954095309521953F4F4F4F5F4F5E
:101750000895F6F790958095709561957F4F8F4F1E
:101760009F4F08952F923F924F925F926F927F9278
:101770008F929F92AF92BF92CF92DF92EF92FF92A1
:101780000F931F93CF93DF93CDB7DEB7CA1BDB0B4D
:101790000FB6F894DEBF0FBECDBF09942A883988F2
:1017A00048885F846E847D848C849B84AA84B984F9
:1017B000C884DF80EE80FD800C811B81AA81B98105
:1017C000CE0FD11D0FB6F894DEBF0FBECDBFED0119
:1017D0000895EE0FFF1F0590F491E02D0994FFCFBF
:1017E0005E0A010164FF01FFFFC01FC01F0101016C
:1017F000737373FF03007D0000C409C40964001003
:101800004661737400004E6F726D616C000045613B
:101810007379000051756164726F00006400D20139
:1018200001200B050000ECFF000204060708080871
:101830000706040200FEFCFAF9F8F8F8F9FAFCFED3
:10184000000204060708086440415A4664640A021C
:10185000969696960840403A10FB30380132FF03C6
:10186000780090D0030090D0030032002064FFFF86
:1018700064200B0A0D0B0C0E0B0F10FA2001010156
:0618800070FF010F64007F
:00000001FF
